:020000040000FA
:1000000078530020D5000000EF000000DFD2000090
:1000100000000000000000000000000000000000E0
:10002000000000000000000000000000F3000000DD
:100030000000000000000000F50000001D7A010033
:10004000F9000000F9000000BD440100C9440100AE
:10005000CD450000318001008985010095850100B2
:10006000C9E50000D1E50000F5600100FD60010078
:1000700051D3000059D300001980010021800100F4
:10008000298001009BE400003980010041800100CB
:1000900049800100AD440100A1AD0100F15401000F
:1000A000850C0000B544010089AD010091AD01004F
:1000B000F7E6000093E4000099520000193A0000AE
:1000C0000348854600F09AFD00480047770C000081
:1000D0007853002009480A4A002100A1814200D932
:1000E0000244084802600848804708480047FEE785
:1000F000FEE7FEE7FEE7FEE7FEE700000000002067
:100100000000000008ED00E0417F0100C100000098
:1001100030B50B46014600202022012409E00D469F
:10012000D5409D4205D31D469540491B2546954027
:1001300040191546521E002DF1DC30BD70B500246B
:100140002546002801DA01244042002901DA012570
:100150004942FFF7DDFFAC4200D04042002C00D006
:10016000494270BDF0B51FB40646002082B0054676
:100170004024019100901BE0019922460F46304631
:1001800000F036FC049A059B801A994110D3104662
:100190001946224600F01CFC361A8F410197224670
:1001A00001200021009F00F013FC38184D41009001
:1001B0002046641E0028DFDC019B00982946324659
:1001C00007B0F0BD38B50446C0681821401E48434A
:1001D000A16840183C214843616840183C214843CD
:1001E0002168451860690C2148432169401869213C
:1001F000C900401A3021FFF7A1FF114A50434219AC
:10020000084600921A2902DB0E49511800910C2170
:10021000FFF794FF0C4A5043009A801800900B4857
:1002200006E0491E425C074B5A43009BD2180092DD
:100230000029F6DC2146684600F006FC009838BD2F
:10024000801F8607805101008033E1013C2B0200B2
:1002500003460B439B0703D009E008C9121F08C0DF
:10026000042AFAD203E00B780370401C491C521E8A
:10027000F9D27047D2B201E00270401C491EFBD295
:1002800070470022F6E710B513460A4604461946A1
:10029000FFF7F0FF204610BD421E5378521C002B82
:1002A000FBD10B781370491C521C002BF9D17047FD
:1002B000421C0178401C0029FBD1801A704703467C
:1002C0000A780270401C491C002AF9D11846704770
:1002D0000321001D401E037812021A43491EF9D55E
:1002E00010467047034610B508330722040E090272
:1002F00021435B1E1C7800022043521EF6D510BD20
:10030000034603220870000A491C521EFAD51846FB
:10031000704770B504460D46072310700E06000A9C
:100320003043090A521C5B1EF7D52046294670BD92
:10033000F8B502464A40D40F42004B0052085B0811
:100340009A4202D20246084611464A0023D0C30D03
:100350004A00DDB2120EAD1A202D35DA490201260F
:10036000490AF6058A19002C00D0524220214F1B61
:100370001146B9402A411018C20D9A4221D0002CD2
:1003800017D0012D08DCDA05801AD20F8019D207A8
:10039000DBB200F09BFBF8BDDA05801A01234000B8
:1003A0001B06C01880185A428018CA0F1043490013
:1003B00007E04908C2071143DA05801A801940088E
:1003C000801800F07BFBF8BD61000122511A001B70
:1003D000F7E70122D2075140AAE70122D207504095
:1003E000A6E7024670B54A40D30FDB0740002DD088
:1003F0004A002AD0010E140E000212020919400A06
:10040000520A8418E50104465443000A120A2E04D5
:100410005043A4194219200CC543AA18120C0125F7
:10042000AD03521C521912047F39240400D0521C0F
:10043000104301D44000491EC2B20C06C009201866
:10044000401C4008802A02D003E0002070BD400814
:100450004000002900DA0020184370BD70B5024644
:100460004A40D50F40004A00ED07400852080028D6
:1004700014D0002A12D0C40DD30D41020120C005B2
:100480005202490A520AE41A091812187D3491429C
:1004900001D3641C00E04900002C01DA002070BD8B
:1004A0000023914201D3891A0343400849000028E0
:1004B000F7D100290AD0914202D10121C90705E0F4
:1004C000914201D2012101E00121C943E005C01898
:1004D000401900F0F3FA70BDF0B5074608465840E1
:1004E00087B0C00F049048000E46590040084908E4
:1004F000BC1A884105D2384631461E4617460B467F
:1005000002465800400810434CD0300D039040057F
:100510005900400D490D0590401A0290402872DAAA
:1005200018030121000B090508430190049800926B
:10053000002805D001995242002088410092019084
:10054000029840210A1A0199009800F041FA0546E4
:100550000C466B4607CB00F05CFAC0197141039A58
:100560000E0D0023D71756401A467A40164344D042
:10057000049A002A2DD0029A012A039A15DC12054A
:10058000C01A914101263605001C7141D20F059E0B
:10059000D2070093019202962A46234600F0DCFA25
:1005A00007B0F0BD38463146FAE71605224A0F4635
:1005B000B218C01AB74101210905001C4F410018AB
:1005C0007F41114618187941E20F10436D196441BB
:1005D00013E0E2076D0815436408C2071443039A49
:1005E00001261205C01A91413605001C7141CE0743
:1005F000400830434908C01851412A46234600F0BC
:100600009EFACDE7FFE7049801224000C117121AB5
:1006100000238B4104983146C417381AA141EEE7F4
:1006200030B40124E407634030BC55E730B4012402
:10063000E407614030BC4FE70000E0FFF0B51FB4B5
:1006400088B00B990998002448400999C00F4900C7
:1006500049080991C0070B990090490049080B917E
:1006600009990898A64608431CD00B990A98084394
:1006700018D0099801244000420D4800410D099806
:1006800024050003000B204309900B980003000B86
:1006900020430B9050181C4940180022019014462A
:1006A000104605E0002001460DB0F0BD032801DA38
:1006B000034600E003239C46C11A0AAE0AE05F002D
:1006C00008ADED5B4F00F75B7D430027AA187C4126
:1006D000491C5B1E6145F2DD410004AB5A52210406
:1006E000120C0A43240C401C0828DFDB01980290FE
:1006F0000099704601910090059B049A079906980D
:1007000000F02AFAD0E700000DFCFFFFF0B50C4620
:100710005C4085B0E40FE40703944C0000266408B5
:1007200059009446490802460296224321D0624667
:100730000A431ED06200570D4A000E032303550DD5
:10074000012402462C492405781B1B0B360B40184C
:1007500023432643614600901C46501AB44103D3FC
:100760000098401C009002E0921800985B4100281D
:1007700003DA0020014605B0F0BD00200121090583
:100780000746864611E064461D46141BB54106D354
:100790006546521BB341744607430C43A646CD073A
:1007A00040084908284392185B4105460D43EAD1A9
:1007B0001046184313D06046194650407140084314
:1007C00006D06046101AB34106D20122002306E08B
:1007D00000220123DB0702E00122D24353100098DC
:1007E00074460105381C6141029C039D0019694152
:1007F00000F0A5F9BFE70000FD030000C217C10F1C
:10080000504010B54018CA079623002100F05EF949
:1008100010BD10B500229623114600F057F910BD07
:100820000EB5C217C10F5040CA0740180021054B32
:100830000293019200910A460B4600F08DF903B035
:1008400000BD0000330400000EB5054902910021EF
:1008500000910A460B46019100F07EF903B000BDFD
:1008600033040000410040020122400AD205090E73
:1008700080187F2901DA00207047962903DC962230
:10088000511AC840704796398840704741000A0E97
:1008900040020121400AC90510B540187F2A02DA3A
:1008A0000020014610BD0021962A03DC96239A1AE7
:1008B000D04010BD963A00F08BF810BD4A000903F5
:1008C0000123090B1B051943094B10B5520D9A4220
:1008D00001DA002010BD064B34339A4203DC9A1A29
:1008E00000F086F810BD03495118884010BD000083
:1008F000FF030000CDFBFFFFC20FD20740004008FE
:100900000BD0C10D0723DB01C91840020905400ABD
:100910001143C20840071143704700200146704749
:1009200010B5002904DB0124E40740428C41214634
:10093000002B04DB1C460123DB075242A3418B4200
:1009400000D1824210BD000010B5002904DB012453
:10095000E40740428C412146002B04DB1C46012366
:10096000DB075242A341994200D1904210BD0000E2
:10097000CB0FDB07490010B5490802460A4307D0F0
:100980000A0D07240903E401090B121B002A01DCEC
:10099000002010BDC900440F0C43C100E018D2056F
:1009A000801800F08BF810BD0122D207002800DB70
:1009B000101A002900DB511A814270470122D20728
:1009C000002800DB101A002900DB511A884270470A
:1009D00010B5202A04DB0146203A9140002010BDCA
:1009E000914020239C1A0346E3401943904010BDD8
:1009F00010B5202A04DB0846203AD040002110BD63
:100A00000B46D340D0402024A21A914008431946F7
:100A100010BD10B5202A06DBCB170846203A10413E
:100A2000C1170B4306E00B461341D0402024A21A05
:100A300091400843194610BD10B5024900F004F872
:100A400010BD00004C43002070B50C4600683C21EE
:100A5000FFF75EFB21603C21FFF75AFB6160182124
:100A6000FFF756FB0546A1600721001DFFF750FB6D
:100A7000A1610F48A90008180E49FFF749FB02467B
:100A8000443288086261E0613B2802D3910700D0BC
:100A9000401C0021084B0A462161995C814203D821
:100AA000401A521C2261F8E7401CE060204670BDED
:100AB0006C0B0000B5050000482B0200002904DA89
:100AC000401C490001D140084000704770B4002428
:100AD000050C05D11024000402D1002921D01124D5
:100AE000050E01D100020834050F01D10001241DBB
:100AF000850F01D18000A41C002801DB4000641C8C
:100B0000002908D020252E1B0D46F540A14000D01D
:100B100001212943084301061B1B000ADB1D02D5E6
:100B2000002070BC7047DB05181880180029F8DA1F
:100B3000401C4900F5D170BC40084000704710B51A
:100B4000002B08DA0024401C614192185B411A43D3
:100B500001D14008400010BDF0B51FB482B0054679
:100B60000C0003D008461AF093FA02E01AF090FA4B
:100B700020300246009021462846FFF729FF049BBB
:100B8000059A04460F4618431143084314D01846EB
:100B900010431BD0009840210A1A18460599FFF708
:100BA00027FF05460E46009A05990498FFF710FFA7
:100BB000084305D0012004E02046394607B0F0BDC7
:100BC0000020C11705430E432C43374300990E986C
:100BD0006305401A7905E40A00220C43FD0A0A3035
:100BE00002D500200146E9E70105101969410C9C76
:100BF0000D9D00196941FFF7A2FFDFE7064C0125B3
:100C0000064E05E0E36807CC2B430C3C98471034B4
:100C1000B442F7D3FFF758FA542D0200742D0200A6
:100C200070B58C180578401C6B075B0F01D10378F9
:100C3000401C2A1106D10278401C03E006780E7091
:100C4000401C491C5B1EF9D12B0705D40023521E02
:100C50000DD40B70491CFAE70378401CCB1A921C88
:100C600003E01D780D70491C5B1C521EF9D5A14292
:100C7000D8D3002070BD10B517F062F91FF02EFF19
:100C8000002010BD10B5C046C046C046C04610BDCD
:100C9000F7B58AB00D460595059D2846E917090F59
:100CA00009180905090E0491002728E0002407E02F
:100CB000380101190A98405C69460855601CC4B2A5
:100CC000102CF5DB002605E00C98805D06A9885500
:100CD000701CC6B2102EF7DB012206A968461AF076
:100CE00005FB002407E06846015D380102190A98F7
:100CF0008154601CC4B2102CF5DB781CC7B2049878
:100D00008742D3DB0DB0F0BDFFB58DB014460D9812
:100D1000002802D0012854D154E025462C46204614
:100D2000E917090F09180911491C09050E0C301B98
:100D3000C0B2089008980790E8B2069007E0069ABB
:100D40000E99079888540698401CC0B206900698E1
:100D5000B042F4DB002005902CE0002708E0059865
:100D60000001C1190E98405C01A9C855781CC7B292
:100D7000102FF4DB002705E01098C05D09A9C855C5
:100D8000781CC7B2102FF7DB002209A901A81AF0BE
:100D9000ADFA002708E001A8C15D05980001C2195D
:100DA0000E988154781CC7B2102FF4DB0598401CB4
:100DB000C0B20590F117090F89190A1105998A42E5
:100DC000CBDC53E025462C462046E917090F0918CD
:100DD0000911491C09050E0C301BC0B20890089877
:100DE0000790069507E0069A0E990798885406988A
:100DF000401C80B206900698B042F4DB00200590BB
:100E00002CE0002708E005980001C1190E98405C0D
:100E100001A9C855781CC7B2102FF4DB002705E0E4
:100E20001098C05D09A9C855781CC7B2102FF7DB10
:100E3000002209A901A81AF059FA002708E001A820
:100E4000C15D05980001C2190E988154781CC7B283
:100E5000102FF4DB0598401CC0B20590F117090F64
:100E600089190A1105998A42CBDC00BF00BF11B075
:100E7000F0BD000010B50446454800780A3803006C
:100E80001AF01DF90B070D17212B353F49535F69E8
:100E90007F002B2C02D10B203D49087075E0432CBC
:100EA00003D10C203A49087002E00A203849087042
:100EB0006BE0452C03D10D203549087002E00A2073
:100EC0003349087061E0522C03D10E20304908707C
:100ED00002E00A202E49087057E0452C03D10F206C
:100EE0002B49087002E00A20294908704DE0472C80
:100EF00003D110202649087002E00A202449087016
:100F000043E03A2C03D111202149087002E00A2065
:100F10001F49087039E0202C03D112201C490870A9
:100F200002E00A201A4908702FE0302C05DB332C30
:100F300003DC13201649087002E00A2014490870E7
:100F400023E02C2C03D114201149087002E00A2060
:100F50000F49087019E020463038C1B2012020F056
:100F6000C1FC312C01D0352C07D10320C0430949E5
:100F7000087500200649087002E00A20044908703C
:100F800003E00A200249087000BF00BF10BD000046
:100F9000A8060020AF2E002010B50446384800787F
:100FA0000A3803001AF08BF809060C16202A343E82
:100FB000485266002B2C02D10B20314908705DE0AD
:100FC000432C03D10C202E49087002E00A202C4942
:100FD000087053E0472C03D10D202949087002E026
:100FE0000A202749087049E0412C03D10E202449EA
:100FF000087002E00A20224908703FE0542C03D117
:101000000F201F49087002E00A201D49087035E0D2
:10101000542C03D110201A49087002E00A20184904
:1010200008702BE03A2C03D111201549087002E01A
:101030000A201349087021E0202C03D11220104906
:10104000087002E00A200E49087017E02046303888
:10105000C1B2022020F046FC312C07D10320C0434E
:101060000849087500200649087002E00A20044972
:10107000087003E00A200249087000BF00BF10BDDD
:10108000A8060020AF2E00202B4909780A2902D09B
:101090000B2944D112E00021284A117030280CDBC2
:1010A00039280ADC11460A780978491C234B197043
:1010B000234988540B21204A11703AE030280ADB7A
:1010C000392808DC1D490A780978491C1B4B19701E
:1010D0001B49885422E04B280DD10021174A11707A
:1010E00000221749CA730A21134A11700321C94308
:1010F000144A117512E0114909780F2904DB032104
:10110000C943104A117503E00221C9430D4A117504
:1011100000220B49CA730A21074A117009E00A210B
:10112000054A11700021054A1170C91E054A117542
:1011300000BF00BF70470000A8060020DF060020A7
:10114000B8230020AF2E002070B50446B2480078C6
:101150000A38030019F0B3FF2C171D27313B455BFC
:101160006597A1ABB5BBC9E0F8FEEDECEBEAEAEAA6
:10117000EAEAEAEAEAEAEAEAEAEAEAEAEAEAEAEACF
:10118000EA6F79838DEA2B2C02D10B20A2490870DB
:101190003FE14D2C03D10C209F49087002E00A204A
:1011A0009D49087035E1492C03D10D209A490870FA
:1011B00002E00A20984908702BE1502C03D10E2040
:1011C0009549087002E00A209349087021E14C2CEF
:1011D00003D10F209049087002E00A208E49087060
:1011E00017E1572C06D100218C48817210208A49C2
:1011F00008700BE0452C06D101218848817232200D
:101200008549087002E00A208349087001E1522CE8
:1012100003D111208049087002E00A207E4908703D
:10122000F7E0492C03D112207B49087002E00A2024
:1012300079490870EDE0582C03D1332076490870C5
:1012400002E00A2074490870E3E0452C03D1342001
:101250007149087002E00A2071490870D9E0432CF6
:1012600003D135206C49087002E00A206A490870F1
:10127000CFE0552C03D112206749087002E00A2004
:1012800065490870C5E0542C03D1132062490870E9
:1012900002E00A2060490870BBE0452C03D114200D
:1012A0005D49087002E00A205B490870B1E03A2C01
:1012B00003D115205849087002E00A2056490870E9
:1012C000A7E0302C02D1162053490870A1E02C2C45
:1012D0000AD11720504908700020504988710A210E
:1012E0004E48001FFEF7CDFF93E02C2C10D0302C81
:1012F00011DB392C0FDC4948807909280BDA474883
:1013000081798079401C454A9071101F445402E055
:101310001820414908707CE02C2C14D13F48807A79
:10132000002809D119203C4908700CE070E027E042
:101330001CE015E00EE007E03848807A012802D171
:101340001A203549087064E02C2C02D11A20324949
:1013500008705EE02C2C02D11B202F49087058E049
:101360002C2C02D11C202C49087052E02C2C06D1C8
:101370001D202949087000212A488172C17248E065
:101380002C2C3BD00D2C39D02649C87A897A000202
:10139000084301218902884228DA20480838FEF7EC
:1013A00097FF451C1D4908392846FEF7A9FF302C38
:1013B00001DB392C07DD412C01DB462C03DD612CE0
:1013C00025DB662C23DC1748C17A807A09020143A9
:1013D000144AD07A927A00021043401C82B211481B
:1013E0008272120AC2720C30445410E000210D487F
:1013F0008172C1720A200849087008E0002007497C
:10140000487201202039C8750A200349087000E09D
:1014100000BF00BF70BD0000ED060020CF2E0020F1
:10142000A8060020AF28002000B52F4909780A3906
:101430000B0019F044FE08050B151F29333D4752D8
:101440002B2802D10B21284A11704AE0432803D1EE
:101450000C21254A117002E00A21234A117040E054
:10146000532803D10D21204A117002E00A211E4A9F
:10147000117036E0432803D10E211B4A117002E09F
:101480000A21194A11702CE04F2803D10F21164A66
:10149000117002E00A21144A117022E04E2803D193
:1014A0001021114A117002E00A210F4A117018E050
:1014B000202803D111210C4A117002E00A210A4AA6
:1014C00011700EE0312804D10321C943074A117578
:1014D00002E00A21044A117003E00A21024A117055
:1014E00000BF00BF00BD0000A8060020AF2E0020F6
:1014F00000B5424909780A390B0019F0E0FD0A06E7
:10150000101A242E38424A5D6A782B2803D10B2109
:101510003A4A117002E00A21384A11706BE0432800
:1015200003D10C21354A117002E00A21334A1170AF
:1015300061E0532803D10D21304A117002E00A21E5
:101540002E4A117057E0512803D10E212B4A1170F9
:1015500002E00A21294A11704DE03A2803D10F21F7
:10156000264A117002E00A21244A117043E0202823
:1015700003D11021214A117002E00A211F4A117083
:1015800039E0014630391E4A117011211B4A117091
:1015900031E02C2803D11221184A11700BE01849B0
:1015A00009780A2251430246303A8918144A1170C8
:1015B0001221124A11701EE04F2809D113210F4A3F
:1015C00011700F4909781F2902DD00210C4A1170A2
:1015D00011E04B2807D10321C9430A4A11750A219A
:1015E000064A117002E00A21044A117003E00A2140
:1015F000024A117000BF00BF00BD0000A806002015
:10160000AE060020AF2E002070B50446D04800780A
:101610000A38030019F053FD0C070D17212B353E36
:101620005F80A0C0E0F32B2C02D10B20C8490870CA
:101630008BE1432C03D10C20C549087002E00A203D
:10164000C349087081E1432C03D10D20C0490870C3
:1016500002E00A20BE49087077E14C2C03D10E202D
:10166000BB49087002E00A20B94908706DE14B2CB3
:1016700003D10F20B649087002E00A20B44908706F
:1016800063E1222C05D11020B14908700020B14936
:1016900008705AE12F2C10D0302C1BDB392C19DCB0
:1016A000AC4800780A214843AA49087020463038DF
:1016B00009784018A74908700CE0A649097808463F
:1016C0006430A549FEF71CFE0020A24908701120D5
:1016D0009F49087039E12F2C10D0302C1BDB392C9E
:1016E00019DC9C4800780A2148439A490870204632
:1016F000303809784018974908700CE09549097806
:10170000481E9549091FFEF7FBFD0020914908700E
:1017100012208F49087018E12C2C10D0302C1ADBC5
:10172000392C18DC8B4800780A2148438949087015
:101730002046303809784018864908700BE0864901
:10174000083984480078FEF7DBFD002081490870E5
:1017500013207F490870F8E03A2C10D0302C1ADBA7
:10176000392C18DC7B4800780A21484379490870F5
:101770002046303809784018764908700BE07649E1
:101780000C3974480078FEF7BBFD002071490870E1
:1017900014206F490870D8E03A2C10D0302C1ADB96
:1017A000392C18DC6B4800780A21484369490870D5
:1017B0002046303809784018664908700BE06649C1
:1017C000103964480078FEF79BFD002061490870DD
:1017D00015205F490870B8E0222C11D0302C0DDBA9
:1017E000392C0BDC5B4800780A21484359490870C2
:1017F000204630380978401856490870A0E0A0E02B
:101800005549143953480078FEF77AFD5248FEF7DF
:101810005FFD0546643D50492846FEF771FD4E4880
:10182000001FFEF755FD451C4B49091F2846FEF7D2
:1018300067FD49481438FEF74BFD05460A21FEF7BF
:101840007DFC060144481438FEF742FD05460A2196
:10185000FEF774FC0E4341498E713F481038FEF785
:1018600037FD05460A21FEF769FC06013A481038A3
:10187000FEF72EFD05460A21FEF760FC0E433749B0
:101880004E7135480C38FEF723FD05460A21FEF758
:1018900055FC060130480C38FEF71AFD05460A21B2
:1018A000FEF74CFC0E432D490E712B480838FEF70D
:1018B0000FFD05460A21FEF741FC060126480838BF
:1018C000FEF706FD05460A21FEF738FC0E432349C4
:1018D0008E702148001FFEF7FBFC05460A21FEF72B
:1018E0002DFC06011C48001FFEF7F2FC05460A21EC
:1018F000FEF724FC0E4319494E701748FEF7E8FC2A
:1019000005460A21FEF71AFC06011348FEF7E0FC23
:1019100005460A21FEF712FC0E4310490E700846D8
:101920000078232802DB084614F0A5FA00200949B4
:1019300008700A20064908700320C043084908754A
:1019400003E00A200249087000BF00BF70BD00001C
:10195000E1060020E20600202D2F0020E3060020F3
:10196000AF2E00202E4909780A2906D00B290ED067
:101970000C2916D00D294DD11CE0492803D10B218B
:10198000274A117002E00A21254A117046E04428D6
:1019900003D10C21224A117002E00B21204A117060
:1019A0003CE03A2805D100211E4A11700D211C4A45
:1019B000117033E0522823D04B2814D0302801DB9B
:1019C000392803DD412824DB462822DC1549097823
:1019D00015291EDA13490A780978491C114B197028
:1019E0001149885415E000210E4A117000220E4959
:1019F0000A75111F0D4A11750A21094A117008E074
:101A00000021084A1170C91E084A11750A21044AAA
:101A1000117003E00A21024A117000BF00BF704735
:101A2000A8060020EA060020C8230020AF2E0020D0
:101A300000B5344909780A390B0019F040FB070555
:101A40000F19232D37415D002B2803D10B212D4A7F
:101A5000117002E00A212B4A117051E0432803D192
:101A60000C21284A117002E00A21264A117047E031
:101A7000472803D10D21234A117002E00A21214A8F
:101A800011703DE0532803D10E211E4A117002E06F
:101A90000A211C4A117033E04E2803D10F21194A44
:101AA000117002E00A21174A117029E03A2803D187
:101AB0001021144A117002E00A21124A11701FE02D
:101AC0004B280CD0302816DB392814DC0E490A7854
:101AD0000978491C0C4B19700C4988540BE0002103
:101AE000094A11700A21074A117000220749CA7376
:101AF000111F074A117503E00A21024A117000BF45
:101B000000BF00BDA8060020E0060020A82300209A
:101B1000AF2E002000B53D4909780A390B0019F0B5
:101B2000CEFA0A06101A242E384248525C6E452816
:101B300003D10B21354A117002E00A21334A11709A
:101B400061E0562803D10C21304A117002E00A21CD
:101B50002E4A117057E0452803D10D212B4A1170F0
:101B600002E00A21294A11704DE04E2803D10E21CE
:101B7000264A117002E00A21244A117043E05428D9
:101B800003D10F21214A117002E00A211F4A11706E
:101B900039E03A2803D110211C4A117002E00A21D1
:101BA0001A4A11702FE0302802D11121174A117002
:101BB00029E02C2803D11221144A117002E00A21D5
:101BC000124A11701FE0312803D113210F4A1170FE
:101BD00002E00A210D4A117015E0352807D10321D2
:101BE000C9430B4A11750A21084A117006E0022107
:101BF000C943074A11750A21044A117003E00A21FA
:101C0000024A117000BF00BF00BD0000A8060020FE
:101C1000AF2E002010B50446314800780A2804D0C1
:101C20000B280FD00C2855D12DE02C2C06D10B20E1
:101C30002B49087000202B49088002E00A2028491F
:101C400008704BE02C2C1AD0302C1BDB392C19DC03
:101C5000244800880A214843224908802046303819
:101C6000098840181F490880084600881A2809D1A9
:101C70000C201B49087000201A49088002E00A2045
:101C8000174908702AE00D2C20D0302C21DB392C8C
:101C90001FDC144800880A21484312490880204666
:101CA0003038098840180F4908801EF0D1FA0D49D4
:101CB000098888420DD1232005F030F80320C04365
:101CC000094908750A200649087002E00A200449FB
:101CD000087003E00A200249087000BF00BF10BD71
:101CE000A8060020EE060020AF2E002000B53449E3
:101CF00009780A390B0019F0E2F90906101A242EA6
:101D0000384248526000452803D10B212C4A1170FB
:101D100002E00A212A4A117050E0562803D10C2112
:101D2000274A117002E00A21254A117046E0452831
:101D300003D10D21224A117002E00A21204A1170BC
:101D40003CE04E2803D10E211D4A117002E00A2109
:101D50001B4A117032E0542803D10F21184A117028
:101D600002E00A21164A117028E03A2803D1102116
:101D7000134A117002E00A21114A11701EE0302846
:101D800002D111210E4A117018E02C2803D1122122
:101D90000B4A117002E00A21094A11700EE0362840
:101DA00007D10321C943074A11750021044A117064
:101DB00002E00A21024A117000E000BF00BF00BD2E
:101DC000A8060020AF2E002070B5044656480078C3
:101DD0000A38030019F073F90805A10F19232D3AE9
:101DE00059A14E2C03D10C204F49087002E00A2063
:101DF0004D49087095E04E2C03D10D204A490870DA
:101E000002E00A20484908708BE04D2C03D10E20D7
:101E10004549087002E00A204349087081E0492CD6
:101E200003D10F204049087002E00A203E490870A3
:101E300077E03A2C06D100213C48817110203A49C4
:101E4000087002E00A20384908706AE02C2C14D08F
:101E5000302C19DB392C17DC34488079092808DA52
:101E6000324881798079401C304A9071101F445467
:101E70000AE000202D49887106E000212C4881727B
:101E8000C1721120284908704BE02C2C3BD00D2C3E
:101E900039D02749C87A897A00020843012189028A
:101EA000884228DA21480838FEF712FA451C1F49F3
:101EB00008392846FEF724FA302C01DB392C07DDDF
:101EC000412C01DB462C03DD612C25DB662C23DC59
:101ED0001748C17A807A09020143154AD07A927A6A
:101EE00000021043401C82B211488272120AC27270
:101EF0000C30445410E000210D488172C1720A2058
:101F00000949087008E0002008494872012020397A
:101F100088750A200449087003E00A200249087005
:101F200000BF00BF70BD0000A9060020CF2E00201A
:101F3000AF28002000B54B4909780A390B0019F089
:101F4000BEF80D080E1826303A444E58626C768062
:101F50008A003A2802D10B21424A11707FE02028E2
:101F600003D10C213F4A117002E00A213D4A117051
:101F700075E0522803D10D213A4A117006E0022182
:101F8000C943394A11750A21364A117067E045285C
:101F900003D10E21334A117002E00A21314A117037
:101FA0005DE0472803D10F212E4A117002E00A217B
:101FB0002C4A117053E0492803D11021294A11708D
:101FC00002E00A21274A117049E0532803D1112168
:101FD000244A117002E00A21224A11703FE054287D
:101FE00003D112211F4A117002E00A211D4A11700B
:101FF00035E0452803D113211A4A117002E00A2165
:10200000184A11702BE0522803D11421154A11707F
:1020100002E00A21134A117021E0452803D115215D
:10202000104A117002E00A210E4A117017E044288C
:1020300003D116210B4A117002E00A21094A1170DE
:102040000DE04B2806D10321C943074A11750A2127
:10205000044A117003E00A21024A117000BF00BF58
:1020600000BD0000A8060020AF2E002000B52649C4
:1020700009780A390B0019F022F807050B11171D12
:1020800023294100542802D10B211F4A117039E045
:10209000492802D10C211C4A117033E04E2802D18C
:1020A0000D21194A11702DE0442802D10E21164A43
:1020B000117027E03A2802D10F21134A117021E054
:1020C000202802D11021104A11701BE0332804D1BE
:1020D0000321C9430D4A11750CE0362804D10321B0
:1020E000C9430A4A117505E0312803D10221C943C9
:1020F000064A11750A21044A117003E00A21024AB6
:10210000117000BF00BF00BDA8060020AF2E002048
:1021100010B50446304800780A38030018F0CFFFA5
:1021200007050F19232D37415600542C03D10B20DE
:102130002949087002E00A20274908704AE0492C22
:1021400003D10C202449087002E00A2022490870BB
:1021500040E04E2C03D10D201F49087002E00A20F8
:102160001D49087036E0442C03D10E201A4908702E
:1021700002E00A20184908702CE03A2C03D10F2005
:102180001549087002E00A201349087022E0202C4B
:1021900003D110201049087002E00A200E4908708F
:1021A00018E0342C0AD1232004F0B8FD0320C043EA
:1021B0000A4908750A200849087006E00220C04351
:1021C000064908750A200449087003E00A200249FC
:1021D000087000BF00BF10BDA8060020AF2E002071
:1021E00070B50446F84800780A38030018F067FF15
:1021F000120A154A7EB0B9E1F8F6F5F4F3F2F1F0FF
:10220000EFEEEDEC2C2C07D10020F0490870F049DE
:1022100008800B20EC4908705EE22C2C1DD10020B8
:102220000021EB4A118000BF0CE0E94909880A222D
:102230005143E74A1180E749095C12888918E44A4A
:102240001180401CE14909788842EEDB0021DF4A19
:1022500011700C21DC4A117013E0DC4800780A2868
:102260000CDA20463038C1B2DA48D84A12788154A4
:10227000D6480078401CD549087002E00020D249B9
:102280000870EDE32C2C1DD100200021D24A1160F2
:1022900000BF0CE0D04909680A225143CE4A1160C0
:1022A000CC49095C12688918CB4A1160401CC749A7
:1022B00009788842EEDB0021C44A11700D21C24A20
:1022C000117012E0C14800780A280BDA2046303835
:1022D000C049BE4A12788854BC480078401CBB49AB
:1022E000087002E00020B8490870B9E32C2C1AD11C
:1022F00000200021B94A118000BF0CE0B7490988CD
:102300000A225143B54A1180B249095C12888918E2
:10231000B24A1180401CAD4909788842EEDB0E219B
:10232000A94A117013E0A948007805280CDA204664
:102330003038C1B2A748A54A12788154A348007822
:10234000401CA249087002E000209F49087087E302
:10235000222C05D100209D4908700F209A49087051
:102360007EE3222C13D100250A219D48FDF789FF29
:1023700000BF04E09748405D994948556D1C93485B
:1023800000788542F6DB10208F49087010E08F48F6
:1023900000780A2809DA8F488C49097844548B4818
:1023A0000078401C8949087002E0002086490870C6
:1023B00056E32C2C07D10020844908708549087009
:1023C0001120814908704BE346E39CE28CE280E2F5
:1023D00056E24AE213E280E108E17EE072E0FFE7C4
:1023E0002E2C57D179480078012804D179484078BB
:1023F0007C4908803AE075480078022809D1754880
:1024000040780A2148437349897840187549088003
:102410002CE06E48007803280FD16E484078642184
:1024200048436C4989780A22514340186949C97860
:10243000401800B26B49088018E06448007804280E
:1024400014D1644840787D21C900484361498978A6
:102450006422514341185F48C0780A22504308184B
:102460005C490979401800B25E4908805D480088DF
:102470000A21484300B25B49088056480078012889
:1024800004D108460088404200B2088012204E491C
:10249000087016E02D2C03D101204E49087010E081
:1024A0004A48007804280CDA20463038C1B2474840
:1024B0000078401C474A115444480078401C434966
:1024C0000870CDE22C2C07D100204049087041490A
:1024D000087013203C490870C2E22C2C5CD13B48A8
:1024E0000078012804D13B4840783F4908803AE011
:1024F00036480078022809D1364840780A214843F6
:10250000344989784018384908802CE02F480078F1
:1025100003280FD12F484078642148432D498978FA
:102520000A22514340182B49C978401800B22E495D
:10253000088018E025480078042814D12548407800
:102540007D21C900484323498978642251434118B9
:102550002048C0780A22504308181E4909794018BB
:1025600000B221490880204800880A21484300B26F
:102570001D49088017480078012804D108460088C2
:10258000404200B2088000201049087011490870CC
:1025900014200D49087016E02D2C03D101200D499F
:1025A000087010E00948007804280CDA204630381A
:1025B000C1B206480078401C064A1154034800780E
:1025C000401C024908704BE2A8060020B10600201A
:1025D000BC060020452F0020C0060020C4060020B5
:1025E000502F0020C6060020C80600202C2C5CD1ED
:1025F000FE480078012804D1FD484078FD49088054
:102600003AE0FA480078022809D1F94840780A21CE
:102610004843F74989784018F64908802CE0F34888
:10262000007803280FD1F248407864214843F049EC
:1026300089780A2251434018ED49C978401800B200
:10264000EC49088018E0E9480078042814D1E848EB
:1026500040787D21C9004843E54989786422514387
:102660004118E348C0780A2250430818E049097924
:10267000401800B2DF490880DE4800880A2148433C
:1026800000B2DC490880DA480078012804D1084605
:102690000088404200B208800020D4490870D44924
:1026A00008701520D449087016E02D2C03D10120A4
:1026B000CF49087010E0CD48007804280CDA204695
:1026C0003038C1B2C9480078401CC94A1154C748C3
:1026D0000078401CC5490870C2E12C2C73D1C34856
:1026E000007801280BD1C2484078C44908800846C8
:1026F00000880A21484300B2C04908804FE0BB4827
:102700000078022810D1BA4840780A214843B849D5
:1027100089784018B9490880084600880A2148434A
:1027200000B2B64908803AE0B0480078032816D1D4
:10273000AF48407864214843AD4989780A22514323
:102740004018AB49C978401800B2AC490880084627
:1027500000880A21484300B2A84908801FE0A34826
:10276000007804281BD1A24840787D21C900484345
:102770009F4989786422514341189D48C0780A22B4
:10278000504308189A490979401800B29B490880BB
:10279000084600880A21484300B2984908809448B6
:1027A0000078012805D195480088404200B293493D
:1027B000088000208D4908708D49087016208E49C8
:1027C00008701BE0FFE72D2C03D101208849087019
:1027D00014E08648007804280DDA20463038C1B26B
:1027E000834A82480078401C115480480078401C7D
:1027F0007E49087002E00A207F49087030E12C2CE5
:102800001FD1002000217E4A118000BF0CE07C49CE
:1028100009880A2251437A4A11807549095C128855
:102820008918774A1180401C704909788842EEDB8C
:1028300000216E4A11706E4A117017216E4A117094
:1028400012E06A48007804280BDA204630386849DC
:10285000664A1278885465480078401C63490870BD
:1028600002E00A2064490870FAE0222C07D1002017
:102870005E4908705E49087018205F490870EFE0F3
:10288000222C14D1002000BF04E05949095C5D4AA4
:102890001154401C554909788842F6DB0021534AFF
:1028A0001170534A11701921534A117010E04F48AA
:1028B00000780A2809DA4E484C49097844544B48B4
:1028C0000078401C4949087002E000204A4908701D
:1028D000C6E02C2C07D100204449087044490870F8
:1028E0001A2045490870BBE02C2C07D140480078DD
:1028F000454908801B204049087003E020463038D5
:102900003B490870ACE02D2C03D1012038490870F8
:10291000A1E0302C17DB392C15DC34480078042872
:102920000DDA20463038C1B2314A30480078401CB8
:1029300011542E480078401C2C4908708BE00A2066
:102940002D49087087E02948007801280BD12848D4
:1029500040782E490880084600880A21484300B282
:102960002A49088013E02148007802280FD1204826
:1029700040780A2148431E49897840182349088035
:10298000084600880A21484300B2204908801748B9
:102990000078032816D1164840786421484314492A
:1029A00089780A22514340181149C978401800B269
:1029B00016490880084600880A21484300B2134996
:1029C000088032E00948007804282ED10848407871
:1029D0007D21C90048430649897864225143411842
:1029E0000348C0780A225043081811E0B1060020BD
:1029F000452F0020CA060020A8060020CC06002093
:102A0000CE0600205A2F0020D0060020D20600203B
:102A100014490979401800B2134908800846008813
:102A20000A21484300B2104908800E480078012866
:102A300005D10D480088404200B20B4908800020B3
:102A40000A490870074908700A20094908700320DC
:102A5000C0430849087503E00A200549087000BF13
:102A600000BF70BD452F0020D2060020B106002017
:102A7000A8060020AF2E00202A4909780A2906D08E
:102A80000B290AD00C291ED00D2945D125E04F284D
:102A900002D10B21234A117042E04B2806D10121BB
:102AA000214A11700C211F4A11700BE0522806D1E7
:102AB00000211D4A11700C211A4A117002E00A21EE
:102AC000184A11702CE00D2803D10D21154A117000
:102AD00002E00A21134A117022E00A2818D1124993
:102AE0000978002904D00321C943104A117503E075
:102AF0000221C9430D4A11750D49097A0B2903D1E9
:102B00000A21084A117006E00021064A117002E00D
:102B10000A21044A117003E00A21024A117000BF21
:102B200000BF7047A8060020DE060020AF2E002060
:102B3000AF28002000B5224909780A390B0018F0A7
:102B4000BEFA08050B11171D23292F392B2802D196
:102B50000B211B4A117031E0512802D10C21184A77
:102B600011702BE0492802D10D21154A117025E082
:102B70004F2802D10E21124A11701FE0502802D1B5
:102B80000F210F4A117019E0452802D110210C4A7B
:102B9000117013E04E2802D11121094A11700DE085
:102BA0003A2803D10321C943064A11750A21044A70
:102BB000117003E00A21024A117000BF00BF00BD7E
:102BC000A8060020AF2E00200E4909780A2902D05D
:102BD0000B2911D105E0572802D10B21094A1170A8
:102BE0000EE04E2804D10321C943074A117502E0C3
:102BF0000A21044A117003E00A21024A117000BF41
:102C000000BF7047A8060020AF2E002014490978A5
:102C10000A2904D00B2908D00C291BD10FE0452824
:102C200002D10B210E4A117018E0452803D10C2166
:102C30000B4A117002E00A21094A11700EE0502877
:102C400004D10321C943074A117502E00A21044A4D
:102C5000117003E00A21024A117000BF00BF7047E3
:102C6000A8060020AF2E002000B5634909780A3974
:102C70000B0018F024FA0B07111B252F39434D695F
:102C80007394BB00222803D10B215B4A117002E030
:102C90000A21594A1170ADE0722803D10C21564A1D
:102CA000117002E00A21544A1170A3E0652803D193
:102CB0000D21514A117002E00A214F4A117099E02A
:102CC000632803D10E214C4A117002E00A214A4ABE
:102CD00011708FE0762803D10F21474A117002E06E
:102CE0000A21454A117085E0222803D11021424A69
:102CF000117002E00A21404A11707BE02C2803D1B8
:102D000011213D4A117002E00A213B4A117071E025
:102D100000213A4A9172D172394A1180302806D185
:102D20000121384A51721221334A11700BE03128C7
:102D300006D10221334A517212212F4A117002E04A
:102D40000A212D4A117055E02C2803D113212A4A5B
:102D5000117002E00A21284A11704BE00A2810D0B5
:102D600030281BDB392819DC254909880A22514300
:102D7000234A11800146303912888918204A11806F
:102D80000CE01F49098801229202914203DA1421C2
:102D9000194A117002E00021174A11702AE0174AFF
:102DA000D17A927A09021143154A1288914212DAB5
:102DB000124AD17A937A0A021A43104BD97A9B7A33
:102DC00009021943491C8BB20C498B721B0ACB7246
:102DD0000C31885409E00321C9430A4A203A11758D
:102DE000012191750A21044A117003E00A21024A67
:102DF000117000BF00BF00BDAB060020AF2800204F
:102E0000AC060020CF2E002010B5044648480078BC
:102E10000A38030018F053F90B07111B252F39430B
:102E20004D57616E8600442C03D10B204049087039
:102E300002E00A203E49087078E0492C03D10C20BA
:102E40003B49087002E00A20394908706EE0532CB3
:102E500003D10D203649087002E00A203449087079
:102E600064E0432C03D10E203149087002E00A20AF
:102E70002F4908705AE04F2C03D10F202C490870BD
:102E800002E00A202A49087050E0562C03D1102095
:102E90002749087002E00A202549087046E0452CC1
:102EA00003D111202249087002E00A20204908704D
:102EB0003CE0522C03D112201D49087002E00A2088
:102EC0001B49087032E03A2C03D1132018490870CE
:102ED00002E00A201649087028E02C2C09D10020B5
:102EE000144908700A211448FDF7CBF91420104941
:102EF00008701BE02C2C0CD00E4800780A2810D249
:102F00000C4801780078401C0A4A10700A48445462
:102F100007E00320C04308492B3908750A200449FB
:102F2000087003E00A200249087000BF00BF10BD0E
:102F3000EB060020EC060020DA2E00200148007885
:102F4000704700004100002003480078002801D1AC
:102F5000012070470020FCE74000002000200449C9
:102F60000978002901D1012000E00020704700000D
:102F70004000002070B555480078030018F09FF815
:102F8000050405102593A3009EE0012000F070FDCC
:102F9000002804D10EF01AFC02204C49087093E07E
:102FA0004B48007800F008F9012000F017F900F014
:102FB00079F915F089FA4749086015F085FA46490C
:102FC00008600320414908707EE0012000F022F9EA
:102FD000012855D115F078FA3F49086015F074FAC8
:102FE0003C490968401A3D49096888425AD300247F
:102FF00000F01CF904463A48406800193849486016
:1030000038480078002803D108468460046013E043
:1030100033488068A04201D2204601E030488068F1
:103020002F49886008460068A04201D9204601E087
:103030002B4800682A4908602A480078401CC0B222
:103040002849087028490978884215DB002524485A
:10305000406823490968401A21498968451A22486D
:103060000078811E2846FDF753F82049096808605A
:1030700004201649087002E002201449087011E08B
:1030800015F022FA14490968401A64280AD900F098
:103090000FF91748007802210843154908700420E9
:1030A0000A49087010E000F0A1F800F0EDFB0021E3
:1030B000102014F045FE01200E4909680870002018
:1030C0000249087000E000BF00BF70BD4000002052
:1030D000510000205400002058000020480000202B
:1030E000F012002050000020520000204400002078
:1030F000410000204C00002010B500F077F800F0EF
:10310000C3FB0021102014F01BFE10BDF8B50546CE
:103110000C4616461F46032C00D20324502C00D91F
:1031200050241B4906980860192D0ADD19480078BB
:1031300001210843174908700120154909680870E2
:10314000F8BD154807600020114909680870134947
:10315000087013494860086088600E49087011487B
:10316000057011490C70114806600EF049FB0121F1
:10317000102014F0E5FD00F091FB00F041F8012172
:10318000084613F011FE01200949087000BFD7E777
:103190004C0000204100002044000020500000208E
:1031A000F0120020510000205200002048000020B2
:1031B0004000002070470000014607484068FF2299
:1031C000F13290430A01FF23F1331A401043024ABF
:1031D0005060002070470000002400400249496B05
:1031E0008143014A5163704780240040034840688E
:1031F000400840000149486070470000002400403A
:103200000348406840084000401C0149486070473E
:103210000024004001460448006B0840002801D00B
:10322000012070470020FCE7802400400148006A2C
:10323000704700008024004010B50446002C01D1E6
:10324000042010BD012016494860022018F09EFDA0
:103250006078A1880843E188084361880843218990
:1032600008430F49496808430D494860084680688B
:1032700009158843217889020122920211400843EE
:10328000074988600846806804218843A17A89003C
:10329000042211400843024988600020D1E7000061
:1032A000002400400120014908607047C02400400C
:1032B0000020014908607047C024004030B50A462C
:1032C00000210EE0D400A41A074D6419635C047851
:1032D0005C4004700478AA256C400470401C4C1CAF
:1032E000E1B20729EEDB30BD70290200F0B587B0EE
:1032F00012F01EFC10210840002810D0042012F00B
:103300003FFCFA480088401CF8490880E121090187
:10331000F6480088FCF712FF88B2F449088012F0E2
:1033200007FC20210840002822D0052012F028FCAC
:10333000EF480078401CEE490870084600783C28A9
:1033400016DB00200870EB48FCF7C2FFE121090101
:103350004418E8492046FCF7D3FFE648001DFCF777
:10336000B7FF0446233CE349091D2046FCF7C8FF8C
:10337000E1480078002804D001280ED002287DD131
:10338000A5E102F07FFD002806D1D8480088DB497E
:1033900008600120D8490870CAE102F073FD0128D5
:1033A0006DD1002106910591D0480088D349096864
:1033B000884207D3CD480088D0490988401AD049AF
:1033C000088009E0C9480088E12109014018CB497B
:1033D0000988401ACA49088008201CF00FFF772886
:1033E00007D1C74800884B21C9004018C44908804C
:1033F0000BE008201CF002FF552806D1C0480088C9
:10340000E121C9004018BE490880002108201EF0B3
:103410009DF9B8480C30FCF75BFFB949098844189E
:10342000B4490C312046FCF76BFFB248417C027C6A
:1034300008021043401C81B2AE480174090A41746D
:1034400006A80EF015FE05A80EF004FE0A216A4635
:103450001820105EFCF772FE00B206900A216A4640
:103460001420105EFCF76AFE00B2059004201CF0E8
:10347000C5FE01283DD1A248008801E054E125E1C4
:10348000FDF7E2F906469F4A9F4BFDF7D7F80191F9
:1034900000909848001DFCF71BFF0646FDF7D4F985
:1034A0000446019B009AFDF7BBF803910290FDF7DB
:1034B00005FA9049091D0490FCF722FF04F050FA28
:1034C000002815D191480078401C904908700721C8
:1034D0008E480078FCF732FEC8B28C490870084666
:1034E000017802201EF032F901210A201EF02EF987
:1034F000E8E069461820085E002820DA8048008845
:10350000FDF7A2F906467F4A814BFDF797F8019136
:1035100000907848001DFCF7DBFE0646FDF794F9A5
:103520000446019B009AFDF77BF803910290FDF79A
:10353000C5F97049091D0490FCF7E2FEC2E0694636
:103540001420085E7721C943884220DA6C4800883D
:10355000FDF77AF904466B4A6D4BFDF76FF803915E
:1035600002906448001DFCF7B3FE0446FDF76CF9B9
:1035700001910090039B029AFDF752F80646FDF771
:103580009DF95C49091D0490FCF7BAFE9AE0694672
:103590001420085E7221C943884220DA5848008806
:1035A000FDF752F906465B4A5B4BFDF747F8019180
:1035B00000905048001DFCF78BFE0646FDF744F9CD
:1035C0000446019B009AFDF72BF803910290FDF74A
:1035D00075F94849091D0490FCF792FE72E06946AE
:1035E0001420085E6821C943884222DA44480088D2
:1035F000FDF72AF90646434A5242484BFDF71EF8AA
:1036000004460D463B48001DFCF762FE0646FDF7EA
:103610001BF922462B4601910090FDF701F803911A
:103620000290FDF74BF93349091D0490FCF768FE41
:1036300048E069461420085E5921C943884220DACF
:103640002F480088FDF700F904462E4A2E4BFCF760
:10365000F5FF019100902748001DFCF739FE044654
:10366000FDF7F2F80646019B009AFCF7D9FF03919B
:103670000290FDF723F91F49091D0490FCF740FE55
:1036800020E01F480088FDF7DFF804461D4A52423B
:10369000234BFCF7D3FF019100901648001DFCF767
:1036A00017FE0446FDF7D0F80646019B009AFCF78A
:1036B000B7FF03910290FDF701F90E49091D04902F
:1036C000FCF71EFE02200C49087000BF30E001F03C
:1036D000ADF9012808D1134B1822D021054801F07B
:1036E00001FC00200449087022E0000010050020C1
:1036F000120500200C2100200105002004050020F7
:10370000140500203333333333331F4024050020A6
:1037100033B330406666666666662D40CCCC214089
:10372000CCCC1A400005002000203049087000BFB2
:1037300000BF2F480078002802D001284FD10BE0AD
:103740000AF03EFA002806D12A4800882A49086073
:1037500001202749087046E00AF032FA01283DD1DD
:103760002448008824490968884207D321480088F2
:1037700021490988401A2149088009E01D4800882C
:10378000E121090140181C490988401A1B49088099
:103790001B480068194909884018194908600846FB
:1037A00000683C2817D9084600683C38086015486E
:1037B000FCF78EFD04463C3412492046FCF7A0FD80
:1037C0001048001FFCF784FD0446153C0D49091FF5
:1037D0002046FCF795FD00200549087003E0002015
:1037E0000349087000BF00BF07B0F0BD010500200D
:1037F0000205002010050020080500201405002007
:103800000C0500201421002007480078002809D169
:1038100006480078002805D105480078002801D125
:10382000012070470020FCE7010500200205002070
:1038300025050020014680200840002801D00846C8
:103840007047302905DB392903DC08463038C0B21F
:10385000F6E7612905DB662903DC08465738C0B264
:10386000EEE7412905DB462903DC08463738C0B2BC
:10387000E6E70846E4E701460A110A235A430B0724
:103880001B0FD218D0B270470348006802210840CD
:1038900001490860704700000024004010B5054849
:1038A00000680121084303490860022018F06EFAFD
:1038B00010BD00000024004030B502460020140274
:1038C000044D63191C68240C24048DB22C431C6025
:1038D00030BD0000000C004030B50246002014024C
:1038E000044D63195C68240C24048DB22C435C6085
:1038F00030BD0000000C004010B5014600200B0256
:10390000014C1A19906810BD000C004030B50246F9
:1039100000201402024D63199C68996030BD0000BC
:10392000000C004070B5024600201402054D6319DA
:103930001C6BAD14AC430D030126360335402C43FC
:103940001C6370BD000C004010B5014600200B0246
:10395000034C1A19D3685B085B005B1CD36010BD75
:10396000000C004010B5014600200B02034C1A1950
:10397000D3685B085B00D36010BD0000000C004002
:1039800070B503460A4600201C02224D6119CC681E
:10399000AD00AC4315782D030326360335402C4388
:1039A000CC60CC6801256D02AC4355786D020126D0
:1039B000760235402C43CC60CC687510AC439578CA
:1039C0002D02761035402C43CC60CC687025AC437A
:1039D000D5782D01702635402C43CC60CC68082565
:1039E000AC431579ED00082635402C43CC60CC68FB
:1039F0000425AC435579AD00042635402C43CC60FA
:103A0000CC680225AC4395796D00022635402C43E5
:103A1000CC6070BD000C004010B500F009F910BD7D
:103A200070B5044600252C2C1BDA14F04DFD05461C
:103A3000A0000D490858A84203D8A00008582D1A24
:103A400006E0A000084908580021C943081A451992
:103A5000A00006490858A84201D8002070BD0120E6
:103A6000FCE70020FAE700004C0C0020FC0C0020D2
:103A700070B504460025182C1BDA14F025FD054608
:103A8000A0000D490858A84203D8A00008582D1AD4
:103A900006E0A000084908580021C943081A451942
:103AA000A00006490858A84201D8002070BD012096
:103AB000FCE70020FAE700008C0B0020EC0B002054
:103AC0000148007870470000B003002010B5064898
:103AD000FCF708FC054B064A43404A40134301D11A
:103AE000012010BD0020FCE7AA190020B8A7F6E5C8
:103AF000D4C3B2A101480078704700009C020020A6
:103B000070B504460025002614F0DEFC0646094880
:103B10000068351A0848844203D1A54201D3012028
:103B200070BD0648844203D1A54201D30120F7E7C6
:103B30000020F5E71800002050C30000C02709004E
:103B40000148007870470000B1030020FFB583B042
:103B500006460F461C4638461CF086FB0290059828
:103B60001CF082FB01906078217800020843002855
:103B700006DD6078217800020843164988420FDB91
:103B800060782178000208431249083188421EDD1E
:103B900060782178000208430E490931884216DA1C
:103BA0006078217800020843B04203D009480F3002
:103BB00086420CD1A01C1CF057FB0546029885429A
:103BC00005D30198854202D8012007B0F0BD00203E
:103BD000FBE70000F0FF000001480078704700009C
:103BE0003A03002001480068704700003C030020B1
:103BF000002002498872C8727047000063230020C9
:103C00000020014908707047DC02002000200149B3
:103C1000C8757047AF2E002000200149087070471A
:103C20009C02002000200149087070473A030020E0
:103C300010B5012014F088FC01280DD114F07EFC91
:103C400057490860084600685649884205D114F073
:103C500091FCFF205449087096E051480068514992
:103C6000884246D214F086FC50480078002803D0E1
:103C70004E48007801281ED101204C49087048495F
:103C80000968484A501A4949491CFCF739FB484918
:103C9000C968491C4805400D4549C968C90AC90297
:103CA0000143434AD16014F05BFC42480078401C59
:103CB0004049087068E03D48401CFCF709FB384962
:103CC0000968384A511A88420FD23949C968491CD3
:103CD0004805400D3649C968C90AC9020143344A3A
:103CE000D160FF20304908704EE0FF202E49087057
:103CF0004AE02B4800682B49884245D914F03AFC29
:103D00002A480078002803D02848007802281ED1CD
:103D100002202649087022490968224A881A234944
:103D2000491CFCF7EDFA2249C968491E4805400DB7
:103D30001F49C968C90AC90201431D4AD16014F06C
:103D40000FFC1C480078401C1A4908701CE01748FA
:103D5000401CFCF7BDFA12490968124A891A8842C8
:103D60000FD21349C968491E4805400D1049C9685A
:103D7000C90AC90201430E4AD160FF200A490870EE
:103D800002E0FF2008490870022014F0DDFB012842
:103D900004D114F0EFFBEE200349087010BD0000C1
:103DA000EC02002000093D00E2020020E4020020B5
:103DB00000200040E302002010B5002013F098FF1F
:103DC000002013F0A9FF112014F008F8022013F0CE
:103DD000F3FF0121022013F025FE022014F022F847
:103DE000042013F0D5FF0121002013F01BFE00205A
:103DF00014F018F80121062002F0D0FC002002F097
:103E000031FD01211C2013F09BFF10BD0020014952
:103E1000087070476404002010B500F001F810BD70
:103E2000F8B5B3480078030017F049F905040FD935
:103E3000FEFDFC000020AF4908700120AC4908706D
:103E4000FF202D301DF090FC50E117F04BFC0028B6
:103E50007ED10D24A8480688A8480568002751E0AF
:103E6000E85D0A2808DAE85D3030C2B22046611CFD
:103E70008CB2A3490A543EE0E85D642816DAE85D96
:103E80000A21FCF75BF93030C2B22046611C8CB2CB
:103E90009B490A54E85D0A21FCF750F93031CAB257
:103EA0002046611C8CB296490A5424E0E85D6421E6
:103EB000FCF744F93030C2B22046611C8CB2904904
:103EC0000A54E85D0A21FCF739F90A210090FCF751
:103ED00035F93031CAB22046611C8CB288490A5487
:103EE000E85D0A21FCF72AF93031CAB22046611C8C
:103EF0008CB283490A542E222046611C8CB2804920
:103F00000A547F1C042FABDB601E84B222222046A1
:103F1000611C8CB27A490A542C222046611C8CB256
:103F200077490A5477493046FCF708F93030C2B275
:103F30002046611C8CB272490A5472493046FCF723
:103F4000FDF800917D21C9000098FCF7F7F800E02A
:103F500044E03030C2B22046611C8CB268490A5439
:103F60007D21C9003046FCF7E9F8009164210098F2
:103F7000FCF7E4F83030C2B22046611C8CB26049D4
:103F80000A5464213046FCF7D9F800910A210098C0
:103F9000FCF7D4F83030C2B22046611C8CB25849CC
:103FA0000A540A213046FCF7C9F83031CAB220461B
:103FB000611C8CB252490A540D222046611C8CB2FD
:103FC0004F490A54122221464D480FF061FD23202B
:103FD0001DF0D6FB02204649087000BF86E00DF0B8
:103FE000B5FF001D002809D142490870032040494F
:103FF0000870FF202D301DF0B7FB26E017F077FB8F
:10400000002804D00DF0A2FFC01C00281DD13948A3
:104010000078401C3749087008460078012811DBF9
:10402000002002E05EE027E010E008703648FCF770
:104030004FF9A521017000202D490870A8203349AF
:10404000087002E001202A4908704FE017F04AFB8F
:10405000002810D12E480068FCF72AF984B21B22F0
:1040600021462B4800680FF013FD02201DF088FB4D
:1040700004201F49087039E00DF068FF001D00287A
:104080000DD11C4908702048FCF722F9A3210170CA
:10409000002017490870A9201C49087021E017F07A
:1040A00026FB00281DD113480078401C11490870D8
:1040B0000846007801280DDB002008701248FCF744
:1040C00007F9A5210170002009490870A8200F49AF
:1040D000087006E0032006490870FF202D301DF00F
:1040E00043FB03E000200249087000BF00BFF8BD99
:1040F00032050020EA05002044050020400500208C
:10410000EB05002010270000DD2300202A050020F9
:104110002006002010B500F001F810BD70B5C148B0
:104120000078002804D003280AD004287ED13CE17E
:104130000320BC490870FF202D301DF015FB6FE1F6
:1041400017F0D0FA002872D10824002504E0B64800
:10415000405DB64948556D1C082DF8DBB44A517ACC
:10416000127A090211430846B249FBF7E7FF3030E3
:10417000C2B22046611C8CB2AC490A54AC4A517A96
:10418000127A090211430846AA49FBF7D7FF0E46E7
:104190007D21C9003046FBF7D1FF3030C2B2204646
:1041A000611C8CB2A1490A54A14A517A127A0902BF
:1041B000114308467D21C900FBF7C0FF0E4664216C
:1041C0003046FBF7BBFF3030C2B22046611C8CB2D8
:1041D00096490A54964A517A127A090211430846BE
:1041E0006421FBF7ABFF0E460A213046FBF7A6FF22
:1041F0003030C2B22046611C8CB28C490A548C4AC1
:10420000517A127A0902114308460A21FBF796FFF8
:104210003031CAB22046611C8CB284490A542C2227
:104220002046611C8CB281490A5401E0F4E0BBE0F5
:10423000002545E07E48001DFCF74AF8405D00116E
:104240000A280CDB7A48001DFCF742F8405D00119B
:1042500037302146621C94B2744A50540BE07448C3
:10426000001DFCF735F8405D001130302146621C1E
:1042700094B26E4A50546E48001DFCF729F8405D18
:104280000007000F0A280DDB6948001DFCF720F825
:10429000405D0007000F37302146621C94B2634A2C
:1042A00050540CE06248001DFCF712F8405D000716
:1042B000000F30302146621C94B25C4A50546D1C91
:1042C0005B49487A097A00020843A842B2DC5A489E
:1042D000007B80210840002828D05748007B8007B9
:1042E000800F002822D02C222046611C8CB24F491E
:1042F0000A5431222046611C8CB24C490A543022A7
:104300002046611C8CB249490A542046611C8CB27B
:1043100046490A540D222046611C8CB243490A5476
:104320003722214641480FF0B3FB36E04248807AFD
:10433000552804D0404876308078552822D12C2248
:104340002046611C8CB239490A5431222046611C36
:104350008CB236490A5430222046611C8CB2334953
:104360000A542046611C8CB230490A540D22204662
:10437000611C8CB22D490A54372221462B480FF07C
:1043800087FB0AE00D222046611C8CB227490A54A3
:104390001622214625480FF07BFB04201DF0F0F982
:1043A00004202049087000BF3AE00DF0CFFD001D49
:1043B00000280DD121490870A920214908701C4806
:1043C000FBF786FFA421017000201649087022E047
:1043D0000DF0BCFDC01C002803D017F088F90028A0
:1043E00019D116480078401C144908700846007816
:1043F00001280DDB002008700D48FBF769FFA5219F
:104400000170A8200E49087000200649087002E0DB
:1044100004200449087003E000200249087000BF2E
:1044200000BF70BD34050020B6290200E72300203C
:10443000DD23002010270000D020002024060020CB
:104440002A0500200020014908707047320500202D
:1044500070B546480078002806D0012805D003280A
:1044600074D006287CD123E07EE000F0DFFA01283A
:104470001DD13F48007816280FD0DC223D493E4828
:10448000FBF7E6FE3D4BDC22012149023A4800F0F1
:1044900029FD03203549087009E0384BDC223649F4
:1044A0000120400200F0D8FC0620304908705BE093
:1044B00000F0BCFA012846D1002500242EE0A1001E
:1044C0002D4A8818FBF704FF0021C943884201D117
:1044D000002525E0A100284A8818FBF7F9FE0646CA
:1044E00031462748FCF760FA09D3A100224A881810
:1044F000FBF7EEFE06462349FCF756FA01D20025EB
:104500000EE0A1001C4A8818FBF7E2FE06460021D7
:10451000FCF74AFA00D00125601CC4B2372CCEDB70
:1045200000BF002D0BD1DC2212491348FBF790FE8F
:10453000124BDC22012149020F4800F0D3FC03207A
:104540000A49087000BF0FE000E009E000F06EFAD1
:10455000012804D10C49087000200449087003E0C8
:1045600000200249087000BF00BF70BDB6040020E3
:104570003C200020502A020027370020B5040020EC
:1045800000007A4400007AC4B704002001460029E4
:1045900006D10D48407F012800D170470020FCE77C
:1045A000012906D10848807F012800D1F5E70020C5
:1045B000F3E7022906D10448C07F012800D1ECE7C7
:1045C0000020EAE70020E8E78823002010B5C04675
:1045D000C04610BD10B507480078002808D106482D
:1045E0000078002804D110F0A7FD012800D110BDEB
:1045F0000020FCE7790B0020840B002010B510F0A0
:10460000A5FD0B48C079202802DB00210848C171B4
:1046100007488079202802DB0021054881710220AB
:1046200008F05CF804460349FBF76AFE10BD000081
:10463000FC2000207A0B002010B511F0D9FF11F0FA
:1046400061FD10F0EBFD10BDF1B584B08F4800782E
:10465000002801D105B0F0BD8D48FBF739FE441CA0
:104660008B492046FBF74CFE8948FBF731FE044698
:104670001421FBF74DFD012908D186490498FBF769
:104680003FFE8449091D0498FBF73AFE8148FBF779
:104690001FFE044621460498FCF790F903D27D4999
:1046A0000498FBF72DFE7B48001DFBF711FE044626
:1046B00021460498FCF778F904D27649091D04983C
:1046C000FBF71EFE72480830FBF702FE054629463E
:1046D0000498FBF72DFE04466D490831FBF710FEE8
:1046E0006B48FBF7F5FD04461421FBF711FD032988
:1046F00008D26748FBF7ECFD04461421FBF708FDE0
:10470000002936D16248FBF7E3FD07466048FBF716
:10471000DFFD0646113614213046FBF7F9FC400058
:104720003D1A2846FCF775F804465948001DFBF76A
:10473000CFFD02905748001DFBF7CAFD07465548BC
:10474000FBF7C6FD019052480830FBF7C1FD009011
:104750000199FBF73EFE06463946FBF73AFE054651
:104760000299FBF7E5FD21460390FBF777FE0490E5
:1047700022E04748FBF7ACFD07464548FBF7A8FD9C
:1047800014210390FBF7C4FC40003E1A3046FCF7AE
:1047900040F804463E480830FBF79AFD06463C4880
:1047A000001DFBF795FD07463146FBF7C1FD0546A9
:1047B0002146FBF753FE04903548FBF789FD04467C
:1047C0001421FBF7A5FC002927D13148001DFBF778
:1047D0007FFD03902F48001DFBF77AFD02902D48C6
:1047E000FBF776FD07462A480830FBF771FD39468E
:1047F0000190FBF7EEFD06460299FBF7EAFD054640
:104800000399FBF795FD04462149091DFBF778FD47
:104810001F4908310020FBF773FD1D48FBF758FDC9
:10482000E121C900884217D919490020FBF768FD2A
:104830001749091D0020FBF763FD154908310020C9
:10484000FBF75EFD12490C310020FBF759FD1049C2
:1048500010310020FBF754FD049802F01DF80446C7
:104860000B492839FBF74CFD09482838FBF730FD88
:10487000044608493439FBF743FD05482838FBF75F
:1048800027FD044604F0BAFD00BFE3E665030020FF
:1048900018190020DC18002010B500F0C7F8012816
:1048A00007D105480078002801D1012010BD002063
:1048B000FCE70020FAE70000B404002010B54C48E3
:1048C0000078030016F0FBFB0A0607112131415165
:1048D0006171868E8AE000204649087001204649B1
:1048E000087002204249087080E012F045FF4148FC
:1048F0000078012808D100203E49087001203E4977
:10490000087003203A49087070E0FFF7A1FD3948AC
:104910000078012808D10020364908700120364966
:10492000087004203249087060E001F0E5FF31486A
:104930000078012808D100202E49087001202E4956
:10494000087005202A49087050E013F029FE294814
:104950000078012808D10020264908700120264946
:10496000087006202249087040E011F07BFB2148C6
:104970000078012808D100201E49087001201E4936
:10498000087007201A49087030E011F0EBF9194857
:104990000078012808D10020164908700120164926
:1049A000087008201249087020E000F03FF8012844
:1049B0000FD112480078162808D016200F49087029
:1049C0000F4B012200210D4800F08CFA0920084904
:1049D00008700BE000F02AF8012802D100200449F9
:1049E000087003E000200249087000BF00BF10BD3E
:1049F000B4040020B7040020B60400203C200020AE
:104A0000B504002010B5FFF759FF00F085F810BD80
:104A100010B5044609F008F8012805D100F006F8A1
:104A2000002801D0012010BD0020FCE703480078D9
:104A3000002801D1012070470020FCE7040000207D
:104A400003480078002801D1012070470020FCE7CE
:104A50000400002000B585B0072103A817F086F9EF
:104A60000C21684617F082F9002168464173817372
:104A7000C1730174417403AA0721402008F0B4FAFD
:104A8000002168464173012141740021C173017402
:104A900003AA0821402008F0A7FA03AA0921402010
:104AA00008F0A2FA01220821402008F0EBFA0122C6
:104AB0000921402008F0E6FA00220721402008F0F2
:104AC000F9FA11481149086001220421104812F036
:104AD00083F9102010F054FD13F0FAF800900D48FF
:104AE0000190402168460172552141720021817276
:104AF00069460648006808F049FC012202210C20A2
:104B000000F0ACFA05B000BD000400403800002001
:104B100020200040A086010010B5C24800780300A4
:104B200016F0CDFA0906071019C0E1FCFBFAF900EE
:104B300075E10320BB4908700FF0CCFCBA4812F0B5
:104B400081F96CE10320B74908700FF0DFFCB6482B
:104B500012F078F963E1B448FEF7D2FF002856D08E
:104B6000B248006808F009FCB148007800283DD13F
:104B700008F062FF01281CD1AD480078401CAC4908
:104B8000087002F0F5FE00220621AA4812F024F96E
:104B900000220721402008F08DFA00220421A648B7
:104BA00012F01AF9A04812F04DF907209D4908703B
:104BB00077E09F480078401C9D49087002F0D8FEBD
:104BC000002206219B4812F007F90022072140200D
:104BD00008F070FA00220421974812F0FDF892487C
:104BE00012F030F908208F4908705AE000209049EF
:104BF000087002F0BDFE00220721402008F05AFA9A
:104C0000894812F01FF904208649087049E008F02D
:104C10000BFF01282ED108F00FFF01280BD102F065
:104C2000A7FE002082490870844812F00BF9062084
:104C30007C49087035E013F047FC81490968401A47
:104C4000C8282ED902F094FE00207949087000226D
:104C50000621784812F0C0F800220721402008F011
:104C600029FA00220421744812F0B6F800206D4998
:104C7000087016E07348008801280FD113F024FC57
:104C800071490968401A7149884207D900206D4965
:104C9000088005216548006808F0D4FB03206149BD
:104CA0000870BCE06048FEF72BFF002817D0FFF724
:104CB000D1FE01220721402008F0FCF90122062143
:104CC0005C4812F089F805215848006808F0BAFBE2
:104CD000554812F0B7F805205249087002E0042048
:104CE000504908709BE05048FEF70AFF00283AD070
:104CF0004E480068406908281CD104214B480068D0
:104D000008F0A0FB002206214A4812F065F80022B4
:104D10000721402003E07EE061E044E027E008F066
:104D2000C9F900220421444812F056F800203D49F8
:104D300008701BE0464800784021884344490870C9
:104D4000002206213B4812F047F8002207214020AC
:104D500008F0B0F900220421374812F03DF8002095
:104D60003049087002E005202E49087057E03348AA
:104D7000FEF7C6FE002812D0002206212D4812F0B0
:104D80002BF800220721402008F094F9002204218A
:104D9000294812F021F800202249087002E006207C
:104DA000204908703BE015F0FFFF1F48FEF7A8FE02
:104DB000002813D0FFF74EFE01220721402008F003
:104DC00079F9012206211B4812F006F8012204217C
:104DD000194812F001F80220124908701FE015F07E
:104DE000E3FF1148FEF78CFE002813D0FFF732FED8
:104DF00001220721402008F05DF9012206210D481B
:104E000011F0EAFF012204210B4811F0E5FF012017
:104E10000449087003E000200249087000BF00BF89
:104E200010BD000004000020C02709003800002049
:104E300005000020080400402020004050C300006E
:104E4000200000202E0000201C00002088130000FD
:104E50003600002070470000F8B505460F4614469E
:104E60001E46402016490870002030702819012184
:104E7000C903884221DC002C1DDD881184421ADC24
:104E800010480580104807601048048010480660EC
:104E9000012204210F4811F09FFF01220721402029
:104EA00008F008F9012206210B4811F095FF0120B6
:104EB0000A490870F8BD0020FCE70020FAE700006E
:104EC00036000020340000200C00002026000020C6
:104ED00014000020202000400804004004000020AE
:104EE00070470000F8B507460D4614461E46602080
:104EF0004D4908700020307028190121C9038842EB
:104F00007EDC002C7DDD881184427ADC47480580F8
:104F1000474807602846E917890E09188911890151
:104F2000691A444A1180104600884021081A4249F3
:104F300008802046E117890E09188902090C3F4AAA
:104F40001180E117890E091889118901611A3C4AFB
:104F500011803A480088002827D136480088001977
:104F600040281ADD01203749088033480088201A7C
:104F700084B22046E117890E091889112F4A118041
:104F8000E117890E091889118901611A2C4A1180CB
:104F9000294800882C49088029E0002029490880F8
:104FA000274800882849088021E0012025490880F9
:104FB00020480088002803D140202349088016E0BB
:104FC0001D480088201A84B22046E117890E09186E
:104FD00089111A4A1180E117890E0918891189016E
:104FE000611A174A11801448008817490880174829
:104FF000066001220421164811F0EEFE012201E0B4
:1050000010E00DE00721402008F054F801220621AD
:10501000104811F0E1FE02200F4908700120F8BD90
:105020000020FCE70020FAE73600002034000020D2
:105030000C000020280000202A0000202C00002066
:105040003000002032000020260000201400002044
:1050500020200040080400400400002070B50446F1
:105060000E4615462046002805DBC206D20E012159
:105070009140144A116000BF3146204616F02EF8C8
:10508000012D0ED12046002809DB00BF00BFC2065B
:10509000D20E012191400C4A116000BF00BF00BF39
:1050A0000FE0204600280ADBC206D20E0121914003
:1050B000054A80321160BFF34F8FBFF36F8F00BF7F
:1050C00000BF70BD80E200E000E100E0F7B588B00D
:1050D000154600247F20C00507900C20069000BFD5
:1050E00009E0A001694A11580898FBF75DFC00D857
:1050F00005E0601CC4B20698401EA042F1DC00BF6F
:1051000063492846FBF750FC3CD8A1015F4A891847
:1051100048690999FBF765F905900999FBF761F969
:105120000646A001594A801801690898FBF759F909
:1051300003900999FBF755F9A101544A8918059084
:10514000C8680999FBF74DF90390A0014F4A8018F0
:1051500081680898FBF745F9A20101904B481018A7
:1051600041680198FBF7E4F802900399FBF7E0F837
:1051700004900599FBF7DCF807463146FBF7D8F8B1
:1051800007907DE043492846FBF70EFC3CD8A1017F
:105190003E4A8918886A0999FBF723F9059009990D
:1051A000FBF71FF90646A001384A8018416A0898A3
:1051B000FBF717F903900999FBF713F9A101334A9B
:1051C00089180590086A0999FBF70BF90390A0016B
:1051D0002E4A8018C1690898FBF703F9A2010190D3
:1051E0002A48101881690198FBF7A2F802900399E8
:1051F000FBF79EF804900599FBF79AF807463146AD
:10520000FBF796F807903BE0A101204A8918C86B8C
:105210000999FBF7E6F807460999FBF7E2F8A201BE
:1052200005901A481018816B0898FBF7DAF803907C
:105230000999FBF7D6F80746A20114495118486BA3
:105240000999FBF7CEF80390A001104A8018016B72
:105250000898FBF7C6F80190A0010C4A8018C16AB3
:105260000198FBF765F802900399FBF761F839465E
:105270000490FBF75DF806460599FBF759F807908F
:1052800028460799FBF7ADF80BB0F0BDE00700200A
:105290000000704100002C4210B5C046C046C04618
:1052A000C04610BDF0B589B004460E460027002068
:1052B0000690059004900390029001900A2E01DA66
:1052C00009B0F0BD0025CEE1A90060580021FBF730
:1052D00075FB06D8A9006058FB490968FBF764FB19
:1052E0000CD3A90060580021FBF75EFB7ED2A90019
:1052F0006058F6490968FBF761FBF7D20498401C37
:10530000C0B20490781CC7B2022F70D1012D49D1D0
:10531000ED49A0680968FBF751FB05D9EB49A06886
:105320000968FBF741FB7DD8E749E0680968FBF7AE
:1053300045FB05D9E549E0680968FBF735FB0BD863
:10534000E14920690968FBF739FB27D9DF49206962
:105350000968FBF729FB21D90021E068FBF724FB52
:105360000BD1D94920690968FBF728FB16D9D74921
:1053700020690968FBF718FB10D9D349E068096870
:10538000FBF71CFB05D9D149E0680968FBF70CFB6A
:10539000C9D800212069FBF707FB43D105950120FF
:1053A000069063E10F2DF8D1C749E06A0968FBF761
:1053B00005FB05D9C549E06A0968FBF7F5FAB2D8DB
:1053C000C149206B0968FBF7F9FA05D9BF49206B81
:1053D0000968FBF7E9FA0ED8BB49606B0968FBF76F
:1053E000EDFA2CD9B949606B096801E038E12CE08D
:1053F000FBF7DAFA23D90021206BFBF7D5FA0BD1A2
:10540000B149606B0968FBF7D9FA18D9AF49606BED
:105410000968FBF7C9FA12D9AB49206B0968FBF799
:10542000CDFA00E0FAE005D9A849206B0968FBF73E
:10543000BBFAADD80021606BFBF7B6FAADD1022004
:105440000690681EC0B2059010E1032F7EDB0D2F81
:105450007CDCF01EA84261DD691C890060589A4915
:105460000968FBF7ABFA07D9691C890060589749AE
:105470000968FBF799FA51D8A91C8900605892492C
:105480000968FBF79BFA07D9A91C890060588F4966
:105490000968FBF789FA0FD8E91C890060588A4926
:1054A0000968FBF78BFA35D9E91C890060588749F0
:1054B0000968FBF779FA2DD9A91C890060580021E9
:1054C000FBF772FA0FD1E91C890060587E49096820
:1054D000FBF774FA1ED9E91C890060587B490968FA
:1054E000FBF762FA16D9A91C890060587649096849
:1054F000FBF764FA07D9A91C890060587349096849
:10550000FBF752FA0AD8E91C890060580021FBF722
:105510004BFA03D1059501200690A7E0052D7DDB10
:10552000E91E8900605868490968FBF747FA07D9FE
:10553000E91E8900605865490968FBF735FA6DD89E
:10554000291F890060586049096800E04EE0FBF7B8
:1055500035FA07D9291F890060585C490968FBF7AB
:1055600023FA0FD8691F8900605857490968FBF76B
:1055700025FA35D9691F8900605854490968FBF735
:1055800013FA2DD9291F890060580021FBF70CFA66
:105590000FD1691F890060584B490968FBF70EFA63
:1055A0001ED9691F8900605848490968FBF7FCF952
:1055B00016D9291F8900605843490968FBF7FEF98D
:1055C00007D9291F8900605840490968FBF7ECF9A1
:1055D00047D8691F890060580021FBF7E5F940D1E1
:1055E00002200690A81EC0B205903FE00E2F38D1D1
:1055F0003549A06B0968FBF7E1F905D93349A06B80
:105600000968FBF7D1F910D82F49E06B0968FBF75F
:10561000D5F907D92D49E06B096800E021E0FBF7D7
:10562000C3F902D80320069020E0274920680968C2
:10563000FBF7C4F905D9254920680968FBF7B4F9D7
:105640000FD8214960680968FBF7B8F905D91F49E7
:1056500060680968FBF7A8F903D80420069005E004
:105660000027681CC5B2B54200DA2DE600BF0698D7
:10567000002863D1089020E0002515E06A1C920004
:10568000A158AA00A058FBF799F90BD2A8002058FE
:105690000390681C80002058A9006050691C890094
:1056A00003986050681CC5B2701E0899401AA84241
:1056B000E4DC0898401CC0B20890701E089988422B
:1056C000DADC022007900EE04403002048030020AB
:1056D0000798800021580298FAF72AFE029007984E
:1056E000401CC0B20790B01E07998842F0DC301F02
:1056F000FBF784F8014600900298FAF7AFFE02909B
:1057000009F00AF80A2818D10498032815DB0021AB
:105710000298FBF753F904D294490298FBF744F935
:1057200009D300210298FBF73FF906D2904902986D
:10573000FBF744F9F9D20020029014E10698012801
:105740004DD10598401CC0B205900598301AC6B2DC
:10575000002509E005982818800021580298FAF7DA
:10576000E7FD0290681CC5B2B542F3DB3046FBF79B
:1057700050F8014600900298FAF770FE019000215F
:105780000198FBF71BF904D27A490198FBF70CF951
:1057900009D300210198FBF707F919D2764901983E
:1057A000FBF70CF914D27548FAF792FD962808D841
:1057B00072480C30FAF78CFD962802D8002002902F
:1057C000D1E08321C9050298FAF748FE0290CAE0A9
:1057D0008321C9050298FAF741FE0290C3E00698BA
:1057E000022845D1002507E0A80021580298FAF7C1
:1057F0009FFD0290681CC5B205988542F4DB0598B0
:10580000FBF707F8014600900298FAF727FE01908F
:1058100000210198FBF7D2F804D256490198FBF712
:10582000C3F809D300210198FBF7BEF819D25249F9
:105830000198FBF7C3F814D25048FAF749FD9628AF
:1058400008D84E480C30FAF743FD962802D80020BD
:10585000029088E08321C9050298FAF7FFFD0290C3
:1058600081E08321C9050298FAF7F8FD02907AE0F9
:10587000069803283AD1E16BA06BFAF759FD029024
:10588000012189070298FAF7E9FD019000210198AA
:10589000FBF794F804D237490198FBF785F809D350
:1058A00000210198FBF780F819D233490198FBF7E2
:1058B00085F814D23148FAF70BFD962808D82F48FE
:1058C0000C30FAF705FD962802D8002002904AE035
:1058D0008321C9050298FAF7C1FD029043E08321B4
:1058E000C9050298FAF7BAFD02903CE00698042830
:1058F00039D161682068FAF71BFD02900121890700
:105900000298FAF7ABFD019000210198FBF756F8D9
:1059100004D218490198FBF747F809D300210198F0
:10592000FBF742F819D214490198FBF747F814D253
:105930001248FAF7CDFC962808D810480C30FAF730
:10594000C7FC962802D8002002900CE08321C905EC
:105950000298FAF783FD029005E08321C9050298B9
:10596000FAF77CFD02900298AAE400008FC2753D10
:105970008FC275BD0AD7233D0AD723BDFC1800206E
:10598000FEB504460E4600200290142E00DD1426BB
:10599000276820680190002518E0A8002158019888
:1059A000FBF70CF802D2A80020580190A80021585B
:1059B0003846FAF7F9FF01D2A8002758A800215865
:1059C0000298FAF7B5FC0290681CC5B2B542E4DB58
:1059D00039460298FAF7FDFC00900199FAF7F9FCB4
:1059E0000290B01EFAF70AFF014600900298FAF7FB
:1059F00035FDFEBDF3B597B00E460020169014900D
:105A00001390002515E0AA00179989582846EA0F37
:105A100012185210920003AB9950691C8A00179912
:105A20008958EA0F1218521092000BAB9950A81C1B
:105A3000C5B2B542E7DB00253AE000242FE0621C46
:105A4000920003AB9958A2009858FAF7B7FF0DD20D
:105A5000A00003A908581590601C80000858A100F8
:105A600003AA5050611C890015985050621C920086
:105A70000BAB9958A2009858FAF7A0FF0DD2A000DE
:105A80000BA908581590601C80000858A1000BAAAB
:105A90005050611C890015985050601CC4B2F10F21
:105AA00089194910491E491BA142C8DC681CC5B2AE
:105AB000F10F89194910491EA942BEDC01270FE0E8
:105AC000B80003AA11581498FAF732FC1490B800E1
:105AD0000BAA11581398FAF72BFC1390781CC7B235
:105AE000F10F89194910491EB942E9DC301FFAF754
:105AF00085FE029013991498FAF71AFC0190029906
:105B0000FAF7ACFC1690169819B0F0BD10B500204D
:105B1000C7494870022088700021C548C17006211D
:105B20000171002141718171DD20C149C871E521F8
:105B3000BF480172D6214172CA218172BD49C1722A
:105B4000090A01730020BA4948730021B8488173DB
:105B5000C17301210174072141741921817400204E
:105B6000B349C8740021B24801754175012181759E
:105B70000721C175992101760F2141760021817697
:105B80000020AB49C876012008770721A848417753
:105B9000192181770021C17730211C300171012149
:105BA0004171022181710721C171192101720146E0
:105BB0000931A148FAF7A4FB01219D482030417228
:105BC000002109304170142181708C21C1700521A0
:105BD00008380173002141739849801C0173090A38
:105BE00041730121C01E41740421113041706321B1
:105BF00081707421C1706E21017162214171512146
:105C00000F3041714921401D41704E218170472163
:105C1000C17044210171412141714F2181714A219B
:105C2000C1714921017243214172482181722D21A4
:105C3000C1724E210173472141734E21817342216C
:105C4000C1730021401F4175153041708170C170D2
:105C5000017141718171153801771C30417081707B
:105C6000C1700171417181710121001DC17000215C
:105C7000C01C41708170C170017133214171782164
:105C800081710021C01E81720421C17218210B3064
:105C9000417000218170AA21C170002101710B386F
:105CA00001744174014612310020FAF729FB604962
:105CB00076310020FAF724FB5D497A310120000497
:105CC000FAF71EFB5A497E3101200004FAF718FB4F
:105CD0005749823101200004FAF712FB54498631FA
:105CE00001200004FAF70CFB51498A31012000041D
:105CF000FAF706FB4E498E3101200004FAF700FB4B
:105D00005A214B4880308174C174002004E0002285
:105D1000474994310A54401C2028F8DB0F2144489D
:105D200080300175AA211430017255218172112130
:105D30004173232181737F21C173022101743221B8
:105D40004174002181740521C174017500214175E0
:105D5000072181751421C175B7210C30017500210F
:105D600041753749801C0175090A41750821801E5B
:105D70000176102141760F2181760421C17605211B
:105D80001B30417001211B384177E1218901801CC2
:105D90000177090A417728211E30017000214170E6
:105DA000811C0020FAF7ACFA00212148C030817133
:105DB000C171014608310020FAF7A2FA1C49D0311E
:105DC0000020FAF79DFA1A49D4311E48FAF798FADA
:105DD0001749D8310020FAF793FA1549DC31002031
:105DE000FAF78EFA00211248D03001824182014632
:105DF00014311548FAF784FA0D489430017C763056
:105E000001717638417C763041717638817C76300C
:105E1000C1707638C17C763081717638017D7338F7
:105E20000173090A41737330417D7630C17110BD31
:105E30003C20002033160000B80B00005203000085
:105E40001A2B0000E0D14D000000404010B514F0C6
:105E5000D5FB0B480078002804D0012803D0022885
:105E600007D103E009E000F017F806E000F0A4F91C
:105E700003E000200249087000BF00BF10BD000011
:105E8000CA04002003480078002801D1012070478F
:105E90000020FCE7CB04002010B5BB4800780828A0
:105EA0007CD007DC030015F00AF90812447C7C5B07
:105EB0008EAAB07C162872D004DC092870D00A287B
:105EC0006FD1F7E017286DD01828F9D11DE101F046
:105ED0003BFD01282CD1AD48C07A401CAB49C872AB
:105EE000C87A0A21FAF72AF9C8B2A849C872E1218A
:105EF0000901242010F040FFA5480088401CA44957
:105F000008800D2000F08EFD0002000EAA2801D1AD
:105F10000EF0C2FA55219F488170232000F08AFDBF
:105F2000482000F087FD0BF057FE012096490870CD
:105F30001BE10CF0BDF8002803D004209249087042
:105F40000DE00CF0ABF8002809D093480CF024FFCA
:105F50009249252010F010FF04208B49087004E1BD
:105F60000CF0A6F800281ED001F0FAFC092806D192
:105F700002208B49087006208349087022E0894876
:105F8000027BC37A10021843014600228548C01DD7
:105F90000BF012FD05207C49087013E04FE0A2E0F1
:105FA00060E0DEE0A9E07C480078A52804D0252048
:105FB000FDF736FD002805D1F1207949087006204B
:105FC00071490870D1E00020FEF7E0FA002806D001
:105FD00001207349087006206B4908700EE06E4876
:105FE0000078A52804D02520FDF71AFD002805D14A
:105FF000F1206B490870062063490870B5E002F093
:10600000A1FA072060490870AFE0674A6749644811
:10601000007801F0AFFE01F00BFD01280ED101F078
:1060200021FD012803D108205749087006E03221DC
:10603000262010F0A1FE0A205349087095E00CF0CC
:106040002DF801280DD1544B00225748018857489C
:106050000DF0D6FC6421262010F08EFE09204A495E
:10606000087082E0232000F0D3FC012804D0262011
:10607000FDF7D6FC00280FD1232000F0DBFC022026
:106080004749087000214348417001200BF028FD6A
:1060900007203D4908700CE03F480078A52808D14A
:1060A00032213C48417003203D49087007203649A1
:1060B00008705AE0482000F0ABFC002806D04820C9
:1060C00000F0B8FC3221262010F056FE2620FDF705
:1060D000A7FC002806D101F08FFC012802D1162070
:1060E0002949087041E00BF0D9FF002804D010F0D6
:1060F00027FF17202449087037E00BF0CFFF002856
:1061000002D01820204908702FE0FEF78FFC0128EC
:1061100026D10D2000F086FC0002000EAA280FD127
:1061200000211C48763881700020214908700B46F8
:106130000122962117487438FEF7D4FE00F0C8FEFD
:106140000BF0F6FC13F02AFFFDF760FEFDF750FDA3
:1061500000211048817000200B4908701549087013
:1061600003E000200849087000BF00BFFFF78AFE67
:10617000002807D12420FDF753FC002802D1182065
:106180000149087010BD0000CB04002063230020EB
:10619000D204002046210020C2040020B80B0000D9
:1061A000D40400203C200020C004002063210020F3
:1061B000D8040020CA04002010B5FD480078030070
:1061C00014F07DFF190E3D5EF175A0DBF2EFEEEDF0
:1061D000F1F1ECEBEAE9E8E7E6E5E4E3E2E1F1001E
:1061E00001F0B2FB012829D1F248C07A401CF149E4
:1061F000C872C87A0A21F9F7A1FFC8B2ED49C8727E
:10620000E1210901242010F0B7FDEB480088401C73
:10621000E94908800D2000F005FC0002000EAA28C4
:1062200001D10EF039F9232000F004FC482000F0E1
:1062300001FC0BF0D1FC0120DD49087090E20BF06D
:1062400037FF00280DD019F0C5FF002805D00DF04C
:106250007BF90220D649087011E00420D449087067
:106260000DE00BF01BFF002809D0D4480CF094FD82
:10627000D349252010F080FD0420CD4908706FE23D
:106280000BF00CFF012811D119F0A4FF012803D154
:106290000520C749087009E0C8480CF07DFDC849D1
:1062A000252010F069FD0420C149087058E20BF068
:1062B000FFFE002812D0002104201BF047FAC1483D
:1062C000027BC37A1002184301460022BD48C01D5C
:1062D0000BF072FB0520B649087012E0B748007851
:1062E000A52804D02520FDF79BFB002809D101211A
:1062F00004201BF02BFAF120B34908700620AC49AA
:1063000008702DE20020FEF741F9002825D019F091
:1063100061FF012805D1AC4908700620A449087026
:106320002AE0072019F06AFF01280FD10021072079
:106330001BF00CFA012019F061FF044621462620CB
:1063400010F01AFD0A209A49087015E001209E49B4
:1063500008700620964908700EE098480078A52835
:1063600004D02520FDF75CFB002805D1F1209649DB
:10637000087006208E490870F2E102F0E3F8072069
:106380008B490870ECE1BBE1B2E1A7E18BE180E170
:106390005EE142E12EE1F8E0F1E0D8E0B4E059E05E
:1063A00033E01FE000E0D7E1884A89498648007859
:1063B00001F0D8FD01F046FB012812D101F058FB95
:1063C000012803D108207A4908700AE0012019F059
:1063D00015FF04462146262010F0CEFC0A20744901
:1063E0000870BDE10BF05AFE01280DD1734B00225D
:1063F0007648018876480DF003FB6421262010F0D2
:10640000BBFC09206A490870AAE1232000F000FBC8
:10641000012804D02620FDF703FB00280FD12320FC
:1064200000F008FB00206B490870022066490870E4
:1064300000216948417007205D49087009E05F4804
:106440000078A52805D103205F4908700720584926
:10645000087085E1482000F0DBFA00280BD04820C6
:1064600000F0E8FA012019F0C9FE04462146262072
:1064700010F082FC47E02620FDF7D2FA002842D136
:1064800001F0BAFA01283ED101F05EFA01280FD1DD
:106490004848C07A401C4749C872C87A0A21F9F7AF
:1064A0004DFEC8B24349C8720520414908702AE030
:1064B00019F090FE012815D147487638007B8021DD
:1064C000084000280AD044487638007B8007800FB7
:1064D000002803D014203649087014E00D203449F8
:1064E000087010E0062019F089FE012808D1042068
:1064F00019F084FE002803D10D202D49087002E018
:1065000016202B4908702BE101F076FA01281DD1E5
:106510000BF0C4FD002819D000202B4908702E482C
:106520002238827E437E10021843014601222A4807
:106530000D380BF041FA012019F060FE04462146A7
:10654000262010F019FC0E201949087008E10120DE
:10655000FEF71CF8002806D001201B4908700F2008
:10656000134908700AE02620FDF75AFA002805D1E1
:10657000F120154908700F200D490870F0E001F076
:10658000D5FF10200A490870EAE0104A10490E4869
:10659000007801F073FA01F041FA012829D101F0E5
:1065A0005BFA01281AD111200149087021E000008E
:1065B000CB04002063230020D2040020C20400206A
:1065C000B80B00003C200020D4040020C0040020B0
:1065D00063210020D504002046210020012019F06D
:1065E0000DFE04462146262010F0C6FB1320634909
:1065F0000870B5E00BF052FD01280DD1604B01226F
:106600006048018860480DF0FBF93221262010F027
:10661000B3FB122059490870A2E0232000F0F8F9DA
:10662000012809D1232000F005FA022057490870FB
:106630001020524908700AE02620FDF7F1F90028E1
:1066400005D103205149087010204C49087087E09B
:10665000482000F0DDF9002803D113F0A5FC012843
:106660000AD1482000F0E6F9012019F0C7FD0446E0
:106670002146262010F080FB2620FDF7D1F90028C6
:1066800006D101F0B9F9012802D116203B49087062
:1066900066E00BF003FD012804D10CF041FF15204A
:1066A000364908705CE00BF0F9FC012815D119F0AF
:1066B00091FD02280ED101213548017213F06EFCC4
:1066C000FDF7A4FBFDF794FA00202C49087031492E
:1066D000087002E016202949087041E00BF0DEFC4A
:1066E000002804D010F02CFC17202449087037E053
:1066F0000BF0D4FC002802D01820204908702FE0AD
:10670000FEF794F9012826D10D2000F08BF9000244
:10671000000EAA280FD100211D4876388170002074
:106720001D4908700B460122962119487438FEF75E
:10673000D9FB00F0CDFB0BF0FBF913F02FFCFDF7BC
:1067400065FBFDF755FA00211148017200200B4945
:1067500008701049087003E000200849087000BF65
:1067600000BFFFF78FFB002807D12420FDF758F961
:10677000002802D118200149087010BDCB04002068
:10678000C2040020C004002063210020D4040020A3
:1067900046210020CA040020D8040020F0B58BB0A8
:1067A00005460E4600242A480A9000200990202120
:1067B00001A8F9F766FD274F012D0ED0022D0CD050
:1067C000042D0AD0062D08D0082D06D00C2D04D09B
:1067D0000420099009980BB0F0BD1E48006A012101
:1067E00049028843710201225202114008431949AB
:1067F0000862002407E0A000174908586843A10078
:1068000001AA5050641C082CF5D300241CE0104849
:106810000A9011E00A98411E0A9100280AD00F48F8
:106820000C49C8620E48C862A00001A90858A1001E
:10683000785001E00720CEE7A0003858A10001AA57
:1068400051588842E6D1641C082CE0D30998C2E76D
:10685000FFFFFF0000000240842502005A5A00009A
:10686000A5A5000010B501460020084A084BDA62D1
:10687000084ADA621A46126A0C239A438B000C24E7
:1068800023401A43024B1A6210BD00005A5A0000FE
:1068900000000240A5A5000070B504464721090686
:1068A0002046FAF78BF801D2002070BD8F21C90570
:1068B0002046F9F796FD0546F9F7D4FFF5E7000005
:1068C00010B5002407F044FE044609480088201A49
:1068D00080B208490860064804800846006805211F
:1068E0000902884203D3032000020249086010BD58
:1068F000C0030020BC03002070B53D48007800288C
:1069000006D0012805D0032862D006286AD123E0EA
:106910006CE0FEF78BF801281DD136480078162868
:106920000FD0482234493548F9F792FC344B4822BD
:106930000D2189013148FEF7D5FA03202C49087052
:1069400009E02F4B48222D490D208001FEF784FAE3
:1069500006202749087049E0FEF768F8012836D17B
:10696000012500241EE0A100244A8818F9F7B0FC94
:106970000021C943884201D1002515E0A1001F4A2A
:106980008818F9F7A5FC1F49884207D8A1001B4ABF
:106990008818F9F79DFC1C49884201D2002503E0C4
:1069A000601CC4B2122CDEDB00BF002D0BD14822CC
:1069B00011491248F9F74CFC114B48220D2189016D
:1069C0000E48FEF78FFA03200949087000BF0DE05A
:1069D000FEF72CF8012804D10C4908700020044966
:1069E000087003E000200249087000BF00BF70BDBE
:1069F000B60400203C200020082A0200DF360020D8
:106A0000B50400209919010066E60000B7040020D3
:106A100001465B2902DA0248405C70470020FCE72F
:106A20006431002001468800014A10587047000078
:106A3000981F002001465B2904DA0020024A5054C6
:106A4000012070470020FCE76431002070B5064645
:106A5000002405F0B9FEC4B2E007C00F00280ED034
:106A6000A548007802218843801CA3490870084685
:106A7000C0784021884340309F49C8700BE09E4851
:106A80000078022188439C4908700846C07840215C
:106A900088439949C8700220204002280ED19648A8
:106AA0000078202188432030934908700846C07838
:106AB0002021884320309049C8700BE08E48007830
:106AC000202188438C4908700846C07820218843DB
:106AD0008949C87004202040042807D1864840789E
:106AE00040084000401C8449487005E082484078D6
:106AF000400840008049487008202040082807D1FD
:106B00007D48407804218843001D7B49487005E09A
:106B100079484078042188437749487020202040F4
:106B2000202807D17448407802218843801C72498C
:106B3000487005E070484078022188436E494870EB
:106B40004020204040280ED16B480078400840008B
:106B5000401C694908700846C0788021884380300D
:106B60006549C8700BE064480078400840006249FD
:106B700008700846C078802188435F49C87080202B
:106B8000204080280ED15C48007840218843403066
:106B9000594908700846C07804218843001D5649A9
:106BA000C8700BE05448007840218843524908706F
:106BB0000846C078042188434F49C870FCF7C0FFDD
:106BC000012807D14C4840781021884310304A49A9
:106BD000487005E04848407810218843464948708D
:106BE0001020204010280ED1434800780821884307
:106BF0000830414908700846C07810218843103099
:106C00003D49C8700BE03C480078082188433A4968
:106C100008700846C078102188433749C8700DF0C5
:106C200017FD0A2807D134484078202188432030B6
:106C30003149487005E030484078202188432E498A
:106C400048702D484078C02188432B4948700FF088
:106C500001F901280ED12848007804218843001D3D
:106C6000254908700846C078082188430830224921
:106C7000C8700BE020480078042188431E49087042
:106C80000846C078082188431B49C870FCF71EFFDE
:106C9000012807D118484078082188430830164950
:106CA000487005E01448407808218843124948702C
:106CB0001148C07840084000401C0F49C870084681
:106CC000807840084000401C8870092019F096FA2E
:106CD000094989780843084988700DF0BFFC0546CA
:106CE000C00F4019C005000E034908710522304647
:106CF000F9F7AEFA70BD0000E00A00200348007802
:106D0000002801D1012070470020FCE7F006002098
:106D100010B50CF057FC11F0B9FC10BD5B2802DA7D
:106D20000121014A115470476431002070B50446B6
:106D30000E460025FE20207060706820A070102094
:106D4000E0705E484078102809D100BF04E05C483C
:106D5000415D281D21546D1C072DF8DB24E05948A6
:106D6000407801280DD1002056494870002505E0E3
:106D70005448801C415D281D21546D1C072DF7DBF4
:106D800009E0002505E04E480E30415D281D2154E4
:106D90006D1C072DF7DB49484078112804D149487C
:106DA000417A201DFCF78AFA44484078492811D0DE
:106DB00006DC11280BD045280AD046284CD108E023
:106DC000512808D0542807D0642845D105E000BFD9
:106DD00000BF00BF00BF00BF00BF38488078E0722E
:106DE00039480078001D20733448007960733348B7
:106DF0004079A07331488079E0733048007A20747C
:106E0000002505E03148415D2846113021546D1CB4
:106E10002D4800888542F5DB28484078912805D127
:106E20002648017A20461130FCF748FA2348027AB6
:106E3000207B0B30C1B2A01C0FF0DCF8224909887E
:106E400011316054162120480088123021541E4808
:106E50000088133030802FE018488078E0721A489C
:106E60000078C01C2073154800796073134840797E
:106E7000A07312488079E073002505E01348415D56
:106E80002846103021546D1C0F4800888542F5DBE0
:106E9000207B0B30C1B2A01C14F0D2FB0A49098838
:106EA00010316054162108480088113021540648DA
:106EB00000881230308000BF00BF70BD0B3B002047
:106EC00091200020013B0020580B0020183B00209F
:106ED0001FB51520AB490860AB48F9F7F9F9A94986
:106EE0004860A948001DF9F7F3F9A6498860A6484B
:106EF0000830F9F7EDF9A349C860A3480C30F9F759
:106F0000E7F9A0490861A0481030F9F7E1F99D4977
:106F100048619D481430F9F7DBF99A4988619A482D
:106F20001C30F9F7D5F99749C86197487238007F46
:106F300095497239497F0902084393497239897F1B
:106F4000090408438F4908628F485638007A8E49F1
:106F50005639C979090208438B4956398979090498
:106F60000843884948628948886287481238C0784F
:106F700085490F3949780902084383490F398978CF
:106F80000904084380490F39C978090608437D4937
:106F9000C8627D480F3800797B490F394979090269
:106FA000084379490F398979090408437549086309
:106FB00075480E30007D7449223149780902084332
:106FC000714922318978090408436F492231C9780F
:106FD000090608436B4948636B48223000796A49C7
:106FE0002231497909020843674922318979090424
:106FF000084365492231C979090608436149886314
:1070000061482230007A60492231497A09020843F6
:107010005D492231897A090408435B492231C97AE2
:10702000090608435749C86357482230007B564930
:107030002231497B0902084353492231897B0904E3
:10704000084351492231C97B090608434D49086468
:107050004D487238C07F4C495639097909020843B6
:10706000494956394979090408434649486446481C
:107070001830F9F72DF9434988646846FFF7E6FCB4
:1070800001990098039102906946487A897A090229
:1070900008433C4948653C482E30807D3A4944319C
:1070A0004978090208433749886537482E30417DC1
:1070B000027D080210433349C86533482E30007EF4
:1070C000086631482E30407E48662F4872388078F6
:1070D0002D497239C978090208432B497239097957
:1070E00009040843284972394979090608432549A2
:1070F000886725480E30807CC86723480E30C17CE5
:107100002048803001602048723841781D48803026
:1071100041601D482E30817E1A48803081601A48B7
:107120003030417F027F08021043164980314861A8
:1071300015484E30417802780802104311498031D9
:1071400088610AF065FA0F498031C8610E48223023
:10715000017C763001717638417C76304171763829
:10716000817C7630C1707638C17C7630817176381A
:10717000017D73380173090A41737330417D7630A4
:10718000C1711FBD981F0020AE200020090026B24B
:107190000020014908707047180B002000200149A9
:1071A000087070475B0B0020002001490870704791
:1071B0006C0B002030B589B004460D46114881782B
:1071C000684681750F480179684601760D48417916
:1071D000684641760B48C17A6846C177094881798B
:1071E000684681760748C1796846C17606480088B6
:1071F000064901AA31C2009105A80FC800F008F89D
:1072000009B030BD033A00200A0B002003380020EB
:10721000FFB581B00D9F0B9E0C9C0025FE202070B9
:1072200060706820A0701020E07000BF04E0584833
:10723000415D281D21546D1C072DF8DB68468079BF
:10724000E0726846C07B2073FB2E45DC301D607306
:107250006846007AA0736846407AE0736846807A90
:1072600020746846C07A60743246204612300A990B
:10727000F8F7EEFF6846C07BC007C00F00280FD0AC
:10728000627B444B21460E310020F9F73DFD607BC7
:10729000C117090F09180911491C0907090E617363
:1072A0000021607B0E302154022509E0607B0E3006
:1072B000205C615D4018C1B2607B0E3021546D1CB2
:1072C000607B0E30A842F1DC1621607B0F30215428
:1072D000607B1030388058E0301D81B200916846E4
:1072E0000078607368464078A0736846007AE0735F
:1072F0006846407A20746846807A60746846C07A2E
:10730000A0743246204613300A99F8F7A1FF684668
:10731000C07BC007C00F002816D069460A881D4BE5
:1073200021460F310120F9F7EFFC69460888C117A3
:10733000090F09180911491C09050A0C0092694630
:10734000487860730878A0730021684600880F3081
:10735000215402250BE0684600880F30205C615DF7
:107360004018C1B2684600880F3021546D1C684631
:1073700000880F30A842EEDC1621684600881030E5
:107380002154684600881130388005B0F0BD0000F7
:107390009F200020F70A002030B589B004460D4632
:1073A00011488178684681750F48017968460176F1
:1073B0000D484179684641760B48C17A6846C177E5
:1073C00009488179684681760748C1796846C1765F
:1073D00006480088064901AA31C2009105A80FC8D5
:1073E000FFF716FF09B030BD183F00205E0B0020EC
:1073F000183D0020014800787047000084020020FA
:107400001CB50721684614F0B1FC012168464170A3
:10741000C1706A460221C02005F0E6FD0322022168
:10742000C02005F0B7FD012203210846FDF716FE36
:107430001CBD000010B500F00FF91348F8F748FF25
:107440001249884205D1002203210A20FDF706FED9
:107450000AE00D48F8F73CFF0D49884204D10022AC
:1074600003210B20FDF7FAFD0748F8F731FF032150
:1074700001610548F8F72CFF142101600021072065
:1074800010F05EFC10BD0000FC120020000800405F
:107490000048004010B500F025F81148F8F718FF33
:1074A00000694021884344180D48F8F711FF046132
:1074B0000B48F8F70DFF006920218843441808485D
:1074C000F8F706FF04610648F8F702FF0069042197
:1074D0008843041D0248F8F7FBFE046110BD00005C
:1074E000FC12002038B580200EF04AF800F06AF84F
:1074F0000121072010F024FC2F493048F8F700FF45
:107500002D48F8F7E5FE00684021884304462A48E4
:10751000F8F7DEFE04602849091D0020F8F7F0FEA8
:10752000254908310420F8F7EBFE234910310220E9
:10753000F8F7E6FE1021684601701F481030F8F792
:10754000C7FEC1B2684641701B480830F8F7C0FE5C
:10755000C1B26846C1701848001DF8F7B9FEC1B243
:10756000684681701448F8F7B3FE044669460FF088
:107570008DFC1148F8F7ACFE1149884205D1012273
:1075800003210A20FDF76AFD0AE00B48F8F7A0FE88
:107590000A49884204D1012203210B20FDF75EFD38
:1075A0000548F8F795FE00684021884344180248D2
:1075B000F8F78EFE046038BDFC1200200048004041
:1075C000000800401CB50721684614F0CFFB0021DD
:1075D000684641706A46C02005F006FD022200217F
:1075E000C02005F04FFD01220021C02005F062FD02
:1075F000012118480FF064FC6A460121C02005F003
:10760000F3FC02220121C02005F03CFD00220121F3
:10761000C02005F04FFD6A460421C02005F0E4FCBF
:1076200002220421C02005F02DFD00220421C020EB
:1076300005F040FD01216846417001716A46032151
:10764000C02005F0D1FC02220321C02005F01AFD64
:107650001CBD0000004800401CB50721684614F01E
:1076600085FB0020694648706A460121C02005F06C
:10767000BBFC00220121C02005F004FD00220121F5
:10768000C02005F017FD6A460421C02005F0ACFCBF
:1076900000220421C02005F0F5FC00220421C020B6
:1076A00005F008FD6A460321C02005F09DFC00227C
:1076B0000321C02005F0E6FC00220321C02005F0D4
:1076C000F9FC6A460021C02005F08EFC002211461C
:1076D000C02005F0D7FC01220021C02005F0EAFC03
:1076E0001CBD00000148007870470000C203002064
:1076F0000020014908707047C203002001200149A1
:1077000008707047C203002070B504460025552C50
:1077100003D10EF07DFA054613E0012C04D10120BF
:1077200004F0DCFF05460CE0022C04D1022004F03A
:10773000D5FF054605E0032C03D1032004F0CEFF5E
:107740000546284670BD000070B504460025112C82
:1077500012D13A480EF03EFA00280BD03748007894
:1077600000040543354840780002054333488078DB
:10777000054361E0324D5FE0222C12D131480EF01A
:1077800029FA00280BD02F480079000405432D4822
:107790004079000205432B48807905434CE0284D91
:1077A0004AE0012C04D10020FFF73CF9054643E0F4
:1077B000022C04D10A20FFF735F905463CE0042CE1
:1077C00004D10B20FFF72EF9054635E0032C04D138
:1077D0000C20FFF727F905462EE0052C04D10620E2
:1077E0000DF092FE054627E0062C04D107200DF08F
:1077F0008BFE054620E0072C04D108200DF084FE06
:10780000054619E0082C04D109200DF07DFE05463F
:1078100012E0092C04D10A200DF076FE05460BE09B
:107820000A2C04D12720FFF7FDF8054604E00B2CB5
:1078300002D119F0F3FF0546284670BD1C04002054
:10784000EEEEEE002304002070B506460024234827
:107850000578012E27D108202840082801D10443AB
:1078600003E00821204688430446042028400428D9
:1078700001D1044303E0042120468843044602204A
:107880002840022801D1044303E002212046884316
:10789000044640202840402802D1012004431AE039
:1078A0006408640017E0022E15D11020284010282B
:1078B00001D1044303E010212046884304460120FF
:1078C0000AF0DAF8002802D08020044303E0802187
:1078D000204688430446204670BD0000070400206F
:1078E00038B504460025022C03D104F09FFF05465D
:1078F00022E0012C04D10C2004F098FF05461BE087
:107900000A2C04D10A2004F091FF054614E0042C4F
:1079100004D1042004F08AFF05460DE0072C04D1B1
:10792000072004F083FF054606E00E2C04D110F07A
:10793000EFFB0090009838BD2846FCE7024610682F
:10794000C840C007C00F70470448807A0349C97A0D
:10795000884201D0012070470020FCE7632300200B
:107960000248C07A0149085C704700006323002088
:107970000248007802490968087070473600002004
:10798000140000200148007870470000DC0200204D
:1079900010B580200DF0E8FD04466006040E40207E
:1079A0000DF0E2FD04436006040E20200DF0DCFD26
:1079B00004436006040E10200DF0D6FD044360065B
:1079C000040E08200DF0D0FD04436006040E0420D0
:1079D0000DF0CAFD04436006040E02200DF0C4FD44
:1079E00004436006040E01200DF0BEFD0443600652
:1079F000040E204610BD00000148007870470000CA
:107A0000F50600200148007870470000640400205B
:107A10000148407A70470000CF2E002003480078CC
:107A2000002801D1012070470020FCE7190B00203D
:107A300003480078002801D1012070470020FCE7AE
:107A40001B0B002003480078002801D1012070475B
:107A50000020FCE7700B0020014800787047000010
:107A60001A0B002001480078704700001C0B002012
:107A70000148007870470000710B0020F0B591B00C
:107A800005460E461746012D7ED1002006900620A1
:107A900004F0CCFE80B2B0490870000A487009209A
:107AA00004F0C4FE80B2AC498870000AC87010F0BF
:107AB0002FFB059000210598F8F776FF1BD2E90708
:107AC000059848400590A5490598F8F78AFC0446B2
:107AD000F8F7C8FE81B2A0480171090A4171014658
:107AE0004879097900020843E90308439A49087173
:107AF000000A487115E099490598F8F772FC0446A8
:107B0000F8F7B0FE80B294490871000A48714879CC
:107B10000979000208434104490C8F480171090AA0
:107B2000417100208C498871C8710A2004F07EFEE2
:107B3000044689490831F8F7E3FB87490C31884846
:107B4000F8F7DEFB8748F8F7C3FB87490390F8F79F
:107B500048FC0490F8F786FE04467F491031F8F798
:107B6000CFFB804914394A7C0B7C1102194308462B
:107B700079491431F8F7C4FB774918310020F8F738
:107B8000BFFB09F04DFD00E0DDE00012724908770F
:107B900009F046FDC1B270484177090A81770CF0BF
:107BA0005DFD6D49C91C0877000A487706A80AF0F0
:107BB00051FA6846008B404281B26748213001701B
:107BC000090A417006A80AF053FA68461821415E76
:107BD00000290EDA008B4042C1B25F482030C170EC
:107BE000C0780121C9034018C1B25B482030C17080
:107BF00005E06846008BC1B257482030C1700AA822
:107C00000AF0C8F9544925310020F8F779FB00241F
:107C10004BE00AA8005D002846D04F482530F8F711
:107C200057FB00014C4925310490F8F769FB0AA87D
:107C3000005D39280DDC48482530F8F749FB0AA9D2
:107C4000095D30390843444925310490F8F758FB61
:107C50002AE00AA8005D662811DC0AA8005D6128F8
:107C60000DDB3D482530F8F733FB0AA9095D57398C
:107C70000843394925310490F8F742FB14E00AA87B
:107C8000005D462810DC0AA8005D41280CDB324864
:107C90002530F8F71DFB0AA9095D373908432E493D
:107CA00025310490F8F72CFB641C0A2CB1DB0AF098
:107CB000C5F929492031487203A8FEF7C7FE049987
:107CC00003980991089008A801782348203081740E
:107CD00008A8417820482030C17408A881781E483F
:107CE0002030017502214175022004F0F7FC079055
:107CF0001D490798F8F775FB0490F8F7B3FD0446A3
:107D000015493631F8F7FCFA13493A310020F8F7F3
:107D1000F7FA672108A8817531210176A121417602
:107D20000321C177122181763421C1763E200A4990
:107D300001AAC1C200910DA80FC8FFF769FA01207E
:107D40000A49087002E0022008490870002008492A
:107D5000087011B0F0BD0000903A00200000C84249
:107D600026B2000020210020000020411A0B002034
:107D7000190B0020F0B591B004460D461646012CB3
:107D80007ED1002071490870022004F0A7FC0C90FD
:107D90006F490020F8F7B4FA6E490C98F8F721FB08
:107DA0000490F8F75FFD07466949091FF8F7A8FA3C
:107DB00002A812F01BFD02A807C809AB07C3694659
:107DC000888C0A21F8F7BAF96149091F08720CF08A
:107DD00045FC5F49091F4872000A88726846018D98
:107DE0005B48001FC172090A01736846408D5849FB
:107DF000091F48730FA80DF0EDFE10A840785449F4
:107E0000091F887310A801785148001FC17308A882
:107E1000817F4F48001F017408A8417F4C48001F14
:107E2000417408A8017F4A48001F817403A8FEF727
:107E30000DFE049903980E910D9008A8007D444909
:107E4000091FC87408A8417D4148001F017508A892
:107E5000817D3F48001F417502218175092018F07E
:107E6000CDF93B49091F897D08433949091F8875A8
:107E70000A20FEF7D7FD0002010E3548001F00E082
:107E80002DE001760A20FEF7CDFD000E3049091FD6
:107E9000C87510F03DF90746F8F7E4FC81B22C48AC
:107EA000001F4176090A81769A2168468175022170
:107EB0000176102141760321C17756218176782100
:107EC000C1761B202249091F01AA61C2009105A8A1
:107ED0000FC8FFF79DF901201F49087030E0032CFF
:107EE00010D11A480078012808DA18480078401C98
:107EF0001649087001201849087021E0022016492F
:107F000008701DE0F12C14D11448007D002808DD14
:107F10000AF0CEF8002804D00021012009F0E0FD8D
:107F200003E032210D488A30417002200A4908706E
:107F300006E00021012009F0D3FD02200649087067
:107F400000200749087011B0F0BD00001D0B002093
:107F5000D23A0020000020411C0B0020BC20002051
:107F60001B0B0020F0B589B004460D461646FB48B1
:107F70000078152877D00CDC022875D004DC0028A6
:107F800010D0012871D1C9E00A286FD01428F9D186
:107F900083E11E286BD01F286AD0202869D02128B1
:107FA000F0D18EE2012C21D10020ED490870ED497D
:107FB0000870ED48C079202802DB0021EA48C17131
:107FC000E948C079002803D11F21E748817105E005
:107FD000E548C079401EC1B2E34881710121042007
:107FE00019F0A0FB0120DD49087096E0022C4CD16D
:107FF000DB480078012827D10FF05CFF0121022027
:1080000019F090FB0020D7490870D7482C38C07968
:1080100055280ED10F20FEF705FD0004000EAA28FA
:1080200003D11E20CD49087077E00A20CB490870A3
:1080300073E00021012009F053FD0220CB490870B4
:108040000020C649087068E0C54800780A2811D1A8
:108050000121022019F066FB0020C24908700A20A5
:10806000BE49087059E095E174E03DE2BAE0CFE125
:10807000DBE1EFE1BA4800781E284ED10020B94973
:1080800008702120B549087047E0032C03D1152062
:10809000B249087041E0F12C39D1B348C0792028A9
:1080A00002DB0021B048C171AF48C079002803D17C
:1080B0001F21AD48817105E0AB48C079401EC1B2B7
:1080C000A9488171FFF74CFC072803D0FFF748FC53
:1080D000012804D10121084619F024FB10E0FFF724
:1080E0003FFC002806D10121084619F01BFB0FF0C8
:1080F000C9FE05E0FFF734FC032801D10FF0C2FEF2
:1081000002209A49087000209449087005E0022076
:1081100096490870002091490870ECE19448007875
:10812000002816D1FCF782FC002812D08E498979EC
:108130009B22514301225203891888B28D4B9B2206
:108140008D49FCF789FE012085490870022083498A
:108150000870D0E1FCF76AFC002842D001200DF045
:10816000EDFC002836D08048A43881798348C17658
:108170007D48A438C17981481B3041707A48A438C1
:10818000017A7E481B30817008A881787B481B30BB
:10819000C17008A8417879481B30017108A801789E
:1081A00076481B3041712021817108A80DF000FD37
:1081B00007A804F035FB002005E007990A5C6E492A
:1081C0009B310A54401CC028F7DBFF2063306C4908
:1081D000088002E09B206A49088014205F490870EB
:1081E00000BF88E167480078002855D1FCF71EFCE5
:1081F000002851D000205F490870FF215A48817142
:10820000C7790CE05848801CF8F762F80121B940A2
:108210000840002802D05448877102E07F1E002FDA
:10822000F0DA00BF50488079FF2814D11F270CE0F6
:108230004D48801CF8F74CF80121B940084000284F
:1082400002D04948877105E07F1E4748C079401E2B
:10825000B842EDDB00BF44488079FF2806D10220F8
:108260004249087000203D49087015E03E4989796F
:108270009B22514301225203891888B23D4B9B2215
:108280003D49FCF7E9FD9B203D4908800A2034491F
:1082900008701420314908702DE1FCF7C7FB002855
:1082A0005BD00F20FEF7BEFBC0B2AA282AD19A20CD
:1082B0003549887002200871102048710320C87267
:1082C00032480088401C31490880084600782E4911
:1082D00088712E4800880012C8711B202849088028
:1082E00012F0BAFC2648008829490D2201AB61C36F
:1082F0000091254905A8F7F7ABFF05A80FC8FEF7C1
:1083000087FF24E067202049887043200871A1205E
:1083100048710320C8721D480088401C1B49088012
:108320000846007818498871184800880012C871FA
:108330001348008810490D2201AB61C30091124916
:1083400005A8F7F785FF05A80FC8FEF761FF012014
:1083500006490870002001490870CCE0700B00202D
:10836000750B0020740B0020FC200020710B0020F6
:10837000790B00205C0B0020413F00208140002051
:10838000720B0020840B0020253F00206E0B002084
:108390000542002059480078012810DA5748007833
:1083A000401C56490870564800781E2803D12020EA
:1083B000544908702BE014205249087027E05048B7
:1083C000007801281DD1FFF7CBFA072803D0FFF76B
:1083D000C7FA012804D10121084619F0A3F910E0D9
:1083E000FFF7BEFA002806D10121084619F09AF9D4
:1083F0000FF048FD05E0FFF7B3FA032801D10FF0B5
:1084000041FD02204049087000203E49087072E09A
:10841000FCF70CFB002807D01E20394908700EF02D
:108420009FFD1F203749087065E00EF00BFF0FF02D
:1084300001F801280DD135480078002803D020200C
:108440003049087005E002202F49087000202D49AE
:10845000087050E0FCF7EAFA002831D09B202C4944
:10846000887001200871102048710320C8722948C3
:108470000088401C274908800846007824498871F4
:10848000244800880012C871204800780C21484315
:10849000401C214908800846008820490D2201AB74
:1084A00061C300911A4905A8F7F7D2FE05A80FC8C5
:1084B000FEF7AEFE01201449087000201149087033
:1084C00019E0FCF7B3FA00280DD0154915480068EB
:1084D000F7F716FF144B0622C2211148FCF702FDE4
:1084E0001E200849087006E0022007490870002095
:1084F0000449087000BF00BF09B0F0BD740B002034
:10850000750B0020700B0020710B0020780B0020F1
:10851000253F00206E0B0020720B0020204200201F
:10852000FE200020880B00205C0B00200120034966
:10853000087000200249087070470000190B0020E5
:108540001A0B002000200249087002490870704789
:10855000700B0020710B0020F0B589B000240020C2
:1085600008900590049000260027FA48007800281B
:1085700002D001287ED129E000F0C4FEF64908604F
:1085800008460068042820D006F0C6F80A2814D14E
:10859000F2480078401CF14908700321EF48007848
:1085A000F7F7CCFD00290DD10020EC4908700FF041
:1085B00053FF0A20EA49087004E00FF04DFF0A203B
:1085C000E74908700120E349087063E3E248007856
:1085D000C007C00F00287DD00020E249087100F0DC
:1085E000ABFE0020E04908700B2017F05FFE07A8E3
:1085F00000F0BEFE06A804F03BF802A800F0A8FEBA
:1086000003A804F041F80024BDE2A000079908582F
:10861000A100D64A5050A00006990858A100D44A9B
:108620005050082C7EDAA00003990858A100D14AC6
:108630005050A00002990858A100CF4A5050A00005
:10864000CC49085C0006A100CA4A5158FF22120218
:10865000114009020843A100C64A5158FF221204E2
:108660001140090A0843A100C24A5158090E0843A3
:10867000A10000E00DE35050A000BF49085C0006D7
:10868000A100BD4A5158FF221202114009020843BD
:10869000A100B94A5158FF2212041140090A0843A7
:1086A000A100B54A5158090E0843A1005050A0003E
:1086B000B0490858C00FC0070121C907884203D13B
:1086C0000020A100AB4A5050A000AB490858C00F91
:1086D000C00700E090E20121C907884203D10020D1
:1086E000A100A54A5050A000A249085800280DD06A
:1086F000A00008584B21C900884207D2A0009D491C
:108700000958059808180590701CC6B2A0009A492F
:10871000085800280FD0A00008584B21C9008842F3
:1087200009D200E007E0A00093490958049808180E
:108730000490781CC7B2A0008C49085C0006A10018
:108740008A4A5158FF221202114009020843A1002F
:10875000864A5158FF2212041140090A0843A10019
:10876000824A5158090E0843A1005050FBF7AEF958
:10877000012808D18148F7F7ABFDA1007B4A515889
:108780004018A1005050A00079490858012109065D
:10879000084088427DD1A00074490858C00FC00726
:1087A0000121C907884212D1A00070490858400031
:1087B0004008A1006D4A5050A00011460858C0431F
:1087C000401CA10050500A2017F070FD02E0172055
:1087D00017F06CFDA00065490858002804D0A000DF
:1087E0000858674988420CD9A000604908580121FF
:1087F000C907884209D3A0005C49085861498842EA
:1088000003D84D2017F052FD36E0A0005749085814
:108810005C49884209D9A000544908585A498842FD
:1088200003D8072017F042FD26E0A0004F49085862
:108830005549884211D9A0004C49085853498842EB
:108840000BD8A0004949085840004008012189047C
:10885000081AA100454A50500EE0002C05D14348AB
:10886000C06BA100414A505006E0601E80003F49A5
:108870000858A1003D4A5050A1003C4A50580EF003
:108880007BFB212017F012FD162017F00FFD58205A
:1088900000E00DE017F00AFD0020324948708870B2
:1088A0000870C87000F03AFD012000F037FD15E1B6
:1088B000A0002F4908580121C9060840884238D134
:1088C00028484078102804DB0020A100274A505097
:1088D00013E024484078401C22494870002C05D100
:1088E0002248C06BA100214A505006E0601E800063
:1088F0001E490858A1001D4A5050A1001B4A50585B
:108900000EF03AFB022017F0D1FC172017F0CEFC36
:108910004D2017F0CBFC002012490870C8702120B0
:1089200017F0C4FC002000F0F9FC012000F0F6FC78
:10893000D4E0A0000E4908580121490608408842A9
:1089400058D108488078102822DB0020A100074A6F
:10895000505031E02103002018030020E0030020E4
:108960005803002059030020B2030020EC16002019
:108970002C170020DC190020FC190020B21900205F
:108980003333030007010080CCCC0080000004805A
:10899000C2488078401CC1498870002C05D1C0486D
:1089A000C06BA100BE4A505006E0601E8000BC496A
:1089B0000858A100BA4A5050A100B94A50580EF0C8
:1089C000DBFA082017F072FC212017F06FFC022060
:1089D00017F06CFC172017F069FC4D2017F066FCAF
:1089E0000020AE490870C87000F098FC012000F02B
:1089F00095FC73E0A000AB490858012189060840A6
:108A000088421DD1A5480078401CA449087008463A
:108A1000007803280EDC002C05D1A148C06BA10012
:108A20009F4A505006E0601E80009D490858A100F2
:108A30009B4A5050A1009A4A50580EF09DFA4DE0C2
:108A4000A00098490858012149070840884204D0ED
:108A5000A00094490858002829D1032017F026FCCB
:108A60008E48C078401C8D49C870002C05D18C48B8
:108A7000C06BA1008A4A505006E0601E8000884901
:108A80000858A100864A50508448C078102808DB56
:108A900000208249C870FDF7F5F9012801D100F0E6
:108AA0006DFCA1007E4A50580EF066FA16E02120B7
:108AB00017F0FCFB002C05D17948C06BA100784A67
:108AC000505006E0601E800075490858A100744AA5
:108AD0005050A100724A50580EF04EFAA000714951
:108AE0000858012109070840884247D1092017F09A
:108AF000DDFB0898401CC0B208900898102809D1E6
:108B0000002405E00120A100654A5050601CC4B259
:108B1000102CF7DB002C15D16148C06B0121C9076F
:108B200088420AD85E48C06B5F49884205D35C48DA
:108B3000C06BA1005A4A505023E00120A100584ABE
:108B400050501EE0601E8000554908580121C90799
:108B500088420ED8601E8000514908585249884208
:108B600007D3601E80004E490858A1004C4A50505F
:108B700007E00120A1004A4A505002E0632017F0AC
:108B800095FB601CC4B2102C00DA3EE5002F08D023
:108B900039460498F7F7BCFA44490190F7F7B0FB5F
:108BA00003E042490020F7F7ABFB002E09D0314625
:108BB0000598F7F7ADFA3D490C390190F7F7A0FB9E
:108BC00004E03A490C390020F7F79AFBFEF796FDCE
:108BD00036480C38F7F77CFB35490190F7F790FBE6
:108BE0003248F7F775FB32490C310190F7F788FBF3
:108BF0000020304908704BE02F48006802210840EF
:108C0000022845D125480079401C2449087100F00C
:108C100093FB00F071FB05462048007905280BDB2B
:108C200005201E49087140211D48F7F72AFB402105
:108C30001C48F7F726FB19E0002410E0002C05D1B2
:108C40001748C06BA100164A505006E0601E800015
:108C500013490858A100124A5050601CC4B2102C8D
:108C6000ECDBA1000E4A50580EF086F9E807C00F61
:108C7000002803D0012017F019FB06E0022028404D
:108C8000022802D1012017F011FB002009490870C9
:108C900000E000BF00BF09B0F0BD00005903002094
:108CA000EC1600202C170020666600000819002032
:108CB000B4180020210300201803002010B5344808
:108CC0000078002802D001285FD14CE00120FDF798
:108CD0009FFE012846D1FDF7ADFE002405E00020EF
:108CE000A1002C4A5050601CC4B2102CF7DB2A4A59
:108CF00000200146F7F70DFB28490020F7F700FB9D
:108D00002649091D0020F7F7FBFA25490020F7F74F
:108D1000F7FA2349091D0020F7F7F2FA214900204C
:108D2000F7F7EEFA00202049086020490860204942
:108D300008602049086000F043F8FBF777FE002840
:108D40000DD01D4B1622FF2101311C48FCF7CAF83B
:108D500000200F490870FF2017F0A8FA02E0012058
:108D60000B49087012E0FBF761FE00280CD0124B93
:108D70001622FF2101311148FCF7B4F80020044904
:108D80000870FF2017F092FA00E000BF00BF10BD8E
:108D900099030020EC16002085030020A018002075
:108DA000E818002066030020007F0020047F0020D8
:108DB000087F00200C7F0020E10300209419002090
:108DC00010B577201D490870882048701C480CF0A9
:108DD00001FF1B48007819498870194841781748E5
:108DE000C1701748817815480171154801791348F9
:108DF00041711448F7F76CFA04461049891DF7F7DA
:108E00007FFA1048001DF7F763FA04460B490A3150
:108E1000F7F776FA0B482830F7F75AFA044607496D
:108E20000E31F7F76DFA07482C30F7F751FA044680
:108E300002491231F7F764FA10BD000094190020BE
:108E4000C3030020A0180020F8B5B2480078030042
:108E500012F035F9090627F9F3F2F1F0EFEEF2001E
:108E6000FBF7E4FD00281BD000240DE0A000AA4A77
:108E700081180020F7F744FAA000A84A81180020C2
:108E8000F7F73EFA601CC4B2122CEFDBA44B16229B
:108E9000A449FF200130FBF7DFFF01209D49087046
:108EA00035E19F480078FBF7B3FD01287ED1FBF741
:108EB000BDFD0128FAD19B480078772877D19948E1
:108EC00040788828FAD1984800689849884229D182
:108ED000042197480CF05EFA012806D19148801DC4
:108EE000F7F7F6F99249086005E08E49891D904828
:108EF0000068F7F705FA04218E480CF04BFA0128B8
:108F000006D188480A30F7F7E3F98A49086005E096
:108F100084490A3187480068F7F7F2F905207D494E
:108F2000087002E007207B4908707E480E30F7F792
:108F3000CFF905468121C905F7F740FD1BD37948D4
:108F40001230F7F7C5F905468121C905F7F736FD57
:108F500011D374480E30F7F7BBF905467649F7F799
:108F600023FD08D36F481230F7F7B2F9054672496E
:108F7000F7F71AFD0CD26B490E310020F7F7C0F954
:108F8000684912310020F7F7BBF9052061490870E4
:108F90006448801DF7F79CF905465F49091DF7F7FE
:108FA000AFF960480A30F7F793F901E04AE02AE0A8
:108FB000054659490831F7F7A3F95A48801DF7F7D4
:108FC00087F905465D49F7F79BF956480E30F7F7E4
:108FD0007FF9054650492C31F7F792F95148123084
:108FE000F7F776F905464C493031F7F789F94A48E1
:108FF000001DF7F76DF90746F7F77EFC0546504A66
:10900000F7F787F91EE04D490020F7F779F9FBF7EC
:109010000DFD002813D0FFF7D3FE414B1622FF2190
:1090200001314048FBF75EFF03203A49087009E030
:1090300056E040E036E025E068E015E003E002207D
:109040003449087063E0FBF7F1FC00280BD0FFF710
:10905000B7FE334B1622FF2101313248FBF742FFA6
:1090600003202C49087052E02D480078FBF7D0FC13
:10907000012806D1FBF7DAFC012802D10720254997
:10908000087044E0FBF7D2FC00280AD0244B1022E1
:10909000FF2107312348801DFBF724FF03201D49D2
:1090A000087034E01520FDF7BDFC2649086001205A
:1090B000254908702BE01A480078FBF7A9FC012825
:1090C0000DD1FBF7B3FC012809D1154B0C221F4928
:1090D000FF205130FBF7C0FE08200E49087016E053
:1090E0000F480078FBF794FC01280ED1FBF79EFC9B
:1090F00001280AD1FAF7EAFC002803D11349083104
:10910000F7F7FEF806200349087000E000BF00BF33
:10911000F8BD0000AD0300209C180020E4180020DA
:10912000CA03002094190020147F00206D5C4B3A84
:10913000007F0020047F0020000080C01D0300206D
:109140008503002078030020AE030020AA19002028
:1091500070B555480078002804D001280BD00628A7
:109160007AD17AE0E121090103200CF0A9FE012067
:109170004D49087095E003200CF0EAFC002814D05B
:109180000BF020FB012810D00320FDF741FC012843
:109190000BD046480078002807D1FAF791FC012847
:1091A00003D011F0FBFD012855D1FBF73FFC00284F
:1091B00051D003200CF0CCFC00282ED13C48F7F70E
:1091C00087F805463B48F7F783F806462946F7F740
:1091D00000F904467F21C9052046F7F7EFFB04D3C9
:1091E00035492046F7F7E0FB13D23248F7F770F81D
:1091F00005462F49F7F784F8FFF7E2FD2F4B1622BB
:10920000FF2101312E48FBF76DFE0620264908702C
:1092100021E00020244908701DE0FAF751FC0128E4
:109220000AD1002027490870274B0422FF21593119
:109230002648FBF757FE0EE000201C490870FFF798
:10924000BFFD1E4B1622FF2101311D48FBF74AFED0
:1092500006201549087024E022E0FBF7E7FB002810
:109260001DD0FF2017F022F80320FDF7D1FB0128C5
:1092700005D10320FDF7DEFB0120154908700BF036
:10928000A1FA012803D011F089FD012804D10120A1
:1092900008F0D6F911F05EFF00200349087000E0E5
:1092A00000BF00BF70BD0000AC0300209803002089
:1092B00054030020A0180020000080BFE20300201B
:1092C00094190020B003002084030020B21900206C
:1092D000AF03002010B5074800780A2807DA0548D0
:1092E0000078401C0349087000F048F801E003F0E2
:1092F00057FD10BDB2030020014800787047000000
:109300008A0200200148007870470000890200208E
:1093100001480078704700008C020020072800DD1B
:10932000704701218140034A12788A4301490A703B
:1093300000BFF5E78A020020042001490870704749
:109340008902002000200149087070478C0200202B
:109350000549C978C900054A8A180349C9784910DE
:1093600089005118016070479A00002030130020D6
:1093700001490160704700003013002010B5FEF76E
:109380003FF8FEF7AFF800200F4908600F4908606A
:109390000F4908700F4908700F4908700F4908708D
:1093A0000F4908700F4908700F4908700F4908707D
:1093B0000F4908600F4908600F4908600FF084F8F2
:1093C0000B49086010BD00007C02002080020020D4
:1093D00084020020850200208602002087020020EF
:1093E000880200208D0200208B0200208C020020C9
:1093F000980200209002002094020020F8B5044654
:10940000002C0AD005200004844202D3174884426D
:1094100003D9062016F04AFF02E0422016F046FF6C
:10942000002C07D003200004844203D2042016F04D
:109430003DFF02E02C2016F039FF0EF069FE0746D2
:109440000B493846F7F7BAFA08D33846F7F754FA13
:1094500005460022074BF7F763FA03D2052016F002
:1094600025FF02E0372016F021FFF8BD0000730C45
:1094700000005C420000E0BFF0B589B00025002785
:1094800000261720FDF7CEFAFE490860084600685E
:1094900003F02FFAFC490860084601680020F6F73F
:1094A00098FFFA49086000242DE0A000F849085808
:1094B0000121C90788421CD3A000F5490858400083
:1094C0004008A100F24A5050A100505803F011FA90
:1094D00000210790F6F781FFA100EE4A5050A0004E
:1094E000EB4908580121C9070843A100E84A505038
:1094F00007E0A100E64A505803F0FBF9A100E54A55
:109500005050601CC4B2102CCFDB05F005F90A28BE
:1095100073D10020E04908701021DE48FBF7C2FE3D
:109520000646DE48066000213046F7F73DFA08D2CD
:109530000A20DB49087031460020F6F74AFF06464C
:1095400002E00120D64908703046FDF7A5F90890E1
:10955000089800F0B3FA07463846FDF79DF9D1495F
:109560000690F6F7CDFECF48F6F7B2FECE4906904C
:10957000F6F7C6FECB48F6F7ABFE0690FFF73EFFC8
:10958000CA48407901280BD1C9480078401CC84915
:10959000087008460078F02805DB0020087002E01B
:1095A0000020C3490870C048F6F792FE002805D095
:1095B000162016F07BFE582016F078FE384608F08C
:1095C00073F80746384601F0FDFB39460020F7F7EF
:1095D000EBF97DD0B748007800280FD1B648006875
:1095E000F7F717F9432109060590F6F737FF3946D3
:1095F0000690F6F7F6FE054612E08EE1AF493846D2
:10960000F6F7EFFE0746AC480068F7F702F939466F
:109610000590F6F7E6FEAA490690F6F71FFF054605
:10962000A8492846F6F7DDFEA7490690F6F716FF8B
:109630000546A6492846F6F711FF054698480078E2
:10964000012813D1A248F6F74DFE03910290284657
:10965000F7F752F901910090039B029AF6F73CFF4D
:109660009B4A05910490F6F754FEE0E01620FDF7C2
:10967000D9F9984988423BD19548F6F733FE0591D0
:1096800004902846F7F738F903910290059B049A55
:10969000F7F75AF905D88E4A00200146F6F739FE49
:1096A00012E08B48F6F71EFE039102902846F7F76A
:1096B00023F901910090039B029AF6F7B7FF844AC1
:1096C00005910490F6F725FE8148F6F70BFE00E0C1
:1096D000A7E005910490F7F74BF973490839069014
:1096E000F6F70EFE70480838F6F7F2FD7A49086082
:1096F0006D48001FF6F7ECFD78490690F7F75EF924
:1097000021D2294676480068F6F712FE74490860AF
:109710006C4973480068F7F751F97BD26949704882
:109720000068F6F756FE6E4908605F48001FF6F7BE
:10973000CFFD64490590F6F7FBFD5B49091F0690D4
:10974000F6F7DEFD66E05848001FF6F7C1FD6549F3
:109750000690F7F733F921D2294661480068F6F7F9
:10976000E7FD5F49086060495D480068F7F726F942
:1097700050D25D495A480068F6F72BFE58490860F8
:109780004948001FF6F7A4FD57490590F6F7D0FDAC
:109790004549091F0690F6F7B3FD3BE04248001F1C
:1097A000F6F796FD4649A0390690F7F707F924D257
:1097B00029464B480068F6F7BBFD494908607F2100
:1097C000C90547480068F7F7F9F823D27F21C90592
:1097D00043480068F6F7FDFD414908603248001F24
:1097E000F6F776FD7F21C9050590F6F7A1FD2E4914
:1097F000091F0690F6F784FD0CE02B48001FF6F7D2
:1098000067FD29460590F6F793FD2749091F069045
:10981000F6F776FD2448001FF6F75AFD3349086035
:1098200005E02148001FF6F753FD304908603A462D
:109830001B480178284611F0E9FA079001218907B1
:109840000798F7F7BBF805D3032189070798F7F7BF
:10985000ABF801D2002007901D48F6F743FD0391B5
:1098600002900798F7F748F801910090039B029A3D
:10987000F6F732FE164A05910490F6F74AFD1448B1
:1098800036E000004003002044030020480300208D
:10989000EC16002054190020580300209C030020DF
:1098A0008D030020F0180020A81800204019002087
:1098B000B3030020A8030020BC030020643B7F3FCB
:1098C000002474490000C8420000614500007A4449
:1098D000850300203C4D0000007F0020A3BBBE4C50
:1098E000900300207696184B00002041047F002052
:1098F000F6F7F8FC05910490F7F73AF85C49069002
:10990000F6F7FEFC5A48F6F7E3FC5A4908605A4855
:1099100005605A485A490860A7E05A48007801286B
:1099200004D100205749087017F034FF1021564821
:10993000FBF7B8FC06465548066000213046F7F7AD
:1099400033F800D200263046FCF7A6FF08900898AE
:1099500000F0B4F807463846FCF79EFF4C49086013
:109960004C48407901280BD14B480078401C4A49AB
:109970000870084600780F2805DB0020087002E018
:10998000002045490870384607F08EFE07463846E5
:10999000FAF75AFE384601F015FA39460020F7F773
:1099A00003F851D0162016F081FC582016F07EFCEA
:1099B0003A480068F6F72DFF432109060590F6F7AF
:1099C0004DFD39460690F6F70CFD35490790F6F740
:1099D00045FD05463348F6F77BFC29460690F6F729
:1099E000A7FC30490790F6F78BFC2F48F6F77AFC76
:1099F000059104902D492846F6F730FD0190F6F7C1
:109A00007BFF03910290059B049AF6F765FD264AB9
:109A100007910690F6F77DFC2348F6F763FC059165
:109A20000490F6F7A5FF12490790F6F769FC1D4868
:109A3000F6F74EFC1E4908601E4805600C48F6F714
:109A400047FC0C4908600DE00948F6F741FC09495C
:109A500008600748001DF6F73BFC17490860002026
:109A60001449086005480649086009B0F0BD0000C7
:109A7000A0180020007F0020187F00206D5C4B3A6A
:109A8000147F00202D030020541900209C03002087
:109A90002403002040190020B3030020BC03002051
:109AA00000001042E81800208503002000007A44DE
:109AB000087F00200C7F0020047F002001B59CB0AF
:109AC00000201B901A90199005200CF037F8002800
:109AD00011D005200CF062F8FD480068FD4988426D
:109AE00003D90120FC49087002E00020FA490870FF
:109AF0000020F7490860F9491C980968884204D396
:109B0000012189041C98884202D300201B90F6E3AF
:109B1000EF480068401CEE4908601C9802F0E9FE1E
:109B20001A90EF491A98F6F75CFC1A90F9F7CEFFF5
:109B300001281AD1EB480068401CEA49086004205B
:109B40000BF0FCFF002813D004200CF027F8E548A8
:109B50000068E049884204D902F0D6FE0120E249BB
:109B600008700020DF49086002E00020DD4908603D
:109B7000DE480078002803D0DD480068199002E034
:109B80000EF0C6FA19901998F6F7B6FE0022D94BD6
:109B900017911690F6F7C4FE0CD2D748F6F798FB4B
:109BA0005F2807D9D4480C30F6F792FB5F2801D91B
:109BB000D24819900BF0A0FCD1490860D1481A99FD
:109BC000F6F70FFC15901A99F6F70BFC1790CE4894
:109BD0001999F6F706FC13901A99F6F702FC1590FE
:109BE000CA481999F6F7FDFB11901999F6F7F9FB98
:109BF0001390C7481A99F6F7F4FB1190C5481999C4
:109C0000F6F7EFFBC4490F90F6F792FB109011990D
:109C1000F6F78EFB12901399F6F7DBFB149015996B
:109C2000F6F786FB16901799F6F782FB1890BB495A
:109C30001898F6F7B9FE7DD800211998F6F7B4FE0A
:109C400004D3B7491998F6F7B9FE03D2B548006DA9
:109C5000179029E01998F6F705FEC0B215901598EF
:109C6000F6F7D7FD0D901999F6F7B7FB14901598F4
:109C70008000AC4908580B901598401C8100A948F9
:109C800040580A900B99F6F7A4FB0C901499F6F73C
:109C9000A8FB0D9015988000A249085801460C9029
:109CA0000D98F6F745FB179017990846F6F799FBBC
:109CB0000C901A99F6F795FB9B490D90F6F791FBDE
:109CC00013901998129000211998F6F76DFE02D2A0
:109CD0000020129006E095491998F6F76FFE01D220
:109CE0009248129092481299F6F77BFB0C9091489B
:109CF0001299F6F776FB08901299F6F772FB0A9024
:109D00008D481299F6F76DFB07901299F6F769FBEB
:109D100008901299F6F765FB09900A99F6F708FB87
:109D20000B900C99F6F755FB84490D90F6F700FB64
:109D3000119000E0ECE182481299F6F752FB0B908B
:109D400080481299F6F74DFB09901299F6F749FBF6
:109D50000A900B99F6F7ECFA7B490C90F6F7E8FAC3
:109D60007A490D90F6F73DFB109078481099F6F778
:109D700038FB0B901399F6F734FB75490C90F6F706
:109D800030FB0D901199F6F769FB0F90714913980C
:109D9000F6F727FB1B906D490F98F6F75FFB0E90C7
:109DA0006D490E98F6F700FE55D26C480E99F6F7FD
:109DB00018FB0C906A480E99F6F713FB08900E9961
:109DC000F6F70FFB0A9067480E99F6F70AFB059025
:109DD0000E99F6F706FB06900E99F6F702FB08902F
:109DE00061480E99F6F7FDFA02900E99F6F7F9FA26
:109DF00003900E99F6F7F5FA04900E99F6F7F1FA3A
:109E000006905A480E99F6F7ECFA01900E99F6F77B
:109E1000E8FA02900E99F6F7E4FA03900E99F6F735
:109E2000E0FA04900E99F6F7DCFA05900699F6F739
:109E3000D0FA07900899F6F77BFA09900A99F6F795
:109E4000C8FA0B900C99F6F773FA49490D90F6F79A
:109E50006FFA169051E147490E98F6F7A5FD36D2F4
:109E600045480E99F6F7BDFA0C9044480E99F6F75E
:109E7000B8FA08900E99F6F7B4FA0A9040480E998D
:109E8000F6F7AFFA05900E99F6F7ABFA06900E9931
:109E9000F6F7A7FA08903B480E99F6F7A2FA029057
:109EA0000E99F6F79EFA03900E99F6F79AFA049037
:109EB0000E99F6F796FA069033480E99F6F791FA4E
:109EC00001900E99F6F78DFA02900E995EE07DE012
:109ED000D8030020B8A10000B103002040030020F7
:109EE00000007A43D4030020B00300203A0300208E
:109EF0003C0300200000E0BFB41800200000A04197
:109F0000B40300209296CA3C68791E3DD141973B2C
:109F10002506A1404CA64A3E2DB245C0000066432E
:109F20000000C842DC2702001E8C0A3200005C429E
:109F300023DB5C421A516A3FA69BC4BB6606DF4422
:109F40003B4A5B372684B3B64703803F00007A4420
:109F500000003841E8F6BA43CDCCAC404B75013D2A
:109F600061E28F3C1A53B03B3EF4553AE93A493826
:109F7000C009653F00004842643B043B5762D83843
:109F8000451E4D3632CE46330689982FF6F729FA0C
:109F900003900E99F6F725FA04900E99F6F721FA38
:109FA00005900699F6F715FA07900899F6F7C0F9A3
:109FB00009900A99F6F70DFA0B900C99F6F7B8F993
:109FC000FE490D90F6F7B4F9169096E0FC490E980C
:109FD000F6F7EAFC55D2FB480E99F6F702FA0C9018
:109FE000F9480E99F6F7FDF908900E99F6F7F9F988
:109FF0000A90F6480E99F6F7F4F905900E99F6F7DF
:10A00000F0F906900E99F6F7ECF90890F0480E99E1
:10A01000F6F7E7F902900E99F6F7E3F903900E9937
:10A02000F6F7DFF904900E99F6F7DBF90690E948A8
:10A030000E99F6F7D6F901900E99F6F7D2F902903B
:10A040000E99F6F7CEF903900E99F6F7CAF9049037
:10A050000E99F6F7C6F905900699F6F7BAF9079042
:10A060000899F6F765F909900A99F6F7B2F90B9095
:10A070000C99F6F75DF9D8490D90F6F759F9169055
:10A080003BE0D6480E99F6F7ACF90C90D4480E99FF
:10A09000F6F7A7F908900E99F6F7A3F90A90D148B8
:10A0A0000E99F6F79EF905900E99F6F79AF9069033
:10A0B0000E99F6F796F90890CB480E99F6F791F9B4
:10A0C00004900E99F6F78DF905900E99F6F789F937
:10A0D00006900E99F6F785F907900899F6F728F992
:10A0E00009900A99F6F775F90B900C99F6F720F993
:10A0F000BE490D90F6F71CF9169016991B98F6F7C5
:10A1000070F91B9019A807C8FAF7E0FF1B90EEE35F
:10A11000B7491998F6F752FC7ED2B6491898F6F767
:10A1200043FC7AD2B4480068014613901A98F6F7B7
:10A13000FFF81590B0480068014611901A98F6F79C
:10A14000F7F81390AC480068014610901A98F6F79B
:10A15000EFF81190A848806A014610901198F6F720
:10A1600040F912901399F6F73CF914901599F6F707
:10A1700038F91790A0480068014610901A98F6F731
:10A18000D7F812909C48006801460F901A98F6F78D
:10A19000CFF810909848406A01460F901098F6F753
:10A1A00020F911901299F6F71CF913901999F6F706
:10A1B00018F915909048006801460E901A98F6F725
:10A1C000B7F80F908C48006A01460E900F98F6F78A
:10A1D00008F910901999F6F704F911901999F6F702
:10A1E00000F913908448C0690D901999F6F7F9F8B1
:10A1F0000E901999F6F7F5F80F901999F6F7F1F80E
:10A2000011907D48006801460B901A98F6F790F877
:10A210000D907948006801E07DE171E001460A9007
:10A220001A98F6F785F80B907348806901460A90F2
:10A230000B98F6F7D6F80C900D99F6F7D2F80F9028
:10A240006D480068014609901A98F6F771F80A906F
:10A2500069484069014609900A98F6F7C2F80B90E0
:10A260001999F6F7BEF80D9063480069089019999E
:10A27000F6F7B7F809901999F6F7B3F80B905E481E
:10A280000068014606901A98F6F752F807905A4867
:10A29000C068014606900798F6F7A3F8099056485B
:10A2A000806806901999F6F79CF807905248406824
:10A2B000014606900798F6F73BF808900999F6F7DB
:10A2C00037F80A900B99F6F733F80C900D99F6F7DA
:10A2D0002FF80E900F99F6F72BF810901199F6F7CA
:10A2E00027F812901399F6F723F814901599F6F7BA
:10A2F0001FF816901799F6F71BF81B90F7E2FDE38D
:10A300003D48C06A014613901A98F6F711F8159067
:10A310003948C06A014611901A98F6F709F8139067
:10A320003548C06A014610901A98F6F701F8119066
:10A330003148406D014610901198F6F752F812908E
:10A340001399F6F74EF814901599F6F74AF8179006
:10A350002948C06A014610901A98F5F7E9FF129053
:10A360002548C06A01460F901A98F5F7E1FF109052
:10A370002148006D01460F901098F6F732F81190C1
:10A380001299F6F72EF813901999F6F72AF8159006
:10A390001948C06A01460E901A98F5F7C9FF0F9048
:10A3A0001548C06C01460E900F98F6F71AF81090F9
:10A3B0001999F6F716F8119019991FE070256B3F5F
:10A3C0000000C843CB694B39C66FA7350D4FA0318C
:10A3D00068681D2DF82DF527CB106F3F574FED37CF
:10A3E000D96F1233D9FBC82D6F73E1A74AA1713F12
:10A3F00000000C4200008C4304070020F5F7F1FF39
:10A400001390FE48806C0D901999F5F7EAFF0E90B5
:10A410001999F5F7E6FF0F901999F5F7E2FF1190FA
:10A42000F648C06A01460B901A98F5F781FF0D9027
:10A43000F248C06A01460A901A98F5F779FF0B9026
:10A44000EE48406C01460A900B98F5F7CAFF0C9055
:10A450000D99F5F7C6FF0F90E848C06A01460990CC
:10A460001A98F5F765FF0A90E448006C01460990D8
:10A470000A98F5F7B6FF0B901999F5F7B2FF0D9012
:10A48000DE48C06B08901999F5F7ABFF0990199950
:10A49000F5F7A7FF0B90D948C06A014606901A98B5
:10A4A000F5F746FF0790D548806B01460690079860
:10A4B000F5F797FF0990D148406B06901999F5F789
:10A4C00090FF0790CD48006B014606900798F5F77E
:10A4D0002FFF08900999F5F72BFF0A900B99F5F7D4
:10A4E00027FF0C900D99F5F723FF0E900F99F5F7C4
:10A4F0001FFF10901199F5F71BFF12901399F5F7B4
:10A5000017FF14901599F5F713FF16901799F5F7A3
:10A510000FFF1B90EBE1BA491898F6F745FA7DD288
:10A52000B648806D014613901A98F5F701FF159013
:10A53000B248806D014611901A98F5F7F9FE139014
:10A54000AE48806D014610901A98F5F7F1FE119013
:10A55000AA4880300068014610901198F5F741FF35
:10A5600012901399F5F73DFF14901599F5F739FFFF
:10A570001790A248806D014610901A98F5F7D8FE02
:10A5800012909E48806D01460F901A98F5F7D0FE04
:10A5900010909A48C06F01460F901098F5F721FF70
:10A5A00011901299F5F71DFF13901999F5F719FFFE
:10A5B00015909248806D01460E901A98F5F7B8FEF6
:10A5C0000F908E48806F01460E900F98F5F709FFA7
:10A5D00010901999F5F705FF11901999F5F701FFFA
:10A5E00013908648406F0D901999F5F7FAFE0E907A
:10A5F0001999F5F7F6FE0F901999F5F7F2FE1190FB
:10A600007E48806D01460B901A98F5F791FE0D90EB
:10A610007A48806D01460A901A9800E06DE0F5F7DF
:10A6200087FE0B907548006F01460A900B98F5F76E
:10A63000D8FE0C900D99F5F7D4FE0F906F48806D01
:10A64000014609901A98F5F773FE0A906B48C06EA0
:10A65000014609900A98F5F7C4FE0B901999F5F791
:10A66000C0FE0D906548806E08901999F5F7B9FE07
:10A6700009901999F5F7B5FE0B906048806D014679
:10A6800006901A98F5F754FE07905C48406E014614
:10A6900006900798F5F7A5FE09905848006E0690B9
:10A6A0001999F5F79EFE07905448C06D0146069033
:10A6B0000798F5F73DFE08900999F5F739FE0A90DD
:10A6C0000B99F5F735FE0C900D99F5F731FE0E90CC
:10A6D0000F99F5F72DFE10901199F5F729FE1290BC
:10A6E0001399F5F725FE14901599F5F721FE1690AC
:10A6F0001799F5F71DFE1B90F9E04048803040683F
:10A70000014613901A98F5F713FE15903B488030D8
:10A710004068014611901A98F5F70AFE13903748E1
:10A7200080304068014610901A98F5F701FE1190AC
:10A7300032488030C06A014610901198F5F751FEFA
:10A7400012901399F5F74DFE14901599F5F749FEFF
:10A7500017902A4880304068014610901A98F5F703
:10A76000E7FD129025488030406801460F901A9806
:10A77000F5F7DEFD109021488030806A01460F9089
:10A780001098F5F72EFE11901299F5F72AFE139006
:10A790001999F5F726FE1590184880304068014653
:10A7A0000E901A98F5F7C4FD0F9014488030406A57
:10A7B00001460E900F98F5F714FE10901999F5F7D1
:10A7C00010FE11901999F5F70CFE13900B4880308C
:10A7D000006A0D901999F5F704FE0E901999F5F796
:10A7E00000FE0F901999F5F7FCFD11900348803099
:10A7F000406801460B901A9804E00000040700200E
:10A8000000008C43F5F794FD0D90FB48406801462D
:10A810000A901A98F5F78CFD0B90F748C06901462D
:10A820000A900B98F5F7DDFD0C900D99F5F7D9FD21
:10A830000F90F1484068014609901A98F5F778FDA5
:10A840000A90ED488069014609900A98F5F7C9FD1C
:10A850000B901999F5F7C5FD0D90E74840690890F0
:10A860001999F5F7BEFD09901999F5F7BAFD0B9006
:10A87000E1484068014606901A98F5F759FD07909F
:10A88000DD480069014606900798F5F7AAFD099092
:10A89000D948C06806901999F5F7A3FD0790D648E6
:10A8A0008068014606900798F5F742FD08900999DF
:10A8B000F5F73EFD0A900B99F5F73AFD0C900D99CE
:10A8C000F5F736FD0E900F99F5F732FD10901199BE
:10A8D000F5F72EFD12901399F5F72AFD14901599AE
:10A8E000F5F726FD16901799F5F722FD1B90C34941
:10A8F0001898F6F759F818D8C14800688830F5F765
:10A90000E7FC1690BE4800689030F5F7E1FC149023
:10A910001B99F5F766FD15901699F5F709FD179047
:10A920001B99F5F75EFD1B9053E0B6491898F6F7B2
:10A930003BF818D8B24800685C30F5F7C9FC1690AF
:10A94000AF4800686430F5F7C3FC14901B99F5F725
:10A9500048FD15901699F5F7EBFC17901B99F5F744
:10A9600040FD1B9035E0A8491898F6F71DF818D857
:10A97000A34800683030F5F7ABFC1690A04800689B
:10A980003830F5F7A5FC14901B99F5F72AFD1590C2
:10A990001699F5F7CDFC17901B99F5F722FD1B9042
:10A9A00017E097480068001DF5F792FC1690944850
:10A9B00000680C30F5F78CFC14901B99F5F711FD2D
:10A9C00015901699F5F7B4FC17901B99F5F709FD4A
:10A9D0001B908E491998F5F7E7FF07D200201999C7
:10A9E000F5F7E2FF02D000201DB000BDF9F76EF8C8
:10A9F000012806D186491B98F5F7D6FF01D800201B
:10AA0000F2E78448F5F764FC1590F5F71DFF002286
:10AA1000814B17911690F5F783FF0DD37D480C30CD
:10AA2000F5F756FC1590F5F70FFF00227A4B1791BA
:10AA30001690F5F775FF07D2412109061B98F5F727
:10AA4000B3FF01D80020CFE700211B98F5F7ACFF3A
:10AA500001D200201B9071491B98F5F7AFFF09D870
:10AA60006F491B98F5F7A0FF04D26E491B98F5F7C4
:10AA7000B8FC1B906C491B98F5F796FF0AD26B49FE
:10AA80001998F5F79BFF04D869491B98F5F7A9FCBD
:10AA90001B906EE164491B98F5F790FF31D865492A
:10AAA0001B98F5F781FF2CD260491998F5F786FFBE
:10AAB0000DD861481B99F5F794FC60491690F5F79D
:10AAC00037FC17901B99F5F78CFC1B9051E15C4902
:10AAD0001998F5F773FFDCD854491998F5F764FF16
:10AAE000D7D258481999F5F77CFC57491690F5F7D5
:10AAF0001FFC17901B99F5F774FC00E03EE11B90DA
:10AB000037E14C491B98F5F759FF1FD84F491B985F
:10AB1000F5F74AFF1AD24E491998F5F74FFF05D8B5
:10AB200040491B98F5F75DFC1B9022E149491998B3
:10AB3000F5F744FFADD848491998F5F735FFA8D285
:10AB400046491B98F5F74DFC1B9012E13C491B98B8
:10AB5000F5F734FF10D8212149061B98F5F724FF9B
:10AB60000AD237491998F5F729FF92D83B491B9823
:10AB7000F5F737FC1B90FCE039491B98F5F71EFFF1
:10AB80000FD838491B98F5F70FFF0AD235491998A5
:10AB9000F5F714FF04D834491B98F5F722FC1B90F5
:10ABA000E7E030491B98F5F709FF65D82F491B9856
:10ABB000F5F7FAFE60D219491998F5F7FFFE05D8A6
:10ABC0002B491B98F5F70DFC1B90D2E025491998ED
:10ABD000F5F7F4FE05D827491B98F5F702FC1B9002
:10ABE000C7E017491998F5F7E9FE04D81E491B98E4
:10ABF000F5F7F7FB1B90BCE08407002000007041D4
:10AC0000B403002000002C4200006643CDCCCC3DB4
:10AC100000001041B41800200000634000003442DE
:10AC2000000002434E62803F0000E0400000F0411F
:10AC300052B87E3F00000841D044583B55C1783F90
:10AC40000000C8416F1283BA3333833F0000904144
:10AC500000003C420000E04100002842643B7F3F8E
:10AC600000000442000018428941803F00005C421D
:10AC700060E5803F1283803F45491B98F5F79EFEB3
:10AC800024D844491B98F5F78FFE1FD242491998E2
:10AC9000F5F794FE0AD841491998F5F785FE05D2D3
:10ACA0003F491B98F5F79DFB1B9062E03D491998C1
:10ACB000F5F784FE5DD838491998F5F775FE58D236
:10ACC00039491B98F5F78DFB1B9052E031491B98D1
:10ACD000F5F774FE24D835491B98F5F765FE1FD2A9
:10ACE0002D491998F5F76AFE0AD82C491998F5F7F5
:10ACF0005BFE05D22A491B98F5F773FB1B9038E0E1
:10AD00002B491998F5F75AFE33D823491998F5F7C6
:10AD10004BFE2ED224491B98F5F763FB1B9028E0CD
:10AD200022491B98F5F74AFE14D822491B98F5F7DB
:10AD30003BFE0FD21E491998F5F740FE19D8164967
:10AD40001998F5F731FE14D217491B98F5F749FB0E
:10AD50001B900EE017491B98F5F730FE09D81649ED
:10AD60001998F5F721FE04D214491B98F5F739FB21
:10AD70001B901B9815F0D8FF1B9000BF10491B9823
:10AD8000F5F71CFE01D20E481B901B982CE6000024
:10AD900000000C4300008C43A4700B4200001842DA
:10ADA000DBF97E3F0000E041643B7F3F0000C84389
:10ADB0000000C84100009644B81E51418941803FBF
:10ADC00000409245F0B585B004460027002003906E
:10ADD00002900190FBF756F8002802D10120974914
:10ADE000087097480078002806D0012823D0022850
:10ADF0002AD0032871D111E100212046F5F7D4FDB6
:10AE000018D003F089FC0A2805D18E48F5F760FABE
:10AE10008D49086004E08D48F5F75AFA8A490860C0
:10AE200003210C200BF04CF800208449087001200D
:10AE300083490870FFE00C200AF08AFE002802D146
:10AE400002207F490870F6E000212046F5F7ACFDAE
:10AE50007ED103F061FC0A287BD17A48F5F738FAF5
:10AE60000546794801682846F5F7B3FA07463F21B9
:10AE700009063846F5F7ADFA03907F21C905384633
:10AE8000F5F7A7FA029072493846F5F7A2FA019051
:10AE900070490298F5F792FD20D86F490298F5F7AE
:10AEA00083FD1BD86748F5F713FA06466B490298ED
:10AEB000F5F797FA31460090F5F78FFA05466149A4
:10AEC000F5F71EFA5F48F5F703FA0090F5F714FD61
:10AED0000546634AF5F71DFA9AE0A8E06149039830
:10AEE000F5F76CFD1FD860490398F5F75DFD1AD89A
:10AEF0005448F5F7EDF9064658490398F5F771FA05
:10AF000031460090F5F769FA05464E49F5F7F8F92C
:10AF10004C48F5F7DDF90090F5F7EEFC0546504A90
:10AF2000F5F7F7F974E051490198F5F747FD6FD847
:10AF30004F490198F5F738FD6AD840480078012854
:10AF400066D14048F5F7C4F906464A49019801E040
:10AF500063E014E0F5F745FA31460090F5F73DFA65
:10AF600005463849F5F7CCF93648F5F7B1F90090C0
:10AF7000F5F7C2FC05463A4AF5F7CBF948E0334805
:10AF8000F5F7A6F90546304801682846F5F721FA95
:10AF9000074639493846F5F71CFA039037493846D1
:10AFA000F5F717FA029036490298F5F707FD15D81C
:10AFB00034490298F5F7F8FC10D82448F5F788F9D9
:10AFC000064626490298F5F70CFA31460090F5F747
:10AFD00004FA05461D49F5F793F919E02A49039843
:10AFE000F5F7ECFC14D829490398F5F7DDFC0FD8E8
:10AFF0001648F5F76DF9064618490398F5F7F1F983
:10B0000031460090F5F7E9F905461049F5F778F96A
:10B0100000200A4908700A4908700CE00021204607
:10B02000F5F7C2FC02D100200549087003E00020BA
:10B030000349087000BF00BF05B0F0BDD003002079
:10B04000CB030020A0180020CC030020E81800202B
:10B0500000002041295C0FBD295C0F3DCDCC4C3E4A
:10B0600085030020295C8FBC295C8F3CCDCC4CBF74
:10B07000CDCC4C3F9A99593F0000FA4300007A44E6
:10B0800000000CC200000C4200008CC100008C418A
:10B0900003480078012800D170470020FCE7000039
:10B0A0008D02002010B5FCF7ABF9FCF71BFA00206D
:10B0B0001549086015490860154908701549087058
:10B0C0001549087015490870154908701549087028
:10B0D00004201549087000201449087014490870AC
:10B0E000144908701449086014490860144908603C
:10B0F0000DF0EAF9104908601920FBF793FCC1B282
:10B100001048C17010BD00007C02002080020020A9
:10B110008402002085020020860200208702002091
:10B12000880200208D020020890200208A0200206F
:10B130008B0200208C020020980200209002002048
:10B14000940200209A000020F8B500260024FE4852
:10B150000078232801D301F000F843007B449B884A
:10B160005B009F4422005100A100F60012012F0154
:10B170005603D803FA0341045E047E04CB04270679
:10B18000DF060607AF07FA07C407E2074E016A01A8
:10B190008A01DA01FA07DD00E70407055705B7055C
:10B1A0000A06D4021D0375069506E849012000062B
:10B1B000F5F7A6F8E5481C38C078102803DD102103
:10B1C000E2481C38C170E2480078012802D1002012
:10B1D000DF4908700DF078F9DE4908600120DA498E
:10B1E0000870DD4908700020DC490870DC490870EF
:10B1F0000120DC4908600020DB490860DB48DC49AD
:10B200000860FCF747F9C4E34E20FBF701FC002877
:10B210002AD00DF059F9CF490968401AD54988421A
:10B2200041D94E20FBF706FCCC48007801283AD1E2
:10B230000DF04AF9C74908600020C849087002208B
:10B24000C14908700120C44908700220C54908603E
:10B250000420C5490860C848C5490860C748C849AE
:10B260000860FCF717F91EE0BC48007801281AD1E5
:10B270000DF02AF9B74908600020B849087002208B
:10B28000B14908700120B44908700220B54908602E
:10B290000420B5490860B848B5490860B748B849BE
:10B2A0000860FCF7F7F8AEE7AD480078012836D122
:10B2B0000020AB490870B148C078B24948700846D0
:10B2C00040780421084004280AD10020AE490860D3
:10B2D0000DF0FAF89F49086019209B4908701EE09C
:10B2E000A9480068401CA849086008460068FF217A
:10B2F0002D3188420ED90020A34908600220A349BD
:10B300000870A348007801210843A1490870FDF79F
:10B31000E1FF04E00120914908708B49087072E751
:10B3200000208E49087003208749087001208A494F
:10B3300008700DF0C9F8874908600620894908603F
:10B34000002089490860934889490860FCF7A2F801
:10B3500059E782480078012816D100207F490870FB
:10B360000DF0B2F87B49086004207749087001208D
:10B37000794908707B49086000207B49086086484D
:10B380007B490860FCF786F83DE77448007801289F
:10B3900017D10DF099F86F49086000206F490870C7
:10B3A00005206949087001206B49087006206D4925
:10B3B000086000206C49086078486D490860FCF717
:10B3C00069F820E765480078012819D10DF07CF86C
:10B3D0006049086000206149087014205A490870CB
:10B3E00001205D49087006205E49086000205E4922
:10B3F00008606B4908706B485D490860FCF74AF8C3
:10B4000001E756480078012816D1002053490870FA
:10B4100015204D4908700DF057F84E49086001207D
:10B420004D4908704F49086000204F4908605E4848
:10B430004F490860FCF72EF8E5E6484800780128F7
:10B440001AD10DF041F843490860002043490870C3
:10B4500016203D49087001203F49087002204149EB
:10B460000860042040490860434841490860434857
:10B4700043490860FCF70EF8C5E639480078012812
:10B480004AD10020364908703C48C0783D49C87010
:10B490000846C0780821084008281DD100203A49F4
:10B4A00008602E4908700DF00FF82A49086017202F
:10B4B00025490870012028490870022029490860A0
:10B4C0000420294908603948294908602B482C493B
:10B4D0000860FBF7DFFF1FE02B480068401C2A498B
:10B4E000086008460068FF212D3188420ED90020EF
:10B4F0002549086002202549087025480078012167
:10B50000084323490870FDF7E5FE05E001201349D3
:10B51000087015200C49087075E61148007801285C
:10B520007DD100200E4908700C4908700CF0CCFF4A
:10B5300008490860114800781249C8700F484078DF
:10B5400088700E48807833E085020020B600002025
:10B550008B02002098020020860200208802002032
:10B5600087020020800200207C02002024210200AB
:10B570006402002050C30000F62002006C0200208C
:10B58000680200205C000020900200208902002058
:10B590008A020020DE20020025210200E4200200B1
:10B5A00078020020EA200200282102001221020075
:10B5B0004870F848C078087000201AE00146093148
:10B5C0008900F54A525C014609318900F24BC918DD
:10B5D00049785218014609318900C91889785218EA
:10B5E000014609318900C918C97851180C19411C44
:10B5F000C8B21028E2DB2106FF221202224012020A
:10B600001143FF2212042240120A1143220E114359
:10B610000846E249F4F774FE002400201BE075E0C0
:10B6200001464F318900DC4A525C01464F318900A6
:10B63000D94BC9184978521801464F318900C918A9
:10B640008978521801464F318900C918C9785118B4
:10B650000C19411CC8B22E28E2DB2106FF2212027F
:10B66000224012021143FF2212042240120A114307
:10B67000220E11430846C949091DF4F741FE002076
:10B6800004E0C749095C8E19411C88B20D2189016B
:10B690008842F6D33106FF221202324012021143D1
:10B6A000FF2212043240120A1143320E114308469F
:10B6B000BA490831F4F724FEBA48F4F709FEB0425B
:10B6C00010D00620B84908700120B8490870B84960
:10B6D00008600020B7490860B748B8490860FBF720
:10B6E000D9FE13E01F20B04908700120AF4908704F
:10B6F0000220AF4908600420AE490860B048AF4955
:10B700000860A448AF490860FBF7C4FE7BE5AE487B
:10B710000078012843D10020AB490870AB4908707C
:10B720000CF0D2FEAA4908609A4800789D4908703A
:10B730009848407848709748807888709548C078D5
:10B74000C8709648F4F7C4FD05469648F4F7C0FD66
:10B75000854210D007209449087001209349087051
:10B760009349086000209349086093489349086012
:10B77000FBF790FE13E020208B49087001208B49D5
:10B78000087002208A49086004208A4908609148AC
:10B790008A4908607F488B490860FBF77BFE32E5E9
:10B7A00089480078012833D10020874908708749EB
:10B7B00008700CF089FE864908607648007879495F
:10B7C0000870744840784870724880788870714872
:10B7D000C078C8707148001DF4F77AFD05467148BD
:10B7E000F4F776FD854203D007206F49087002E028
:10B7F0001E206D49087001206C4908706C49086072
:10B8000000206C4908606C486C490860FBF742FEF8
:10B81000F9E46E48007801287CD1002500206B49AE
:10B8200008700CF051FE6A4908606B480068401EC1
:10B830006A490978884235D95C20694908706749A6
:10B840000878C10F09184910654A51706349087892
:10B85000C10F091849104900411AC907090E917012
:10B8600000BF09E05D480078C00140194C49095CFF
:10B87000E81C5B4A11546D1C802DF3D301204B4909
:10B88000087083204A49086000204A4908605448EB
:10B890004A490860FBF7FEFD50480078401C4F49BC
:10B8A000087036E05C204E4908704C490878C10F9A
:10B8B000091849104A4A517048490878C10F0918B7
:10B8C00049104900411AC907090E9170002509E085
:10B8D00042480078C00140193149095CE81C404ADF
:10B8E00011546D1C3F4800688542F1D301202F4957
:10B8F00008703C480068C01C2D49086000202D4994
:10B90000086037482D490860FBF7C4FD0720264929
:10B91000087000BF77E42D48007801281CD10CF096
:10B92000D3FD2B49086000202849087008201E49D3
:10B93000087001201D490870FF20FF301C49086075
:10B9400000201C4908600120184908701248801C1A
:10B950001A490860FBF79EFD55E41C480078012851
:10B9600016D10CF0B1FD1A49086000201749087083
:10B9700009200D49087001200C4908700C49086025
:10B9800000200C4908600C480C490860FBF782FD58
:10B99000E4E30EE26C020020620000205602002068
:10B9A000292102005C000020850200208602002080
:10B9B000800200207C020020262102006402002078
:10B9C0001421020068020020870200208802002063
:10B9D0009802002016210200700200207802002048
:10B9E000F013002074020020FE480078012817D1CF
:10B9F0000CF06AFDFC4908600020FA4908700A2032
:10BA0000FA4908700120FA4908700620F9490860CF
:10BA10000020F9490860F948F9490860FBF73AFD48
:10BA20009CE3F048007801281AD10CF04DFDEE4956
:10BA300008600020EB4908700B20EC4908700120D9
:10BA4000EB4908700220EB4908600420EA490860CD
:10BA5000EC48EB490860EC48EC490860FBF71AFD3C
:10BA60007CE3EB480078012847D10020E8490870C2
:10BA7000E548C078E749C8700846C0780221084008
:10BA800002281AD10020E44908600CF01DFDD649B7
:10BA900008600020D34908700C20D44908700120A8
:10BAA000D3490870D34908600020D3490860DB48B7
:10BAB000D3490860FBF7EEFC1FE0D7480068401C44
:10BAC000D549086008460068FF212D3188420ED90B
:10BAD0000020D14908600220D1490870D14800787F
:10BAE00001210843CF490870FDF7F4FB05E0012070
:10BAF000BC4908700A20BD4908702FE3B948007896
:10BB0000012816D10CF0E0FCB74908600020B549C7
:10BB100008701A20B54908700120B5490870B54968
:10BB200008600020B4490860BF48B5490860FBF7C9
:10BB3000B1FC13E3AB48007801281AD10CF0C4FC27
:10BB4000A94908600020A74908701B20A749087070
:10BB50000120A74908700220A64908600420A649D0
:10BB60000860A848A6490860A748A8490860FBF7EC
:10BB700091FCF3E2A648007801284AD10020A449AC
:10BB80000870A148C078A349C8700846C078082149
:10BB9000084008281DD100209F490860914908707D
:10BBA0000CF092FC904908601C209049087001201C
:10BBB0008F49087002208F49086004208E49086070
:10BBC0009A488F490860904890490860FBF762FCEA
:10BBD0001FE091480068401C8F49086008460068D3
:10BBE000FF212D3188420ED900208B4908600220A8
:10BBF0008B4908708B4800780121084389490870F7
:10BC0000FDF768FB05E00120764908701A207749A6
:10BC10000870A3E27E48007801285AD100207C49B0
:10BC20000870704908700CF04FFC6F490860764846
:10BC30000078784908707448407848707248807875
:10BC400088707148C078C8707948F4F741FB0546A0
:10BC50007048F4F73DFB854227D076480068401CC9
:10BC6000744908600846006803280DD90020086060
:10BC700002206B4908706B4800780121084369492C
:10BC80000870FDF727FB24E00720584908700120C1
:10BC900057490870574908600020574908605F48B5
:10BCA00057490860FBF7F6FB13E01D204F49087069
:10BCB00001204F49087002204E49086004204E4977
:10BCC00008605D484E4908604F4850490860FBF7DE
:10BCD000E1FB43E24E48007801284DD100204C4959
:10BCE0000870404908700CF0EFFB3F490860464877
:10BCF0000078484908704448407848704248807845
:10BD000088704148C078C8704948001DF4F7E0FACF
:10BD100005464048F4F7DCFA85421AD045480068E9
:10BD2000401C444908600846006803280DD90020DB
:10BD3000086002203A4908703A4800780121084317
:10BD400038490870FDF7C6FA09E00720274908704E
:10BD500005E00020374908601E20244908700120B2
:10BD600023490870234908600020234908602B48B4
:10BD700023490860FBF78EFBF0E11A4800780128A0
:10BD800017D10CF0A1FB1849086000201549087074
:10BD90000D20164908700120154908700620154924
:10BDA0000860002014490860244815490860FBF722
:10BDB00071FBD3E10B480078012848D10CF084FBDB
:10BDC00009490860002007490870012008490870E7
:10BDD00008490860002008490860194808490860B7
:10BDE00030E0000088020020980200208502002038
:10BDF00086020020800200207C020020F820020041
:10BE000064020020F62002006C020020680200207C
:10BE1000870200205C000020900200202621020002
:10BE2000890200208A020020282102001421020039
:10BE3000560200209402002016210200FE2002007B
:10BE400024210200FBF726FB2120D549087085E15B
:10BE5000D448007801281AD10CF036FBD24908608A
:10BE60000020D04908702220CD4908700120CF4918
:10BE700008700220CE4908600420CE490860CE48F0
:10BE8000CE490860CE48CF490860FBF703FB65E167
:10BE9000CD480078012844D10020CB490870C8481B
:10BEA000C078CA49487008464078042108400428F0
:10BEB00017D10020C64908600CF006FBBA4908609B
:10BEC0000120BA490870BA4908600020B9490860E1
:10BED000C048BA490860FBF7DDFA0E20B049087087
:10BEE0001FE0BB480068401CB9490860084600686C
:10BEF000FF212D3188420ED90020B549086002206B
:10BF0000B5490870B548007801210843B349087065
:10BF1000FDF7E0F905E00120A24908702120A049C1
:10BF200008701BE19F480078012821D10020AC490E
:10BF300008709C4908700CF0C7FA9B490860A94832
:10BF4000C078A8491431C97848437D214843C117B6
:10BF5000490E0918C8117D21C900F4F7EFF8C01C7B
:10BF600087B23946082009F0ABFF0F208C490870D2
:10BF7000F4E0082009F0ECFD00280BD102209649DE
:10BF80000870964800780121084394490870FDF72D
:10BF9000A1F996E09248007801283ED192480088A5
:10BFA000FF21013108439049088000208F49087023
:10BFB0008B4908708B48C0788A491431C978484346
:10BFC0007D214843C117490E0918C8117D21C900B8
:10BFD000F4F7B4F8C01C87B23946082009F070FFA6
:10BFE0000CF072FA7049086012206D490870012047
:10BFF0006E49087002206E4908607A481430C07893
:10C000000C2148436B49086079486C4908607948BD
:10C010006C490860FBF73EFA53E077480078012846
:10C020000BD1F8F703FD012807D100206F490870F4
:10C03000714908705A49087043E0FDF769F9012811
:10C040001AD1FDF77FF90020684908700CF03CFA1E
:10C050005549086010205249087001205349087062
:10C06000062053490860002052490860634853493C
:10C070000860FBF70FFA24E0FDF74AF902281AD10D
:10C08000FDF760F90020594908700CF01DFA464987
:10C0900008601020424908700120444908700620B9
:10C0A00043490860002043490860554843490860F7
:10C0B000FBF7F0F905E001204C4908700F203849E2
:10C0C00008704BE03748007801280CD100203E4929
:10C0D00008703449087036490860364908600F20F6
:10C0E0002F49087002E010202D49087036E03648CC
:10C0F0000078012815D100203349087029490870BB
:10C100001320274908700120284908702849086031
:10C110000020284908602F4828490860FBF7BAF931
:10C1200002E012201E49087018E01E48007801281D
:10C130000FD10020244908701A4908701C49086072
:10C140001C4908600120244908700F201449087018
:10C1500002E013201249087000E000BF00BF104841
:10C1600000780F281BD00E480078002817D00CF05C
:10C17000ABF90D490968401A224988420FD3174884
:10C1800000780221084315490870022012490870FE
:10C1900000200849086006490860FDF79BF8F8BDD3
:10C1A00085020020880200209802002086020020DC
:10C1B000800200207C020020F620020064020020A1
:10C1C0006C02002068020020870200205C00002032
:10C1D0009002002026210200890200208A0200200D
:10C1E0008402002086000020600400208D020020D0
:10C1F00004210200301300208B0200201E210200C7
:10C2000018210200B0AD01007047000010B52548AC
:10C210000078002804D0012812D002283ED12AE05C
:10C2200002F07AFA0A2805D107F052FC02201D49D3
:10C23000087004E000F0B0F801201A4908702EE000
:10C2400002F06AFA0A2815D1002002F069F90020EC
:10C2500015490870082000F08DF800201349086087
:10C260001349086013490860134814490860022004
:10C270000C49087013E002F04FFA01280DD100209C
:10C280000F49088000F088F8102000F073F80D487E
:10C290000A49086001200349087000E000BF00BFA0
:10C2A00010BD0000640300203A030020087F002036
:10C2B0000C7F0020187F00205A6B7C8D107F00209F
:10C2C0001C7F00208D7C6B5AF8B52548007800282B
:10C2D00002D0012840D107E03C21052009F0F0FD03
:10C2E00001201F49087038E0052009F031FC0028C2
:10C2F00031D1022000F0F2F900901220FAF788FB09
:10C3000000281ED11748F3F7E3FF05462946009899
:10C31000F4F75FF804461449F4F750FB11D21148C2
:10C32000F3F7D6FF04461149F3F7EAFF0F48F3F796
:10C33000CFFF0646F4F7E0FA04460D4AF3F7E9FFAB
:10C3400006E01220FAF776FB06490098F3F7D8FFCB
:10C3500000200349087000E000BF00BFF8BD0000E6
:10C360001C0300201D03002000001643A01800201D
:10C3700085030020082803D10121064A117008E036
:10C38000102803D10221034A117002E00021014A62
:10C39000117070478C020020F0B585B009F01EF8CE
:10C3A0000546802102F080F80CF08EF8964908606E
:10C3B0000421964808F0EEFF012817D00421944884
:10C3C00008F0E8FF012811D0002190480068F4F738
:10C3D000EBFA0BD38F498D480068F4F7EFFA05D3D9
:10C3E00000218B480068F4F7DFFA04D20020874967
:10C3F0000860874908600221874808F0CBFF0128C0
:10C4000002D10020844908804D20FAF701FB002862
:10C4100043D04D20FAF70EFB7F480088F4F7F9F976
:10C42000432109060290F4F719F87C490390F3F7C9
:10C430007FFF0746754801683846F3F7D2FF064686
:10C44000734801683046F3F773FF05467449F3F704
:10C4500057FF7448F3F73CFF03906F480088F4F7E8
:10C46000D8F9432109060090F3F7F8FF6B490190D2
:10C47000F3F75EFF0290654801680298F3F7B1FF99
:10C4800007466949F3F7EAFF06460399F3F750FFB9
:10C4900005466449F3F734FF3FE05F480088F4F74E
:10C4A000B8F9432109060290F3F7D8FF07465F4920
:10C4B000F3F73EFF0390554801680398F3F791FFA7
:10C4C0000646534801683046F3F732FF05465449A3
:10C4D000F3F716FF5348F3F7FBFE03904E4800882E
:10C4E000F4F797F9432109060090F3F7B7FF0746E1
:10C4F0004E49F3F71DFF0190444801680198F3F796
:10C5000070FF49490290F3F7A9FF06460399F3F734
:10C510000FFF05464349F3F7F3FE4248F3F7D8FE11
:10C520000746F4F7E9F90546414AF3F7F2FE002021
:10C530004049086001204049087000203F490870C8
:10C540003749091DF3F7DCFE354908310020F3F7C0
:10C55000D7FE344908310020F3F7D2FE304930319C
:10C560000020F3F7CDFE2E4934310020F3F7C8FE4A
:10C570002B4938310020F3F7C3FE29493C31002014
:10C58000F3F7BEFE264940310020F3F7B9FE002440
:10C5900005E00020A1002A4A5050601C84B2102CF3
:10C5A000F7DB40212748F3F76CFE002405E000206C
:10C5B000A100254A5050601C84B2102CF7DB0024E7
:10C5C00005E00020A100214A5050601C84B2142CC8
:10C5D000F7DB002405E00020A1001D4A5050601C3C
:10C5E00084B21E2CF7DB00201A4908801A49087013
:10C5F0001A4908801A4908801A4908701A490860BF
:10C600001A49087005B0F0BD4C0300200C7F0020D3
:10C61000087F00200080BB441C7F00200AD7034015
:10C62000E8180020A018002000007A44C3F5A83EB6
:10C6300085030020187F0020650300203A030020B6
:10C64000EC1600202C1700206C170020AC170020DF
:10C65000FC170020340300203603002028030020AC
:10C660002A0300202C030020600300202D0300205B
:10C670000349C9788900034A89180160704700009E
:10C680009A000020301300200349C978C900034AEA
:10C6900089180160704700009A00002030130020C4
:10C6A00010B50221C02000F093FC012805D10349F8
:10C6B00008700221C02000F05FFC10BD8402002041
:10C6C00005480078002804D00020034908700120A4
:10C6D00070470020FCE70000AF030020F8B50446D7
:10C6E00023000EF0ECFC0D6A080C2A3D42474C5129
:10C6F000565B60656A003248F3F7EAFDF8BD3048E2
:10C700000838F3F7E5FD05460021F4F74DF90FD29F
:10C710002B4908390020F3F7F3FD29480838F3F7CF
:10C72000D7FD0746F4F7E8F80546264AF3F7F1FD8A
:10C7300023480838F3F7CCFDE0E72148001FF3F762
:10C74000C7FD05460021F4F72FF904D21C49091F43
:10C750000020F3F7D5FD1A48001FF3F7B9FDCDE728
:10C760001748001DF3F7B4FDC8E715480830F3F784
:10C77000AFFDC3E712480C30F3F7AAFDBEE710483F
:10C780001030F3F7A5FDB9E70D481430F3F7A0FD1D
:10C79000B4E70B481830F3F79BFDAFE708481C30AF
:10C7A000F3F796FDAAE706482030F3F791FDA5E7D9
:10C7B00003482430F3F78CFDA0E70020C0439DE739
:10C7C000A818002085030020002014490979134A85
:10C7D000D27852001143114A5279920011430F4A04
:10C7E0005278D20011430D4A127A120111430B4ABA
:10C7F000927852011143094AD27992011143074AB2
:10C800001278D2011143054A927912021143034A68
:10C81000527A5202114388B270470000401900203A
:10C8200001490160704700002A16002010B5044637
:10C8300023000EF044FC0D3C080C11161B20252A89
:10C840002F343C393C001B48F3F742FD10BD19481A
:10C850000838F3F73DFDF9E71648001FF3F738FDF8
:10C86000F4E71448001DF3F733FDEFE711480830F3
:10C87000F3F72EFDEAE70F480C30F3F729FDE5E763
:10C880000C481030F3F724FDE0E70A481430F3F7C2
:10C890001FFDDBE707481830F3F71AFDD6E7054818
:10C8A0001C30F3F715FDD1E703480068CEE7002000
:10C8B000C043CBE7F018002024030020FEB5054656
:10C8C0000C462846F3F7A5FF07468F21C905F3F765
:10C8D000C5FD06462046F3F79CFF31460090F3F76E
:10C8E00080FD0746F3F7BEFF0190019800F018FDA8
:10C8F000FEBD70B504462046F3F78BFF05468F2139
:10C90000C905F3F7ABFD70BD70B50024F7F7DEF88D
:10C91000012827D12948F3F7DBFCC00FC00701210C
:10C92000C907884210D12548F3F7D2FCC043461C02
:10C930003046FFF7DEFF0546214801682846F3F739
:10C94000F7FC1F4908600DE01C48F3F7C1FC0646E0
:10C95000FFF7CFFF05461A4801682846F3F73DFD6B
:10C9600017490860164800680121C9074840044675
:10C9700014492046F4F718F804D313492046F4F775
:10C980001DF800D270BD00212046F4F70DF80CD23E
:10C990000120C00744402046F9F77EFF401EC543F2
:10C9A00006492846F3F7ACFC06E02046F9F774FF89
:10C9B00005460249F3F7A4FC00BFE3E7B2190020E3
:10C9C0009C0300200AD723BD0AD7233D01480068F5
:10C9D00070470000107F002010B50D480078002837
:10C9E00013D10C48007800280FD10B48007801289B
:10C9F0000BD10A480078002807D1FCF783FC0421FA
:10CA00000840042801D1012010BD0020FCE70000EF
:10CA1000A003002099030020AC0300202103002084
:10CA200010B50020284988704870C87008702749E0
:10CA30000870274908702749087027490870274956
:10CA4000087005E0F8F768F8FAF762F9FCF7FCF906
:10CA5000234800780028F5D00421224808F09AFCE9
:10CA600001280BD000211F480068F3F79DFF05D374
:10CA70001D491C480068F3F7A1FF02D21B48194961
:10CA800008601B4800681B4988420AD018480068A3
:10CA90001949884205D017481549086013481149BB
:10CAA0000860134800681449884206D11020FFF737
:10CAB00061FC0020FAF732F904E000200F49086019
:10CAC0000F49086010BD00004019002064030020D9
:10CAD0002103002099030020AC0300201C03002048
:10CAE000AE030020387F0020000070420000A0410B
:10CAF000107F00205A6B7C8D8D7C6B5A087F002044
:10CB00000C7F0020F8B507460C463846F3F781FE47
:10CB100005461549F3F7F4FB1348F3F7D9FB0090EA
:10CB2000F3F7EAFE0546114AF3F7F3FB0E48F3F775
:10CB3000CFFB05460E49F3F7E3FB0B48F3F7C8FBC1
:10CB40000C4908602046F3F764FE05460649091DB6
:10CB5000F3F7D6FB0448001DF3F7BAFB064908605B
:10CB6000012006490870F8BDA018002085030020A8
:10CB700066030020007F0020047F0020980300202F
:10CB8000FEB5FFF743FBFBF7E7FC08F0C7FC01F03D
:10CB9000C3FD0A2856D171480078002802D0012828
:10CBA0004FD122E008F0C4FF0821084008281BD11B
:10CBB000FAF798FD012817D1032008F0E1FFFAF7F2
:10CBC00097FDF9F77DFE0BF07FFC6549086065482D
:10CBD0000078FCF751FCF9F755F9002804D1012041
:10CBE000614908705D4908702BE0FAF77BFD012868
:10CBF00026D1032008F0C4FFFAF77AFDF9F760FEAA
:10CC00000BF062FC56490968401A584908600BF05D
:10CC10005BFC53490860554800685549884202D971
:10CC20005448524908604F480078FCF725FCF9F752
:10CC300029F9012804D10020484908704A490870A0
:10CC400000BF84E001F068FD012819D1FAF79AFECF
:10CC5000012815D10BF038FC47490860FAF742FD6E
:10CC6000012874D1FAF744FDF6F7CAFFF9F728FE58
:10CC70003C480078FCF700FC2220F9F7DBFE66E078
:10CC800001F04AFD012862D10BF01EFC3A49096807
:10CC9000401A3A4988425AD32220F9F7B9FE0028AF
:10CCA00052D1F9F7EFF8012851D135480088F3F750
:10CCB000B0FD432109060290F3F7D0FB0746314946
:10CCC000F3F736FB0646304801683046F3F789FB38
:10CCD00005462E4801682846F3F72AFB04462C49EE
:10CCE000F3F70EFB2B48F3F7F3FA02902448008881
:10CCF000F3F78FFD432109060090F3F7AFFB2149BD
:10CD00000190F3F715FB07461F4801683846F3F713
:10CD100068FB06462049F3F7A1FB05460299F3F7A5
:10CD200007FB04461B49F3F7EBFA1A48F3F7D0FA6E
:10CD30000646F3F7E1FD0446184AF3F7EAFA022043
:10CD400004F07EFC0EF006FA2220F9F773FEFBF7E2
:10CD5000B5FFFCF7FDF9FFF7B7FAFEBDA003002011
:10CD6000A403002058030020A8030020BC030020D7
:10CD70008096980080841E004C030020E0C81000BC
:10CD80001C7F0020C3F5A83E0C7F0020087F0020F8
:10CD9000E8180020A018002000007A448503002035
:10CDA0000120034908700020024908707047000004
:10CDB0008D02002085020020FEB505465B4806680E
:10CDC00007685B4805705B480570002D60D0002443
:10CDD00005E00020A100584A5050601C84B2102C7D
:10CDE000F7DB002405E00020A100544A5050601CED
:10CDF00084B2142CF7DB002405E00020A100504A87
:10CE00005050601C84B21E2CF7DB00204D49087086
:10CE10004D4908804D4908804D4908804D490870AA
:10CE20004D4908604D4908704D49F3F769FA4D497D
:10CE30000020F3F765FA4B4928310020F3F760FA38
:10CE400048492C310020F3F75BFA46493031002085
:10CE5000F3F756FA424934310020F3F751FA4049CA
:10CE600038310020F3F74CFA002405E00020A1003F
:10CE70002E4A5050601C84B20A2CF7DB00203A493D
:10CE800008703A4908703A4908703A4908604BE01E
:10CE900036480078032840DD00241EE0A100234A24
:10CEA00050583146F3F78AFD02D8A0001F490E58AA
:10CEB000A1001E4A50583946F3F776FD02D8A0006B
:10CEC0001A490F58A000194A11582A480068F3F768
:10CED0002FFA28490860601C84B2244800788442F4
:10CEE000DCDB22490978881EF3F788FC3146029082
:10CEF00020480068F3F76DFA39460090F3F769FAB5
:10CF000001900299F3F7AAFA1A490860002017491C
:10CF1000087001201649087006E0002013490870C7
:10CF20001349087013490860FEBD00007418002002
:10CF300065030020390300206C170020AC17002087
:10CF4000FC170020360300203403002028030020B3
:10CF50002A0300202C030020600300202D03002062
:10CF6000A8180020F0180020370300203803002004
:10CF70003A0300203C03002070B504460D460449E6
:10CF800060180022294609F027FF002070BD00002C
:10CF9000100E0240F8B504460E4615460548A90095
:10CFA0004018071901223146384609F015FF0020C4
:10CFB000F8BD0000300D024070B504460D4603492F
:10CFC00060182946FAF7BAFC70BD0000040D024053
:10CFD00070B504460D46034960182946FAF7AEFCC1
:10CFE00070BD0000000E024070B504460E461546A6
:10CFF000214960180022314609F0EEFE00201F4949
:10D000006118B20088502A781B49091F6018314600
:10D0100009F0E2FE6A7818490C396018314609F0C7
:10D02000DBFEAA78144910316018314609F0D4FEAD
:10D03000EA78114914316018314609F0CDFE2A7999
:10D040000D4918316018314609F0C6FE6A790A495F
:10D0500020316018314609F0BFFE0948806801217F
:10D06000C9038843A979C9030122D20311400843A7
:10D0700003498860002070BD0C0D0240000C024086
:10D08000000F024010B50346024818188C000251E8
:10D09000002010BD000C024070B504460D46044946
:10D0A00060180122294609F097FE002070BD00009B
:10D0B0000C0D024070B504460D4616460349601833
:10D0C0003246294609F088FE002070BD080D024056
:10D0D0000146042901D1024800E0024870470000DF
:10D0E00000020040004000400146002906D001290E
:10D0F00007D0022907D0032909D106E001208007C3
:10D1000006E0044804E0044802E0044800E000BFF0
:10D1100000BF704700010040006000400064004014
:10D1200070B588B0044600250026042C01D0052CDB
:10D1300071D1102168460EF019FE2046FFF7C8FF96
:10D140000546362161435D4A891808461030F3F7D9
:10D15000BFF881B26846418036216143574A891839
:10D1600008461430F3F7B4F8C1B26846417036206F
:10D170006043524940180830007E01281AD100202F
:10D18000694688800AF0A4FD0290362161434B4A2B
:10D19000891808461C30F3F79BF881B26846C180B5
:10D1A00036216143454A891808460830F3F790F85C
:10D1B000039013E00320C002694688804B21490296
:10D1C0000291012189026846C180362161433B4AB0
:10D1D000891808460830F3F77BF80390362060433F
:10D1E000364940180830407E69460870284601F0EC
:10D1F00029FA0021284601F0EFF90121284601F023
:10D20000EBF90021284601F006FA0121284601F039
:10D21000EEF951E0FFE7102104A80EF0A7FD20462B
:10D22000FFF762FF064636216143244A8918084603
:10D230001030F3F74DF881B26846418236216143E0
:10D240001E4A891808461430F3F742F8C1B26846FE
:10D2500041740AF03DFD069036216143174A891852
:10D2600008461C30F3F734F881B2684681823621D3
:10D270006143124A891808460830F3F729F80790E5
:10D28000362060430D4940180830417E68460174DD
:10D2900004A930460CF0BEFB002130460CF084FBA4
:10D2A000012130460CF080FB002130460CF09BFB46
:10D2B000012130460CF083FB08B070BDAC0D00209E
:10D2C00070B504460A212046F2F738FF06010A210C
:10D2D0002046F2F733FF7018C5B2284670BD08B576
:10D2E0000020009000BF00980028FCD008BDF8B5D1
:10D2F0000446002500270FE00A212046F2F71EFF12
:10D300008EB23046B840284385B2381DC7B20A21D4
:10D310002046F2F713FF84B2002CEDD12846F8BD69
:10D32000F8B50446002500270EE00A212046F2F752
:10D33000EFFE0E463046B8400543381DC7B20A21FD
:10D340002046F2F7E5FE0446002CEED12846F8BD53
:10D3500010B500F089F810BD10B5C046C04610BD2C
:10D3600070B504460D4601260022294620460830A5
:10D3700009F032FD0026304670BD014601208A6862
:10D3800008239A438A60002070470000F8B50546DC
:10D390000C460127244885420CD12448806A10217C
:10D3A0008843224988620846806A102108431F4941
:10D3B00088620BE01D48806A202188431B498862EF
:10D3C0000846806A20210843184988620020A86026
:10D3D000207AA860606800012168884201D9012094
:10D3E000F8BD207A402814D10120286061682068A7
:10D3F000F2F78EFEC008401EC6B2092E03DA0021E5
:10D40000284600F01FF83146284600F016F8074677
:10D4100008E000202860607A4000A17A084360722A
:10D42000607A28613846DBE70004004000200040B5
:10D4300001460020CA68D0B2704702460120516000
:10D440000020704770B504460D460126012229468A
:10D450002046083009F0C0FC0026304670BD024668
:10D460000120D1600020704710B5F74800780F28E0
:10D4700071D00CDC0C284FD004DC00280FD00B2816
:10D480006AD117E00D2856D00E28F9D192E0153850
:10D4900003000DF014FE05FDFCFBFAF96100052107
:10D4A000EA480068FFF75CFF0421E8480068FFF7DE
:10D4B000C9FF9DE2E5480068406908280FD10521B1
:10D4C000E2480068FFF74CFF0421E0480068FFF7DE
:10D4D00047FFA221DD480068FFF7C1FF1BE0DB48E2
:10D4E00000684069182816D10C20D749087005211A
:10D4F000D6480068FFF734FF0421D4480068FFF7DE
:10D500002FFFD3480088FF22120210400112CF489B
:10D510000068FFF7A4FF6BE2CC4800684069282848
:10D5200008D10D20C8490870C9480178C74800686B
:10D53000FFF795FF5CE2C5480068406928280CD1D8
:10D540000521C2480068FFF77DFF0421BF4800683D
:10D55000FFF706FF2DE09CE03CE2BC480068406914
:10D5600010281ED10521B9480068FFF7F9FE0421F3
:10D57000B6480068FFF7F4FEA321B4480068FFF73F
:10D580006EFFB4480088012805D10221AF48006829
:10D59000FFF7E6FE0DE00221AC480068FFF752FFFE
:10D5A00007E0AA4800684069402802D10E20A64939
:10D5B00008701DE2A54800684069502831D1A5488F
:10D5C000008800285FD0A1480068FFF731FFA2491A
:10D5D00009680870A0480068401C9F490860052140
:10D5E0009A480068FFF7BCFE042198480068FFF7DE
:10D5F000B7FE98480088401E964908800846008873
:10D60000012808D10F209049087002218F48006836
:10D61000FFF7A6FE37E002218C480068FFF712FFF3
:10D6200031E08A480068406958282CD18748006852
:10D63000FFF7FEFE88490968087087480068401CAB
:10D640008549086083480088401E82490880084652
:10D650000088002817D105217C480068FFF780FE6C
:10D6600004217A480068FFF7EDFE0AF02DFF7B49A0
:10D6700008607B4800781021884310307849087092
:10D68000002071490870B3E18CE1C0E078E068E007
:10D6900032E06E480068406958282CD16B48006819
:10D6A000FFF7C6FE6C49096808706B480068401CAB
:10D6B0006949086067480088401E66490880084636
:10D6C0000088002817D1052160480068FFF748FE50
:10D6D00004215E480068FFF7B5FE0AF0F5FE5F49D9
:10D6E00008605F4800781021884310305C4908705A
:10D6F0000020554908707BE100205A4908805348B2
:10D700000068406908280FD1052150480068FFF7DC
:10D7100027FE04214D480068FFF722FEA2214B4856
:10D720000068FFF79CFE1BE0484800684069182825
:10D7300016D1162044490870052144480068FFF7B7
:10D740000FFE042141480068FFF70AFE40480088A8
:10D75000FF221202104001123C480068FFF77FFED2
:10D7600046E13A4800684069282808D11720364920
:10D7700008703748017835480068FFF770FE37E1D8
:10D78000324800684069282840D132480088401E4D
:10D7900034490988884221D10AF096FE324908604E
:10D7A0002D4800682F4A1288815C28480068FFF7DE
:10D7B00056FE2E48008801280CD12D4800880028EC
:10D7C00008D12C480088002804DD2A480088401E23
:10D7D0002849088018201C49087017E01D48008857
:10D7E000401E20490988884210DD1720164908701C
:10D7F000194800681B4A1288815C14480068FFF7CA
:10D800002EFE18480088401C16490880F0E00F489A
:10D8100000684069282816D11448008800282BD1B8
:10D82000094908700E4800781021884310300C49CF
:10D830000870052105480068FFF792FD04210348A0
:10D840000068FFF7FFFDACE0060000203800002074
:10D8500034000020260000200800002020000020C6
:10D8600036000020240000201C0000203200002090
:10D87000280000202C00002060480088002830D0BC
:10D880005F4800885F49098840185D4908805E4804
:10D8900000685C49098840185B4908605B4800885B
:10D8A000002803DD40205A49088006E059480088D6
:10D8B0005749088000205749088000204F490880B8
:10D8C0001920554908700120544908800521544801
:10D8D0000068FFF745FD042151480068FFF7B2FDDD
:10D8E0005FE04A48008800281DDD45480088403038
:10D8F000434908804448006840304349086040205C
:10D900004349088019204449087001204349088090
:10D91000052143480068FFF723FD042140480068C3
:10D92000FFF790FD3DE03B480088002821DD3448AA
:10D93000008840303249088033480068403032491E
:10D940000860344800883249088000203149088046
:10D9500019203149087001203049088005213048DC
:10D960000068FFF7FDFC04212D480068FFF76AFD01
:10D9700017E028480088002813D12A480078102191
:10D98000884310302749087000202349087005217A
:10D9900023480068FFF7E4FC042121480068FFF7F2
:10D9A00051FD25E01E4800684069102811D115205E
:10D9B0001949087005211A480068FFF7D1FC0421B5
:10D9C00017480068FFF7CCFCA22115480068FFF754
:10D9D00046FD0DE000201049087005211048006840
:10D9E000FFF7BEFC04210E480068FFF72BFD00BFC7
:10D9F00000BF0B480068FFF7C0FC10BD28000020E6
:10DA0000340000202A000020080000202C00002004
:10DA10002600002030000020060000202E000020FC
:10DA2000380000203600002002480078C006C00FF1
:10DA30007047000036000020024800788006C00FC2
:10DA400070470000360000201CB50220F5F78AFF61
:10DA5000072168460EF08AF90021684641700121CD
:10DA600081700021C17001714171012181716A468B
:10DA700003210020FFF7B8FA002203211046FFF728
:10DA800001FB012203210020FFF714FB1CBD10B590
:10DA900000F004F80220F5F757FF10BDF0B587B08D
:10DAA000072168460EF062F9142102A80EF05EF913
:10DAB0000021684641706A4603210020FFF794FA6E
:10DAC000042203210020FFF7DDFA012108200AF0DB
:10DAD00037F90021684601724173C17201218173D7
:10DAE000017300218172417202A90220F5F748FFFB
:10DAF0000AF0EEF807460D49F2F70AFB84B201205E
:10DB00000004001B85B229460220F5F7D5FE01204E
:10DB10000004001B86B231460220F5F7DDFE01212C
:10DB20000220F5F7FFFE07B0F0BD0000E02801007D
:10DB30001CB5002108200AF003F90220F5F712FFB6
:10DB40000122062141208001FFF7B4FA072168462F
:10DB50000EF00CF90021684641700121817000210E
:10DB6000C17001714171012181716A460B218020D0
:10DB7000FFF73AFA00220B218020FFF79BFA6A4652
:10DB80000C218020FFF730FA01220C218020FFF7C2
:10DB900091FA6A4603210020FFF726FA00220321AA
:10DBA0001046FFF76FFA012203210020FFF782FAE7
:10DBB0001CBD0000014800787047000030050020BF
:10DBC00003480078002801D1012070470020FCE7BD
:10DBD000300400201CB5FFF761FF072168460EF0F6
:10DBE000C5F8002168464170012181700021C17093
:10DBF00001710121417181716A4606214120800134
:10DC0000FFF7F2F90122062141208001FFF752FAC5
:10DC10000BF03AF90020034908702920F9F77EF843
:10DC20001CBD00003004002010B52B4800780028EF
:10DC300004D0012821D0022848D129E02920F8F772
:10DC4000E7FE00280BD02920F8F7F4FE4B21C9008D
:10DC5000112009F091F801201F4908700CE000F034
:10DC600077F8012808D100F087F8C821112009F0C1
:10DC700083F80120184908702CE004200AF082FF84
:10DC8000012804D10BF000F902201349087021E0AB
:10DC90001120F5F7C5FE002817D104200AF072FF05
:10DCA000012812D100F038FD0A280ED1F9F7AAFE9A
:10DCB00000280AD1F9F722F8012806D10BF0A4F8C0
:10DCC00000F05AF800200449087003E000200249DF
:10DCD000087000BF00BF10BD3004002010B5074819
:10DCE0000078012808D11020F5F79AFE002803D10A
:10DCF00002490870FFF7A8FE10BD00003C0000209C
:10DD000010B500240AF0E0FB05490968441A0548EB
:10DD10000068844201D3002010BD0120FCE7000010
:10DD2000B0020020AC02002010B500240AF0CCFBA9
:10DD300005490968441A05480068844201D3002057
:10DD400010BD0120FCE70000A8020020A402002072
:10DD500001480078704700002D0400200146024869
:10DD600000780840704700002B040020014800782C
:10DD7000704700009F020020002001490870704792
:10DD80002D0400200146034800788843014A1070A2
:10DD9000012070472B040020002801DD082800DD49
:10DDA0007047421E01239340D9B2034A12788A4336
:10DDB000014B1A7000BFF3E79F0200200348007870
:10DDC000002801D1012070470020FCE79D020020BF
:10DDD00003480078002801D1012070470020FCE7AB
:10DDE0002A04002010B50AF033F903F0DBFB10BD64
:10DDF0000020034908700349087003490870704700
:10DE00002A0400202B0400202C04002010B579489F
:10DE10000078002802D001286FD1D3E0FFF7A6FFD9
:10DE2000754908700846007803000DF048F90906A6
:10DE30005067B0A0B0B0B097B0000D20F8F7F2FD79
:10DE4000000E6E490978884215D00D20F8F7EAFDDA
:10DE5000000E6A4908700D20F8F7E4FD000EAA28AC
:10DE600003D12C20F8F75AFF05E0002201214120C0
:10DE70008001FFF71FF92C20F8F7CAFD002822D0F7
:10DE80000D20F8F7CFFD000EAA281CD12C20F8F7A2
:10DE9000D1FD0AF025F9002811D10022032102202A
:10DEA000F7F7DCF80022012141208001FFF702F999
:10DEB0000A21202008F060FF01204E490870002050
:10DEC0004F49087002E000204A49087078E00120BC
:10DED000FFF762FF0020484908704A480078012196
:10DEE0000843484908700120474908705A20F8F74C
:10DEF00015FF00203F49087062E077E00220FFF73D
:10DF00004BFF00203C49087000F0FAFBFF2105316F
:10DF100088420ED11F20F8F785FD002809D0394826
:10DF200000780821084337490870002031490870FB
:10DF300013E000F0E5FB3549884205D1314800780F
:10DF4000202108432F4908702E48007802210843F9
:10DF50002C49087000202749087031E00420FFF7A1
:10DF60001BFF0020244908702249087028E0032084
:10DF7000FFF712FF00202049087022480078042192
:10DF800008432049087000201A49087018E0012051
:10DF9000FFF702FF0220FFF7FFFE0320FFF7FCFE62
:10DFA0000420FFF7F9FE0520FFF7F6FE0620FFF735
:10DFB000F3FE0720FFF7F0FE0820FFF7EDFE00BF9D
:10DFC00000BF14E02020F5F72BFD01280DD1012220
:10DFD000114641208001FFF76DF801220321022044
:10DFE000F7F73CF800200349087000E000BF00BFCD
:10DFF00010BD00002A0400202C0400202E04002064
:10E000002F0400202B0400202D0400200203000018
:10E0100010B5F848007803000DF051F80A064C9E40
:10E02000BEFAF9F8F7F6F5F4F3480078002812D0B4
:10E030000020F14908702220F5F7F2FC00280AD1EF
:10E040002320F5F7EDFC012805D1EC4800780821E4
:10E050000843EA490870F5F74DFDE949087008469C
:10E060000078002814D00846007800F0D0F9012884
:10E0700005D1F5F7D1FD0020DE49087019E0F5F76C
:10E08000CBFD022000F0F2F90120DA49087010E01F
:10E090003220F8F7BDFC002808D03220F8F7CAFC7F
:10E0A0000020D84908802C20F8F738FE0020D149FC
:10E0B00008709CE1FFF738FE002849D1D04800786D
:10E0C00000F0A5F9012806D1022000F0CFF90220C6
:10E0D000C84908703FE0CC480078401CC0B2CA492B
:10E0E000087001282DDBC6480078022818D1C548E1
:10E0F0000088401CC3490880084600881E2816DD99
:10E100000022012141208001FEF7D4FFBB480078A6
:10E1100004210843B94908700020B649087010BDB1
:10E12000B84800881E2802DD3220F8F7F7FDB34812
:10E13000007801210843B14908700320AD490870F7
:10E1400002E00120AB490870022000F08FF902E0E4
:10E150000120A84908704AE1FFF7E6FD002817D121
:10E16000A748007800F053F9012808D10020A649FB
:10E170000870F5F751FD00209E4908700BE0F5F797
:10E180004BFD022000F072F901209A49087002E06C
:10E190000220984908702AE1FFF7C6FD00285BD1EC
:10E1A0009748007800F033F9012806D1022000F0EA
:10E1B0005DF904208F49087051E093480078401CB5
:10E1C000C0B291490870C8283FDB8D48007802280A
:10E1D0001FD18C480088401C8A4908800846008866
:10E1E0001E281DDD0022012141208001FEF762FF73
:10E1F00082480078042108438049087000207D4946
:10E2000008708CE7EFE0D4E0A6E08EE070E044E038
:10E2100026E07C4800881E2802DD3220F8F77EFDCB
:10E220007648007802210843744908700120724939
:10E2300008700021222008F09FFD9621232008F07D
:10E240009BFD05206B49087002E0032069490870B6
:10E25000022000F00BF902E0032066490870C6E0D6
:10E26000FFF762FD002814D16548007800F0CFF870
:10E27000012805D10020644908705E4908700BE050
:10E28000F5F7CAFC022000F0F1F8032059490870A4
:10E2900002E0042057490870A9E0FFF745FD002877
:10E2A00022D15748007800F0B2F8012806D10220A8
:10E2B00000F0DCF806204F49087018E0FFF756FD23
:10E2C00002210840002808D14F4908701E2000F0A4
:10E2D000BBF807204749087009E0022000F0C6F8A3
:10E2E00005204449087002E00520424908707EE09C
:10E2F000FFF71AFD002814D14148007800F087F894
:10E30000012805D10020404908703A4908700BE007
:10E31000F5F782FC022000F0A9F8052035490870C5
:10E3200002E006203349087061E0FFF7E9FC0028AD
:10E330000BD13549087031480078042108432F4932
:10E34000087000202B49087005E0022000F08EF8CC
:10E350000820284908704AE0FFF7E6FC002824D18D
:10E360002748007800F053F8012806D109202149F8
:10E370000870022000F07AF81AE023480078401C68
:10E38000C0B22149087064280BDB002008701B48CC
:10E3900000780221084319490870072015490870C0
:10E3A00006E007201349087002E0082011490870B0
:10E3B0001DE0FFF7B9FC002811D11148007800F0EA
:10E3C00026F8012805D100200F4908700949087076
:10E3D00008E0F5F721FC07200649087002E0092053
:10E3E0000449087003E000200249087000BF00BF24
:10E3F00000BF94E69D020020A00200209F020020A2
:10E40000B4020020B60200209E020020704710B522
:10E410000446022C04D10D21802000F007F810BD25
:10E420000B210120000300F001F8F8E770B5044665
:10E430000D4629462046FEF7BFFD002801D00120E9
:10E4400070BD0020FCE7000010B50446044860439E
:10E45000044908600AF038F80349086010BD00005C
:10E4600040420F00AC020020B002002010B504466C
:10E470007D20C000604381004018034908600AF015
:10E4800023F80249086010BDA4020020A802002061
:10E49000704710B5C046C04610BD10B502F026FF4B
:10E4A000C046C04610BD00003EB504460D460A21D8
:10E4B00068460DF05BFC0121092009F041FC0721B1
:10E4C000684601700021C1708170002C03D00320C8
:10E4D0006946487002E0022069464870002168469B
:10E4E00001714171012181710804401B81B26846AC
:10E4F00001816946094802F03AFF084802F012FF1C
:10E500000121064802F021FF012203211120F6F724
:10E51000A5FD0121014802F00EFF3EBD000F0040A5
:10E5200010B50446012C08D10121092009F008FC8E
:10E530000121064802F0FFFE07E00021092009F052
:10E54000FFFB0021014802F0F6FE10BD000F004065
:10E550000149096888B27047400F00403EB5044643
:10E560000A2168460DF002FC0121242009F0E8FB95
:10E570000721684601700021C1708170002C03D012
:10E5800003206946487002E0022069464870002175
:10E59000684601714171817101816946094802F043
:10E5A000E6FE084802F0BEFE0021064802F0CDFE5D
:10E5B000012203211120F6F751FD0121014802F04B
:10E5C000BAFE3EBD400F004010B502F0A1FE10BDE6
:10E5D00010B502F0A2FE10BD70B504460D46002233
:10E5E00029462046143008F0F7FB002070BD70B5B6
:10E5F00004460D4600222946201D08F0EDFB0020B0
:10E6000070BD70B504460D4601222946201D08F054
:10E61000E3FB002070BD70B504460D46012229467B
:10E62000201D08F0D9FB002070BD70B504460D46D2
:10E630000026294620461030F9F780F90646304674
:10E6400070BD0000F0B587B005460C460127224A90
:10E6500007CA04AB07C300200390002C02D104209A
:10E6600007B0F0BD00206860608861780843E188E9
:10E670000843A1880843217808436860207840282F
:10E6800002D02078C02824D1E088C117C90D09180C
:10E690004912890004AA515A8EB2E168B140084675
:10E6A000F2F7B7F80290A068F2F7B3F80190029978
:10E6B000F1F7D4FE03903F2109060398F1F738FEE5
:10E6C0000290F2F7CFF880B2A86104212846FFF744
:10E6D00098FF00273846C3E7A425020001460868D2
:10E6E000C0B2704702461068000A0002CBB218435D
:10E6F00010600020704710B502F0A4FE10BD0000AD
:10E700000348007800020349097808437047000075
:10E71000FF0300200004002003480078042801D1F2
:10E72000012070470A20FCE7FF03002010B50120FC
:10E730001749087017490020F1F7E2FD1321002066
:10E7400001F0E4FB1321012001F0E0FB1321022082
:10E7500001F0DCFB1321032001F0D8FB132104207E
:10E7600001F0D4FB1321052001F0D0FB132106207A
:10E7700001F0CCFB1321072001F0C8FB1321082076
:10E7800001F0C4FB1321092001F0C0FB10BD000003
:10E79000C3020020C4020020032803D0072801D0B0
:10E7A000082833D14F49096A82004F4B9A58120901
:10E7B00091434C4A116281004C4A51580909820028
:10E7C0004B4B9A5812091143464A526A8A434549AB
:10E7D0004A628100474A515809098200464B9A58BB
:10E7E000120911433F4A926A8A433E498A62810074
:10E7F000424A515809098200414B9A581209114363
:10E80000384AD26A8A433749CA626AE002283CD150
:10E810003449C96A8200394B9A5812099143314AE6
:10E82000D1621146896A8200324B9A58120991438B
:10E830002C4A91621146496A82002C4B9A5812095F
:10E840009143284A51621146096A8200264B9A5820
:10E8500012099143234A1162114649688200244BF0
:10E860009A5891431F4A51601146C9688200244B4F
:10E870009A5891431B4AD1601146896882001E4B09
:10E880009A589143174A91602BE016490968820013
:10E89000154B9A589143134A11608100134A5158FD
:10E8A0008200134B9A5811430E4A52688A430D490D
:10E8B0004A6081000F4A515882000F4B9A58114309
:10E8C000084A92688A4307498A6081000B4A515876
:10E8D00082000B4B9A581143024AD2688A4301497D
:10E8E000CA607047405C0040E4240200BC2402007F
:10E8F0000C250200942402005C2502006C24020016
:10E9000034250200F8B505460C462B000CF0D7FB69
:10E91000140B2532485E7287A1B0CFF4F2F1F0EF0C
:10E92000EEEDECEBEAE9A000D4490858A100D44A86
:10E93000515808430090A000D24E3058A600D24F44
:10E94000BE5930430246A000D04E3358A000D04EEE
:10E950003158204602F0ECFB8EE100200090A00030
:10E96000CA490B58A000C7490A580021204602F0A6
:10E97000DFFB81E1A000C14908580090A000C34E10
:10E980003058A600C34FBE5930430346A000BE4EC8
:10E990003258A000BE4E3158204602F0C9FB6BE150
:10E9A000A000B64908580090A000B84E3058A60004
:10E9B000B84FBE5930430346A000B24E3258A000B3
:10E9C000B34E3158204602F0B3FB55E1A000AC49EC
:10E9D00008580090A000AD490858A100AD4E7158EC
:10E9E00008430346A000A7490A580021204602F028
:10E9F0009FFB41E1A000A1490858A100A04A51583D
:10EA000008430090A000A34E3358A0009D4E3258FA
:10EA1000A0009F4E3158204602F08AFB2CE1A00056
:10EA200096490858A100964A515808430090A00002
:10EA3000944E3058A600944FBE5930430246A00071
:10EA4000944E3358A000924E3158204602F070FB8D
:10EA500012E1A000894908580090A0008B490B588A
:10EA6000A00088490A580021204602F061FB03E11A
:10EA7000A00082490858A100814A515808430090DB
:10EA8000A000824E3058A600824FBE593043034644
:10EA9000A0007C4E3058A6007B4FBE593043024642
:10EAA000A0007B4E3158204602F042FBE4E0A0007B
:10EAB00072490858A100724A515808430090A000BA
:10EAC000724E3058A600734FBE5930430346A00023
:10EAD0006C4E3258A0006E4E3158204602F028FB92
:10EAE000CAE0C8E0C3E0B7E0A5E08CE078E062E00F
:10EAF00048E034E01DE0FFE7A00060490858A100AD
:10EB00005F4A515808430090A00060490858A1008E
:10EB1000604E715808430346A0005A490858A100A6
:10EB2000594E7158084302460021204602F000FB6E
:10EB3000A2E0A000524908580090A000514E305861
:10EB4000A600514FBE5930430246A000514E3358E3
:10EB5000A0004F4E3158204602F0EAFA8CE0A000A7
:10EB600046490858A100464A515808430090A00061
:10EB7000454B1A58A000464B19580023204602F076
:10EB8000D7FA79E000200090A000404E3058A6004F
:10EB9000404FBE5930430346A0003A4E3058A600BD
:10EBA000394FBE5930430246A000394E31582046F5
:10EBB00002F0BEFA60E0A00030490858A100304AD7
:10EBC000515808430090A000324E3358A0002E4EFA
:10EBD0003258A0002E4E3158204602F0A9FA4BE0E0
:10EBE000A00026490858A100254A51580843009022
:10EBF000A00028490B58A00023490A5800212046AC
:10EC000002F096FA38E0A0001C490858A1001C4AFE
:10EC1000515808430090A0001C490858A1001D4EFF
:10EC2000715808430346A00017490A58002120469E
:10EC300002F07EFA20E0A000114908580090A000E0
:10EC4000144E3358A000104E3258A000104E3158C8
:10EC5000204602F06DFA0FE000200090A0000D4960
:10EC60000B5800221146204602F062FA04E02046CA
:10EC7000FFF792FD00E000BF00BFF8BD6C2402006A
:10EC800034250200BC2402000C250200942402005A
:10EC9000E42402005C25020010B5FDF795FD4A4909
:10ECA00008704A480078002802D001287ED138E058
:10ECB00005F0CEFC46490978884206D005F0C8FC2C
:10ECC000434908700120414908703F4800782021DD
:10ECD000084040490978884208D03B480078202104
:10ECE00008403C49087001203849087011F0D8FEEE
:10ECF00039490978884206D011F0D2FE36490870A9
:10ED000001203249087011F0ADFE3449097888427B
:10ED100006D011F0A7FE3149087001202B49087078
:10ED200050E005F095FC0A2803D1012001F0C8FB52
:10ED300002E0002001F0C4FB26480078202803D11F
:10ED4000012001F001FB02E0002001F0FDFA224861
:10ED50000078012802D101F081F802E0002001F0E2
:10ED60007DF81E480078012802D101F0E5F802E0A4
:10ED7000002001F0E1F81A480078002803D10120B2
:10ED800001F03EF802E0002001F03AF81548007862
:10ED9000032807D013480078042803D011480078CE
:10EDA000052804D1012001F06BFB03E006E0002000
:10EDB00001F066FB00200549087003E000200349CC
:10EDC000087000BF00BF10BD07040020FC03002036
:10EDD0000104002002040020030400200404002099
:10EDE0000504002006040020F3B583B00E46092771
:10EDF00000BF0398029000210298F1F7D5FD03D2DD
:10EE0000F90702984840029033000CF058F90604C4
:10EE10000F1C2937455358480299F1F7E2FA02903E
:10EE200001F06EFB019001F0A7F84BE05348029906
:10EE3000F1F7D7FA029001F063FB514908430190C2
:10EE400001F09AF83EE04F480299F1F7CAFA0290B1
:10EE500001F056FB4C490843019001F08DF831E078
:10EE60004A480299F1F7BDFA029001F049FBE1210D
:10EE7000C9040843019001F07FF823E04448029957
:10EE8000F1F7AFFA029001F03BFB6121090508435D
:10EE9000019001F071F815E03E480299F1F7A1FAEE
:10EEA000029001F02DFB212149050843019001F05A
:10EEB00063F807E00298029001F022FB019001F054
:10EEC0005BF800BF00BF0298F1F7E0FC04460D4676
:10EED00020462946002358405940084320D016E0D8
:10EEE0000A22002320462946F1F73CF9D0B23946E0
:10EEF0007A1E57B20190C8B2019901F007F80A22B0
:10EF0000002320462946F1F72DF904460D4600213D
:10EF1000084661406840014306D0002FE0DA03E074
:10EF20000021092000F0F2FF002E15DD062E13DA75
:10EF300001F0E6FA0121C906B1400843019001F051
:10EF40001BF806E039467A1E57B2C8B2002100F01D
:10EF5000DDFFF01CB842F5DD002F0BDB002103982C
:10EF6000F1F722FD06D239467A1E57B2C8B21221F5
:10EF700000F0CCFF05B0F0BD002474490050C34739
:10EF80000000C20700401C460000840700007A44CD
:10EF90000000C84200002041F8B507460C4608258D
:10EFA000002F16D010E00A213846F1F7B1F8009191
:10EFB00029466A1E55B2C8B2009900F0A7FF0A217F
:10EFC0003846F1F7A5F80746002F19D0002DEADAE8
:10EFD00016E00620001BC6B208E029466A1E55B29C
:10EFE000C8B2002100F092FF701EC6B2002E01D000
:10EFF000002CF2D1002C03D10021082000F086FF64
:10F0000023000CF05CF805040A131C252E0001F007
:10F0100077FA009000F0B0FF29E001F071FA0121C9
:10F0200049040843009000F0A7FF20E001F068FACF
:10F03000012189040843009000F09EFF17E001F0D1
:10F040005FFA0121C9040843009000F095FF0EE02B
:10F0500001F056FA012109050843009000F08CFFE9
:10F0600005E001F04DFA009000F086FF00BF00BF00
:10F07000F8BD0000F8B50446FFF758FB23000CF07C
:10F080001EF806CE042B7998CBCE0120400200F06A
:10F0900073FF02206B49087008460078F8F734FBCC
:10F0A0006949086008460068009068490098F1F7CF
:10F0B0007BFC08D266490098F1F7D0F9054601219A
:10F0C000FFF792FE07E062490098F1F7C7F905469D
:10F0D0000321FFF789FEB3E05E4800F04DFF0320F7
:10F0E0005849087008460078F8F70EFB5649086042
:10F0F00008460068009058490098F1F755FC0BD27B
:10F1000053490098F1F7AAF90121C907484005467B
:10F110000321FFF769FE2CE050490098F1F744FC09
:10F120000BD24B490098F1F799F90121C9074840E2
:10F1300005460421FFF758FE1BE049490098F1F706
:10F1400033FC0BD242490098F1F788F90121C90735
:10F15000484005460521FFF747FE0AE03C49009874
:10F16000F1F77CF90121C907484005460621FFF760
:10F170003BFE65E00720400200F0FEFE0120314921
:10F18000087008460078F8F7BFFA2F49086008466B
:10F190000068F1F73EFB07468F21C905F1F75EF9DC
:10F1A00006462A49F1F75AF905460121FFF71CFEE8
:10F1B00046E00120C00200F0DFFE55202149087022
:10F1C00008460078F8F7A0FA1F490860084600686A
:10F1D0000A280DD20021072000F098FE0021062009
:10F1E00000F094FE002118480068FFF7D5FE12E0F9
:10F1F00015480068642809D20021062000F086FE28
:10F20000002111480068FFF7C7FE04E000210E4806
:10F210000068FFF7C1FE13E000F040FE10E00E2191
:10F22000022000F073FE0E21032000F06FFE0A2181
:10F23000042000F06BFE0121052000F067FE00BFF6
:10F2400000BFF8BD080400200C04002000007A4430
:10F250000000C84200020008002474498096184B40
:10F2600020BCBE4CFEB50446FFF760FA01F048F939
:10F27000054600F081FE23000BF021FF0FFD09453C
:10F28000819FD0FCFBFAF9F8F7F6F5F4FD001120A8
:10F29000FE49087008460078F8F756FAFC490860FD
:10F2A000084600680002010F012000F02FFEF84818
:10F2B00000680003010F022000F028FE1221032045
:10F2C00000F024FEF24800880004010F042000F042
:10F2D0001DFEEF4800880005010F052000F016FE16
:10F2E0001221062000F012FEE94800780006010F06
:10F2F000072000F00BFEE64800780107090F082000
:10F3000000F004FE56E32220E04908700846007829
:10F31000F8F71AFADE490860084600680002010F93
:10F32000012000F0F3FDDA4800680003010F02201D
:10F3300000F0ECFD1221032000F0E8FDD448008825
:10F340000004010F042000F0E1FDD1480088000511
:10F35000010F052000F0DAFD1221062000F0D6FD95
:10F36000CB4800780006010F072000F0CFFDC84809
:10F3700000780107090F082000F0C8FD1AE30121F9
:10F38000084600F0C3FD1221022000F0BFFD01205D
:10F39000BE49087008460078F8F7D6F9BC490860FD
:10F3A000096809090A225143B94A12781207120F53
:10F3B00088180021FFF7F0FDFCE20221012000F097
:10F3C000A5FD1221022000F0A1FD0220AF49087026
:10F3D00008460078F8F7B8F9AD4908600120C00484
:10F3E00000F0CAFDAA480068010F052000F08EFD5C
:10F3F000A74800680001010F062000F087FDA4481F
:10F4000000680002010F072000F080FDA04800689E
:10F410000003010F082000F079FDCBE20321012059
:10F4200000F074FD1221022000F070FD03209749C6
:10F43000087008460078F8F787F99549086008468B
:10F4400000680002010F032000F060FD9048006892
:10F450000003010F042000F059FD8D4800880004CE
:10F46000010F09E07CE149E116E1EBE0C7E0A3E030
:10F470007FE05BE019E09CE2052000F047FD844856
:10F4800000880005010F062000F040FD804800784C
:10F490000006010F072000F039FD7D4800780107C4
:10F4A000090F082000F032FD84E20420774908703B
:10F4B00008460078F8F748F975490860084600687A
:10F4C000010F012000F022FD714800680001010FCA
:10F4D000022000F01BFD6E4800680002010F0320AF
:10F4E00000F014FD6A4800680003010F042000F0DA
:10F4F0000DFD674800880004010F052000F006FD9F
:10F50000634800880005010F062000F0FFFC6048FA
:10F5100000780006010F072000F0F8FC5C48007836
:10F520000107090F082000F0F1FC43E2042101204B
:10F5300000F0ECFC1221022000F0E8FC0520534909
:10F54000087008460078F8F7FFF851490860084647
:10F550000068F1F779F900224E4B01910090F1F724
:10F56000D5F80546F1F704FA07460321FFF73CFCFE
:10F5700020E20521012000F0C9FC1221022000F048
:10F58000C5FC06204149087008460078F8F7DCF809
:10F590003F49086008460068F1F756F900223D4BE4
:10F5A00001910090F1F7B2F80546F1F7E1F907464D
:10F5B0000321FFF719FCFDE10621012000F0A6FC64
:10F5C0001221022000F0A2FC0720304908700846F2
:10F5D0000078F8F7B9F82E49086008460068F1F796
:10F5E00033F9054600222B4BF1F790F8019100907A
:10F5F000F1F7BEF907460321FFF7F6FBDAE1072131
:10F60000012000F083FC1221022000F07FFC082082
:10F610001E49087008460078F8F796F81C490860FB
:10F6200008460068F1F710F900221A4B019100908A
:10F63000F1F76CF80546F1F79BF907460321FFF750
:10F64000D3FBB7E10821012000F060FC1221022069
:10F6500000F05CFC09200D49087008460078F8F7B6
:10F6600073F80B49086008460068F1F7EDF80022CE
:10F67000084B01910090F1F749F80546F1F778F948
:10F6800007460321FFF7B0FB94E1000009040020C6
:10F69000100400200000F0400921012000F036FC99
:10F6A0001221022000F032FC0A20C34908700846EB
:10F6B0000078F8F749F8C14908600120C00400F05B
:10F6C0005BFCBE4800880004010F052000F01EFC12
:10F6D000BA4800880005010F062000F017FCB74863
:10F6E00000780006010F072000F010FCB3480078F6
:10F6F0000107090F082000F009FC5BE10A21012045
:10F7000000F004FC1221022000F000FC0220AA49B3
:10F71000087008460078F8F717F8A8490860012033
:10F72000C00400F029FCA54800880004010F052052
:10F7300000F0ECFBA14800880005010F062000F056
:10F74000E5FB9E4800780006010F072000F0DEFB75
:10F750009A4800780107090F082000F0D7FB29E13B
:10F760000B209549087008460078F7F7EDFF93499C
:10F77000086008460068019008460078012836D1E4
:10F780000B21002000F0C2FB1221012000F0BEFB83
:10F7900068460179022000F0B9FB1221032000F035
:10F7A000B5FB694648790A21F0F7C8FCC5B229467D
:10F7B000042000F0ABFB694648790A21F0F7BEFC53
:10F7C000CDB22946052000F0A1FB1221062000F051
:10F7D0009DFB68468179072000F098FB12210820E4
:10F7E00000F094FB6846C179092000F08FFB734854
:10F7F0000078022836D10B21002000F087FB12216F
:10F80000012000F083FB68460179022000F07EFBB6
:10F810001221032000F07AFB694648790A21F0F7AB
:10F820008DFCC5B22946042000F070FB694648797A
:10F830000A21F0F783FCCDB22946052000F066FBD3
:10F840001221062000F062FB68468179072000F053
:10F850005DFB1221082000F059FB6846C1790920A0
:10F8600000F054FB55480078032878D1122100207D
:10F8700000F04CFB694648796421F0F75FFCC5B2A3
:10F880002946012000F042FB694648790A21F0F739
:10F8900055FC06460A21F0F751FCCDB2294602205C
:10F8A00000F034FB694648790A21F0F747FCCDB2F5
:10F8B0002946032000F02AFB694688798021084008
:10F8C00000281CD01221042000F020FB6946897911
:10F8D0004806400E0A21F0F731FCC5B22946052042
:10F8E00000F014FB694689794806400E0A21F0F7BA
:10F8F00025FCCDB22946062000F008FB17E01321B5
:10F90000042000F003FB694688790A21F0F716FC11
:10F91000C5B22946052000F0F9FA694688790A211E
:10F92000F0F70CFCCDB22946062000F0EFFA1321C7
:10F93000072000F0EBFA6946C8790A21F0F7FEFBD0
:10F94000C5B22946082000F0E1FA6946C8790A21C3
:10F95000F0F7F4FBCDB22946092000F0D7FA17489A
:10F960000078042824D10B21002000F0CFFA1221C6
:10F97000012000F0CBFA68464179022000F0C6FA77
:10F980001221032000F0C2FA694688790A21F0F7B3
:10F99000D5FBC5B22946042000F0B8FA694688793B
:10F9A0000A21F0F7CBFBCDB22946052000F0AEFAD4
:10F9B00000E000BF00BFFEBD0904002010040020CD
:10F9C00070B50446FEF7B2FE00F09AFD054600F061
:10F9D000D3FA012C02D0022C79D14DE00121084646
:10F9E00000F094FA1221022000F090FA01204B4915
:10F9F000087008460078F7F727FF4949086008466D
:10FA000000784007C00F002804D00121052000F035
:10FA10007DFA03E00021052000F078FA40480078E4
:10FA20000007C00F002804D00121062000F06EFA64
:10FA300003E00021062000F069FA39480078C00789
:10FA4000C00F002804D00121072000F05FFA03E076
:10FA50000021072000F05AFA314800788007C00FD3
:10FA6000002804D00121082000F050FA03E0002112
:10FA7000082000F04BFA4FE00221012000F046FA86
:10FA80001221022000F042FA0220244908700846A0
:10FA90000078F7F7D9FE2249086008460078C006CA
:10FAA000C00F002804D00121052000F02FFA03E048
:10FAB0000021052000F02AFA194800788006C00FBE
:10FAC000002805D00121062000F020FA04E022E001
:10FAD0000021062000F01AFA114800784006C00FF5
:10FAE000002804D00121072000F010FA03E00021D3
:10FAF000072000F00BFA0A4800780006C00F002823
:10FB000004D00121082000F001FA03E000210820C0
:10FB100000F0FCF900E000BF00BF70BD0A04002047
:10FB200014040020F0B587B00546FEF7FFFD2B005A
:10FB30000BF0C5FA07FD052755A8E3FCFD00A64814
:10FB4000407A552804D10120400200F015FA03E064
:10FB50000520C00100F010FA0220A04908700846F4
:10FB60000078F7F7BDFE9E490860084600680590DA
:10FB70009C490598F0F772FC06460121FFF734F91D
:10FB800026E19548407A552804D10720400200F02C
:10FB9000F3F903E01D20C00100F0EEF901208F49C8
:10FBA000087008460078F7F79BFE8D490860084604
:10FBB0000068F0F749FE064600228B4BF0F7A6FDE1
:10FBC00000228A4B01910090F0F7A0FD0391029072
:10FBD000F0F7CEFE01210490FFF706F9F8E07E4829
:10FBE000407A552804D10120C00200F0C5F903E095
:10FBF0001120C00100F0C0F90A20784908700846B9
:10FC00000078F7F76DFE7649086008460068012124
:10FC1000C907884219D37248006888437049086050
:10FC200008460068F0F710FE064600226E4BF0F71B
:10FC30006DFD00226E4B01910090F0F7FFFC0391E7
:10FC40000290F0F795FE044613E065480068F0F76F
:10FC5000FBFD06460022644BF0F758FD0022654B81
:10FC600001910090F0F7EAFC03910290F0F780FE1A
:10FC7000044661492046F0F7F1FB06460021FFF7F4
:10FC8000B3F8A5E05448407A552804D10120C002B9
:10FC900000F072F903E01120C00100F06DF90121BC
:10FCA000084600F033F91221022000F02FF9042059
:10FCB0004A49087008460078F7F712FE484908607C
:10FCC00008460068F0F7C0FD06460022464BF0F7F4
:10FCD0001DFD0022474B01910090F0F7AFFC03910E
:10FCE0000290F0F745FE044644492046F0F7B6FB83
:10FCF00006460021FFF778F86AE03748407A552831
:10FD000004D10120C00200F037F903E01120C00146
:10FD100000F032F90221012000F0F8F8122102204F
:10FD200000F0F4F807202D49087001E023E03EE0E0
:10FD300008460078F7F7D4FD2949086008460068AE
:10FD4000F0F782FD06460022274BF0F7DFFC002289
:10FD5000284B01910090F0F771FC03910290F0F7AD
:10FD600007FE044625492046F0F778FB06460021A9
:10FD7000FFF73AF82CE01848407A552803D12020A4
:10FD800000F0FAF802E0A02000F0F6F80E20134987
:10FD9000087008460078F7F7A3FD11490860084687
:10FDA0000068059003210598FFF71EF810E00E216A
:10FDB000032000F0ABF80E21042000F0A7F80A2180
:10FDC000052000F0A3F80421062000F09FF800BFF2
:10FDD00000BF07B0F0BD0000462100200B0400204A
:10FDE000180400200050C3470000F04000408F403E
:10FDF000000039C0000039400000C84200401C46E5
:10FE00001249087012490978104A127891421BD0A1
:10FE10000E4909780E4A117001210E4A117000280E
:10FE200009D00A4A11700C49097804229143091D2E
:10FE3000094A117008E00021044A11700649097846
:10FE400004229143044A117070470000C10200204F
:10FE5000C2020020C3020020C402002001210C4A7B
:10FE60001170002809D00B4A11700B490978490814
:10FE70004900491C084A117008E00021054A117028
:10FE80000549097849084900034A11707047000084
:10FE9000C3020020BF020020C402002010B50120D0
:10FEA0001749087017491848F0F72AFA0821002066
:10FEB00000F02CF80821012000F028F80821022089
:10FEC00000F024F80821032000F020F80821042085
:10FED00000F01CF80821052000F018F80821062081
:10FEE00000F014F80821072000F010F80821084657
:10FEF00000F00CF80821092000F008F810BD0000FF
:10FF0000C3020020C4020020FFFFFF0F0A280EDA00
:10FF100001228240064B1B881A43054B1A80142984
:10FF200002DA044A115402E01322024B1A547047B9
:10FF3000BA0200207314002001210C4A117000281D
:10FF400009D00B4A11700B49097802229143891C90
:10FF5000084A117008E00021054A11700549097826
:10FF600002229143034A117070470000C30200202F
:10FF7000C0020020C402002070B50446012046499A
:10FF8000087046480078002807D140222146914356
:10FF900008464349F0F7B4F909E0404800780128E1
:10FFA00005D14021214308463D49F0F7A9F93D48D4
:10FFB0000078002809D03A48F0F78AF91021084360
:10FFC00005463749F0F79CF908E03548F0F780F925
:10FFD0001021884305463249F0F792F932480078FB
:10FFE000002809D02E48F0F773F908210843054688
:10FFF0002B49F0F785F908E02948F0F769F908215D
:020000040001F9
:10000000884305462649F0F77BF928480078002800
:1000100009D02348F0F75CF901210843054620493F
:10002000F0F76EF908E01E48F0F752F945086D0048
:100030001B492846F0F764F91D480078002809D0CC
:100040001748F0F745F90221084305461449F0F72F
:1000500057F908E01248F0F73BF9022188430546BA
:100060000F49F0F74DF913480078002809D00C48E3
:10007000F0F72EF90421084305460949F0F740F945
:1000800008E00748F0F724F90421884305460449AD
:10009000F0F736F970BD0000C3020020BC0200205A
:1000A000C4020020BD020020BE020020BF020020CA
:1000B000C0020020C102002010B59E480078002830
:1000C0001CD101209B490870FCF780FC9A498842AA
:1000D0000AD10420994908700120994908700846FE
:1000E0000078FFF71FFD23E101209449087094492F
:1000F000087008460078FEF7BDFF19E10220FDF701
:100100002DFE002834D000208E4908700220FDF713
:1001100039FE8A480078042810D1894800780328DD
:100120000CD1012085490870002085490870FEF730
:10013000FDFA8248007800F027F9F9E07F4800785E
:100140000428D0D003217D480078EFF7F7FFC8B22C
:100150007A49087008460078401C087000207849E9
:100160000870FEF7E3FA7548007800F00DF9DFE05B
:100170000120FDF7F3FD00285AD0002071490870D6
:10018000FEF7D4FA0120FDF7FDFD6C480078012848
:100190000FD105216A480078EFF7D0FFC8B268494F
:1001A000087008460078401C087008460078FEF782
:1001B00061FF6248007802280FD10E216048007864
:1001C000EFF7BCFFC8B25E49087008460078401CD3
:1001D000087008460078FFF745F85848007803286B
:1001E00011D157490878C10F091849104900411A1F
:1001F000534A117010460078401C1146087008469A
:100200000078FFF7DDFB4D480078042895D10621E2
:100210004B480078EFF792FFC8B24949087008468A
:100220000078401C087008460078FFF77BFC7FE0F0
:100230000420FDF793FD002815D0002041490870E7
:100240000420FDF79FFD3D480078042870D0FEF79C
:100250006DFA01203949087039490870084600785C
:10026000FEF708FF64E00820FDF778FD002819D0AC
:10027000002034490870FEF759FA0820FDF782FD86
:1002800004202E49087000202D4908702B48007862
:1002900000F07AF800F034F9802108430446FFF7B3
:1002A0006BFE45E01120F6F7B3FB002812D00020CA
:1002B00024490870FEF73AFA1120F6F7BBFB01203B
:1002C0001E49087005201E49087008460078FEF790
:1002D000D1FE2DE00020F6F79BFB002812D0002075
:1002E00018490870FEF722FA0020F6F7A3FB042055
:1002F0001249087001201249087008460078FFF77B
:1003000011FC15E01020F6F783FB002810D0002028
:100310000C490870FEF70AFA1020F6F78BFB012053
:10032000064908700649087008460078FEF7A2FEE4
:1003300010BD0000FE0300208D7C6B5AFF030020DF
:1003400000040020FD03002001210C4A1170002848
:1003500009D00B4A11700B490978082291430831E2
:10036000084A117008E00021054A11700549097812
:1003700008229143034A117070470000C302002015
:10038000BE020020C402002070B50446FEF7CEF97C
:10039000002C17DD052C15DA00F0B2F80546FFF742
:1003A000EBFD12210320FFF7B1FD0A210420FFF726
:1003B000ADFD21460520FFF7A9FD12210620FFF71C
:1003C000A5FD0FE00E210320FFF7A0FD0E21042064
:1003D000FFF79CFD12210520FFF798FD0A2106205A
:1003E000FFF794FD70BD000010B52148007800288B
:1003F00002D0012836D123E01E480078012803D11D
:100400001D480078012807D11A480078022803D037
:1004100018480078032807D13C21012005F050FD41
:100420000120134908700AE012480078042806D118
:100430001249012005F044FD01200D49087015E026
:10044000012005F085FB00280BD101200949087027
:100450000949087008460078FEF70CFE00200449A0
:10046000087003E000200249087000BF00BF10BD03
:10047000FD030020FF03002000040020302A0000BC
:1004800001210C4A1170012809D10B4A11700B4946
:100490000978402291434031084A117008E0002158
:1004A000054A11700549097840229143034A1170A9
:1004B00070470000C3020020BC020020C4020020DC
:1004C00001210C4A1170002809D00B4A11700B4908
:1004D0000978102291431031084A117008E0002178
:1004E000054A11700549097810229143034A117099
:1004F00070470000C3020020BD020020C40200209B
:1005000010B50248EFF7E4FE10BD0000C402002061
:1005100010B509210020FCF7BFFD0A210020FCF7DF
:10052000BBFD0B210020FCF7B7FD0C210020FCF7E0
:10053000B3FD04218020FCF7AFFD05218020FCF7EE
:10054000ABFD00214020FCF7A7FD01214020FCF776
:10055000A3FD02214020FCF79FFD0C210120000398
:10056000FCF79AFD0D2101200003FCF795FD0E21FB
:1005700001200003FCF790FD0A214020FCF78CFDD0
:100580000B214020FCF788FD0C214020FCF784FD66
:100590000D214020FCF780FD0E214020FCF77CFD62
:1005A0000F214020FCF778FD0821C020FCF774FDE6
:1005B0000921C020FCF770FD0A21C020FCF76CFD6A
:1005C0000B21C020FCF768FD06218020FCF764FDAC
:1005D00007218020FCF760FD08218020FCF75CFDEE
:1005E00009218020FCF758FD08210020FCF754FD6C
:1005F00003214020FCF750FD04214020FCF74CFD76
:1006000005214020FCF748FD06214020FCF744FD71
:1006100010BD000007480078002809D1064800787E
:10062000002805D105480088002801D10120704725
:100630000020FCE7B8020020C3020020BA0200201C
:100640000D480078022805D10C480078022801D115
:100650000020704708480078042805D10748007832
:10066000002801D00020F4E705480078002801D0D8
:100670000020EEE70120ECE7FF030020000400204B
:10068000FC0300201FB5082102A80BF06FFB082116
:1006900068460BF06BFBFFF73BFF0121162007F0CC
:1006A0004FFB2E480090001401900F21490501983E
:1006B0008843019001210903019888430190019822
:1006C0000009000101904900019888430190490008
:1006D000019888430190490001988843019049009E
:1006E000019888430190890001988843019049004E
:1006F0000198884301904900019888430190684619
:1007000000F0D8FD012168460172032141720021E9
:100710008172C17203210173012141730021817330
:100720000121C17302A800F067FD00F057FD002011
:100730000B4908700B4908800B4908700B49087079
:100740000B4908700B4908700B4908700B49087079
:100750000B4908700B49EFF7D3FD1FBD0000FFFFE9
:10076000B8020020BA020020BC020020BD02002016
:10077000BE020020BF020020C0020020C1020020F3
:10078000C3020020C402002010B5002015490870E3
:100790001549087015490870FCF718F91449884282
:1007A00006D104201349087001201349087004E0A1
:1007B0000120104908701049087001200F49087085
:1007C00000200F4908700F4908700F4908700F4941
:1007D000087001200E49087000200E4908600E497B
:1007E000086010BDFC030020FD030020FE03002074
:1007F0008D7C6B5AFF0300200004002001040020C0
:100800000204002003040020040400200604002049
:10081000050400200C0400201804002010B502205C
:1008200005F096F9002814D10121022005F048FBBB
:10083000FEF732FAFFF7D8FD00F012FCF5F722FBC5
:10084000012803D10020FFF7DBFA02E00120FFF7C7
:10085000D7FAFFF731FC10BD10B5FE48007800282C
:1008600006D0012814D002287ED003287DD1FFE2D3
:10087000F9480078002803D1F8480088002806D0FD
:100880000120F449087007F01FFEF5490860D4E321
:10089000F1480078002869D0F2480078C107C90FF4
:1008A000F14840788006C00F81420BD0EE48407876
:1008B00020218843EB49097849012022114008434F
:1008C000E9494870E74800788007C10FE64840785A
:1008D0000007C00F81420DD0E348407808218843CB
:1008E000E04909788907C90FC90008221140084367
:1008F000DD494870DB4800784007C10FDA482030F6
:1009000080784007C00F81420FD0D74820308078D0
:1009100004218843D34909784907C90F8900042273
:1009200011400843D04920318870CE480078000734
:10093000C10FCD4840784007C00F81420DD0CA4852
:10094000407804218843C74909780907C90F8900FD
:10095000042211400843C4494870C2480078C006C8
:10096000C00FC149097B02E07EE265E3AAE1890785
:10097000C90F88420DD0BC48007B02218843B94989
:100980000978C906C90F4900022211400843B64937
:100990000873B44800788006C00FB3490979890705
:1009A000C90F88420DD0B048007902218843AD4973
:1009B00009788906C90F4900022211400843AA4953
:1009C0000871A84800784006C00FA749097A89072E
:1009D000C90F88420DD0A448007A02218843A1495A
:1009E00009784906C90F49000222114008439E496F
:1009F00008729C480078C0099B49097A4907C90FC9
:100A000088420DD09848007A042188439549097896
:100A10000906C90F8900042211400843924908724F
:100A2000904840788007C00F8F4909788907C90F1F
:100A300088420DD08C480078022188438949497842
:100A40008907C90F490002221140084386490870EE
:100A5000844840784007C00F834909784907C90F87
:100A600088420DD080480078042188437D49497828
:100A70004907C90F89000422114008437A490870C8
:100A8000784840780007C00F774909794907C90FAE
:100A900088420DD07448007904218843714949780F
:100AA0000907C90F89000422114008436E490871E3
:100AB0006C4880788007C10F6B484078C007C00F32
:100AC00081420AD0684840784008400065498978EA
:100AD0008907C90F08436449487062488078400715
:100AE000C00F6149097BC907C90F88420AD05E4817
:100AF000007B400840005B4989784907C90F0843DB
:100B000059490873574880780007C00F5649097A39
:100B1000C907C90F88420AD05348007A40084000EC
:100B2000504989780907C90F08434F4908724D4851
:100B30008078C006C00F4C490979C907C90F88429F
:100B40000AD0494800794008400046498978C906DA
:100B5000C90F084344490871424880788006C00F95
:100B600041490978C907C90F88420AD03E48007830
:100B7000400840003B4989788906C90F08433A4933
:100B80000870384880784006C00F37490978490610
:100B9000C90F88420DD0344800784021884331493C
:100BA00089784906C90F89014022114008432E491E
:100BB00008702C488078C1092B4820304078C00943
:100BC00081420FD028482030407880218843254931
:100BD00089780906C90FC9018022114008432249BA
:100BE000203148701F48C078C107C90F1E48203007
:100BF00040788006C00F81420DD01B4820304078DD
:100C0000202188431749C97849012022114008430F
:100C10001549203148701348C0788007C00F124929
:100C20000978C906C90F88420DD00F4800781021F5
:100C300088430C49C9788907C90F0901102211405E
:100C40000843094908700748C0784007C00F0649A3
:100C5000097B0BE0B8020020C3020020BA0200208A
:100C6000C8020020C4020020405C00404907C90FB0
:100C700088420DD0F248007B04218843F149C978AD
:100C80004907C90F8900042211400843EC49087341
:100C9000EC48C0780007C10FE9484078C00981429C
:100CA0000DD0E748407880218843E649C978090794
:100CB000C90FC901802211400843E1494870002052
:100CC000E1490870E148008800287DD0DF480078BD
:100CD000C007C00F00280DD0DC4800884008400045
:100CE000DA4908800020FDF757FDD949087800212E
:100CF000FDF708FED54800880221084000280CD0E6
:100D0000D24800888843D14908800120FDF744FD7E
:100D1000CF4948780121FDF7F5FDCC480088042132
:100D2000084000280CD0C94800888843C74908807B
:100D30000220FDF731FDC64988780221FDF7E2FD6A
:100D4000C24800880821084000280CD0BF4800880D
:100D50008843BE4908800320FDF71EFDBC49C878C2
:100D60000321FDF7CFFDB948008810210840002875
:100D70000CD0B64800888843B44908800420FDF7A9
:100D80000BFDB34908790421FDF7BCFDAF4800888D
:100D90002021084000280CD0AC4800888843AB498B
:100DA00008800520FDF7F8FCA94948790521FDF7E1
:100DB000A9FDA64800884021084000280ED0A3487D
:100DC00000888843A14900E046E008800620FDF73E
:100DD000E3FC9F4988790621FDF794FD9B48008834
:100DE0008021084000280CD0984800888843974903
:100DF00008800720FDF7D0FC9549C8790721FDF749
:100E000081FD92480088FF210131084000280CD064
:100E10008E48008888438D4908800820FDF7BCFC77
:100E20008B49087A0821FDF76DFD8848008801216B
:100E30004902084000280CD0844800888843834930
:100E400008800920FDF7A8FC8149487A0921FDF7AF
:100E500059FD00207D49088002207E49087007F076
:100E600033FB7D490860E8E003207A490870E4E03C
:100E700074480078C107C90F714840788006C00FD8
:100E800081427DD16F4800788007C10F6C4840785F
:100E90000007C00F8142F4D16A4800784007C10FB3
:100EA0006748203080784007C00F8142E9D165480B
:100EB00000780007C10F624840784007C00F8142A8
:100EC0005ED160480078C006C00F5D49097B890784
:100ED000C90F884254D15B4800788006C00F58493A
:100EE00009798907C90F88424AD1564800784006D7
:100EF000C00F5349097A8907C90F884240D1514828
:100F00000078C0094E49097A4907C90F884237D18C
:100F10004C4840788007C00F494909788907C90FB4
:100F200088422DD1474840784007C00F444909788E
:100F30004907C90F884278D1424840780007C00F5E
:100F40003F4909794907C90F88426ED13D488078E9
:100F50008007C10F3A484078C007C00F814264D172
:100F6000384880784007C00F3549097BC907C90F49
:100F700088425AD1334880780007C00F304900E0DA
:100F800053E0097AC907C90F88424ED12D488078AD
:100F9000C006C00F2A490979C907C90F884244D140
:100FA000284880788006C00F25490978C907C90FED
:100FB00088423AD1234880784006C00F20490978FA
:100FC0004906C90F884230D11E488078C1091C48A3
:100FD00020304078C009814227D11A48C078C10723
:100FE000C90F1748203040788006C00F81421CD1BD
:100FF0001448C0788007C00F11490978C906C90F85
:10100000884212D10F48C0784007C00F0C49097BB5
:101010004907C90F884208D10A48C0780007C10FA4
:1010200007484078C009814202D001200649087073
:1010300000200849087000E000BF00BF10BD00009C
:10104000405C0040C4020020C3020020BA0200201D
:1010500073140020B8020020C8020020704700006E
:1010600010B52848007801280FD1274800780028BB
:101070000BD026480078F6F747FB254909688842D7
:1010800003D021480078FDF7F5FF1E4800780228BC
:101090000FD11D48007800280BD01E480078F6F7C5
:1010A00053FB1D490968884203D017480078FEF7B2
:1010B000D9F81448007803280FD113480078002885
:1010C0000BD016480078F6F7BFFB1549096888422F
:1010D00003D00D480078FEF773FC0A480078042816
:1010E0000FD10948007800280BD00E480078F6F799
:1010F000F7FB0D490968884203D003480078FEF7E2
:1011000011FD10BDFF030020000400200804002092
:101110000C04002009040020100400200A04002010
:10112000140400200B040020180400207047000065
:1011300070B5049C8DB2002D05D0274D2D688EB260
:101140003543254E356095B2002D05D0224D6D6892
:1011500096B23543204E75609DB2002D05D01E4DD0
:10116000AD689EB235431C4EB560A5B2002D05D0CA
:10117000194DED68A6B23543174EF5600D0C2D04E0
:10118000002D06D0144D2D6A0E0C36033543124E39
:101190003562150C2D04002D06D00F4D6D6A160C0E
:1011A000360335430C4E75621D0C2D04002D06D000
:1011B000094DAD6A1E0C36033543074EB562250C4A
:1011C0002D04002D06D0044DED6A260C3603354360
:1011D000014EF56270BD0000405C004000210549F1
:1011E000002004E000220A60091D421CD0B2102831
:1011F000F8DB7047405C00402D4909680722520225
:1012000091430278520207235B021A401143284A95
:10121000116011460968DA10914342789201DB109F
:101220001A401143224A1160114609682022914355
:101230008278520120231A4011431D4A1160114641
:10124000096818229143C278D20018231A4011432A
:10125000174A11601146096806229143027952002B
:1012600006231A401143124A11601146496892152B
:10127000914342791202FF2301331A4011430C4A71
:10128000516011464968802291438279D2018023BE
:101290001A401143064A516011460968490849003D
:1012A000C279D207D20F1143014A11607047000082
:1012B000005C0040024A0168D160416811617047DA
:1012C000005C004010B510F049FA03E0F3F7F6FABD
:1012D000F3F722FC0EF0C2FF0028F7D100F084F9EA
:1012E00000210148017210BD4621002010B50648BA
:1012F00000F035F8002805D0034800F013F801206D
:101300000249087010BD0000000F0040DC02002000
:1013100010B5042007F050FB10BD10B5052007F0F4
:101320004BFB10BD10B50446002211462046143078
:1013300005F052FD10BD70B505460C462246002151
:1013400028460C3005F048FD70BD70B505460C46CA
:1013500022460A2128460C3005F03EFD70BD10B52E
:101360000446002120461030F6F7E8FA10BD30B5EB
:1013700002467D23DB00D0680724E402A0430C78FA
:10138000E4020725ED022C402043D060D0683024D1
:10139000A0434C78240130252C402043D060D068F5
:1013A00001246402A0438C78640201256D022C4064
:1013B0002043D060D0686C10A043CC7824026D101C
:1013C0002C402043D060D0680824A0430C79E4006E
:1013D00008252C402043D060D0680424A0434C79D9
:1013E000A40004252C402043D060D0680224A043F0
:1013F0008C79640002252C402043D06005E0D06841
:101400000006C00F002800D004E018465C1EA3B2FE
:101410000028F4D100BF002B01D1092030BD506855
:10142000000C00040C89204350600020F6E7000007
:101430000348C06A400840000149C8627047000084
:101440000024004010B5FFF7F3FF10BD10B507F002
:1014500072F800287ED0F1F781FD0028FAD004F060
:10146000DFFB0028F6D003F0FFF800287ED0F3F76A
:10147000E7FA00287AD0042007F092FB002875D004
:10148000052007F08DFB002870D0FCF797FC0028A2
:101490006CD0FFF7BFF8002868D0F9F7F9FD0028F5
:1014A00064D0FCF78DFB002804D10F20F5F7B0FACB
:1014B00001285BD1FCF78CFC002857D0F5F71EFC07
:1014C000002804D10F20F5F7A3FA01284ED1FFF729
:1014D000B7F800284AD0FBF77FFA002804D10F2084
:1014E000F5F796FA012841D106F034FE00283DD0E8
:1014F00006F052FD002804D10F20F5F789FA0128E3
:1015000034D100F0DFFD002804D10F20F5F780FA78
:1015100001282BD1F2F778F9002804D10F20F5F734
:1015200077FA012822D105F0CDFA002804D10F2046
:10153000F5F76EFA012819D1042007F0FFFD002805
:1015400014D0052007F0FAFD00280FD0042008F081
:10155000BDF800E00AE0002808D0052008F0B6F841
:10156000002803D0F3F798F9002801D1002010BD1E
:101570000120FCE710B5024600230020002100BF37
:101580000BE0074C0419237D002B04D0072902DA55
:1015900053544C1CE1B2441CE0B20A28F1DB10BDEC
:1015A000600E10001CB5072168460AF0DFFB012120
:1015B0006846417081700021C17001714171012143
:1015C00081716A460B2101200003FBF70DFD032208
:1015D0000B2101200003FBF7DDFC01220321022087
:1015E000F3F73CFD1CBD00000748006807490840B0
:1015F000884205D10448006880B20349086002E0CF
:101600000020014908607047247F002000005AA58F
:101610000248006880B2014908607047247F0020BA
:101620000548006805490840884203D1024800681F
:1016300080B270470020FCE7207F002000005AA500
:1016400007490968074A1140914202D01146044AED
:101650001160034909680143014A116070470000A5
:10166000207F002000005AA510B504F061FA022185
:101670000840022813D1012004F082FA032004F06C
:1016800015FC072004F012FC4A20F5F747FB012067
:101690000349087003490870062004F007FC10BDD8
:1016A000DA040020DB04002070B5044606F030FDAB
:1016B00005463A492846EFF777F90AD238492046D5
:1016C000EFF772F968D237492046EEF78AFE0446F2
:1016D00062E032492846EFF771F91FD832492846AF
:1016E000EFF762F91AD22E492046EFF767F90AD8C8
:1016F0002E492046EFF758F905D22D492046EEF73E
:1017000070FE044648E02B492046EFF757F943D8CE
:1017100029492046EEF765FE04463DE02749284664
:10172000EFF74CF90FD826492846EFF73DF90AD2D2
:101730001E492046EFF738F92ED822492046EEF709
:1017400050FE044628E01E492846EFF737F90FD827
:101750001D492846EFF728F90AD216492046EFF727
:101760002DF919D817492046EEF73BFE044613E041
:1017700015492846EFF722F90ED809492046EFF718
:101780001DF909D809492046EFF70EF904D2084996
:101790002046EEF726FE0446204670BDAE47834144
:1017A00000000841643B7F3FA470B3410000C84182
:1017B0004E62803F00003443EC51803FE17AE041CB
:1017C000A4700B428941803F9A9927420EB50C21A3
:1017D00068460AF0CBFA0021684601700821417082
:1017E0000321090341800121490281800021C18038
:1017F00001218903018100218172F1F71DFD0EBDD8
:1018000010B507210020FBF747FC00218020FBF7E3
:1018100043FC02218020FBF73FFC03218020FBF7E3
:101820003BFC10BD10B56048FCF758FF5F490870DD
:1018300008460078F1F718FA5C480078F0F7C4FA27
:101840005A480078EFF780FC5948007A030009F005
:1018500036FC3C1F2122235A5055A04B242526A09C
:10186000A0272829A046A02A2B2CA05FA0A041A039
:10187000643A3235377838872D823920692E2F34F3
:10188000367D6E303173A0A08C3391963B9B3CA08B
:1018900000BF00BF00BF00BF00BF00BF00BF00BF50
:1018A00000BF00BF00BF00BF00BF00BF00BF00BF40
:1018B00000BF00BF00BF00BF00BF00BF00BF00BF30
:1018C00000BF00BF00BF00BF00BF38480078F1F77D
:1018D000D3F85FE035480078F0F72CFB5AE0334846
:1018E0000078F0F7C3FB55E030480078EFF7CCFB09
:1018F00050E02E480078EFF74FFB4BE02B48007884
:10190000EFF7B8FA46E029480078EFF7F1FD41E03B
:1019100026480078F0F764FC3CE024480078F0F7B3
:1019200087F837E021480078EFF76EFE32E01F4875
:101930000078F0F717F82DE01C480078F1F7FAF876
:1019400028E01A480078F0F7D1F923E0174800782A
:10195000F1F75AFA1EE015480078F0F7DBF819E0C5
:1019600012480078F0F756F914E010480078F1F7C3
:101970002BF90FE00D480078F0F7CAFB0AE00B489E
:101980000078F1F743F905E008480078EFF74CFDDF
:1019900000E000BF00BF054800780649087001213B
:1019A000044802F077FF10BD00400040DC06002034
:1019B000AF280020EF2E002030B503460C46154618
:1019C000002D10D115480360154804801548C07ECD
:1019D000012802D102F060FA01E0F2F733FD0020A5
:1019E0001149087012E0012D07D11048036010481A
:1019F0000480012008F048FC08E0022D06D10D48C3
:101A000003600D480480022008F03EFCB0200B4922
:101A1000087002200A49087030BD0000400500200F
:101A2000440500208823002056050020480500209A
:101A30004C05002050050020540500202A050020F8
:101A40002905002010B50022052101200003FBF725
:101A500031FB00200149087010BD00003005002056
:101A600010B5012205211003FBF724FB01200149D9
:101A7000087010BD3005002070B50546002D04D05B
:101A8000012D05D0032D22D11EE01348C07970BD71
:101A9000002611484A304078002803D00E484A30CA
:101AA00046780FE000240BE00B48801CEEF710FC9A
:101AB000E040C007C00F002801D0701CC6B2641CF3
:101AC000202CF1DB3046E2E70448007ADFE700BF74
:101AD00000BF0020DBE70000FC200020323F002098
:101AE00070B505460C46002D04D0012D05D0032D00
:101AF00016D112E00C48C47113E006F0DBF90A4974
:101B0000891C2046EEF7FCFB002107484A30417053
:101B1000012105200FF006FE03E00448047200E0F6
:101B200000BF00BF70BD0000FC200020323F00203D
:101B300010B5FFF787FF002005494876487788777A
:101B4000C877B0200349087000200349087010BD11
:101B5000882300202A050020290500201CB5072124
:101B600068460AF003F9002168464170012181703E
:101B70000021C17001714171012181716A46052105
:101B800001200003FBF730FA6A4604218802FBF7C4
:101B90002BFA6A46032101200003FBF725FA6A4667
:101BA0000221C802FBF720FA0022052101200003D0
:101BB000FBF780FA00220221C802FBF77BFA002221
:101BC00004218802FBF776FA00220321012000039A
:101BD000FBF770FA1CBD000070B586B0684603F0D4
:101BE000F9FFCA48EEF774FBC949884214D2C748C6
:101BF0004638EEF76DFB0646E1210901EEF788FA5B
